:1080000000000020BD870000758500008585000008
:108010008585000085850000858500008585000038
:108020008585000085850000858500008585000028
:108030008585000085850000858500007599000014
:108040008585000085850000858500008585000008
:1080500085850000858500008585000085850000F8
:1080600085850000858500008585000085850000E8
:1080700085850000858500008585000085850000D8
:1080800085850000858500008585000085850000C8
:1080900085850000858500008585000085850000B8
:1080A00085850000858500008585000085850000A8
:1080B0008585000085850000858500008585000098
:1080C0008585000085850000858500008585000088
:1080D0008585000085850000858500008585000078
:1080E0008585000085850000858500008585000068
:1080F00085850000858500008585000005950000C8
:108100008585000085850000858500008585000047
:108110008585000085850000858500008585000037
:108120008585000085850000858500008585000027
:108130008585000085850000CDE70000858500006D
:108140008585000085850000858500008585000007
:1081500085850000858500008585000085850000F7
:1081600061ED0000858500008585000085850000A3
:1081700085850000858500008585000085850000D7
:1081800085850000858500008585000085850000C7
:1081900085850000858500008585000085850000B7
:1081A00025DC000095DC000085850000993D01007C
:1081B0008585000085850000858500008585000097
:1081C0008585000085850000858500008585000087
:1081D0008585000085850000858500008585000077
:10840000FFFFFFFFFFFFFFFFFFFFFFFF7EFFFFFFFD
:1084100010B5054C237833B9044B13B10448AFF3BE
:1084200000800123237010BD2821FF1F00000000E1
:1084300044A801000C4B43B10C480D4910B5AFF3F3
:1084400000800C48036823B910BD0A48036833B99B
:108450007047094B002BF7D0BDE810401847064B7A
:10846000002BF5D0184700BF0000000044A8010011
:108470002C21FF1F2821FF1F0000000000280346B9
:10848000B8BF00F11F035B11012B2BD0022B15D0BD
:1084900003B170471D4A434203F01F03D2F8801115
:1084A00000F01F0058BF5842012303FA00F00143B7
:1084B000C2F880111368184310607047134A434292
:1084C00003F01F03D2F8881100F01F0058BF584274
:1084D000012303FA00F00143C2F88811936818439E
:1084E00090607047094A414201F01F0100F01F00EF
:1084F00058BF4842D2F8841103FA00F00143C2F891
:108500008411536818435060704700BF00E100E0D9
:1085100080281ADC40280FDC20281FDC434203F0AF
:108520001F0300F01F00124A58BF5842012303FAEC
:1085300000F0C2F88000704700F01F0001230C4AD1
:1085400003FA00F0C2F88800704700F01F00012312
:10855000074A03FA00F0C2F88C00704700F01F00D1
:108560000123034A03FA00F0C2F88400704700BFF9
:1085700000E100E0684620F007018D4601B401BC2F
:1085800085467047684620F007018D4601B4FFBE5E
:1085900001BC8546704700BF4FF0E020F0B5364B78
:1085A000364A374CC0F8084D41F244053549364F3C
:1085B0004CF220544DF628164FF4E970D481D68140
:1085C00041F23804108059511A59304E304831491F
:1085D00042F4D0521A515E5141F248042E4E1A59BB
:1085E00022F00F0242F002021A5141F204024FF04F
:1085F000240E9C5844F480349C501D6825F40025BA
:108600001D60856C3D408564C46C80253C40C4641D
:1086100081F801E03570985820F001009850A223AD
:108620000B70CB78032403F01F030020CB700A46A5
:108630000C71487193799807FCD5164A9379D9063D
:10864000FCD4144A937903F00C03082BFAD140238D
:10865000104953718B7903F00C03082BFAD10D4AA2
:1086600093795B06FCD522230A4913708B7903F0BA
:108670000C030C2BFAD1F0BD007004400020054023
:108680000080000000003301FFF8FFFE000013012E
:1086900000900440004006400050064080F31188DE
:1086A000704700BFF0B41A4D1A4C2B691A4E1B4A82
:1086B0001B481C4923F0807323F4E06341F2140744
:1086C00043F4E0632B610025E55104F582531C68F7
:1086D00044F004041C60336823F0784323F0010362
:1086E0003360137803F08C0343F050031370537816
:1086F00003F09C0343F040035370937803F0EC03C2
:108700009370857081F8145385F31188F0BC70471D
:10871000009004400070044000D0004000D00740AA
:1087200000E0074000E100E0E2B140EA010313F09D
:10873000030F07D1032A05D951F8043B40F8043B45
:10874000043AF1E7DB0707D4012A05D931F9023BE6
:1087500020F8023B023AE7E711F8013B00F8013B41
:10876000013AE1E7704700BF704700BF884201D07F
:1087700002B1D9E7704700BF10B50C4C24B913E023
:1087800070B9A3688BB10C34216860680029F7D0F8
:108790008142A268F7D0002AF5D0FFF7C5FFF2E7C3
:1087A000A268002AEFD0F8E710BD10BDDCC90100B7
:1087B000704700BF704700BF704700BF10B5FFF79C
:1087C000F7FF1D4CFFF7E8FE2046002807D085463E
:1087D00081B04FF000006FEA0000009001B0174B2D
:1087E000174AD21A0AD0002113F0030012D1032A2B
:1087F00010D9043A43F8040B002AF5D1FFF7BCFF67
:10880000FFF7DAFF0F4900200FF076FD0E4B1860DE
:108810008047FEE713F0010007D1012A05D0023A94
:1088200023F8020B002ADFD1E8E7013A03F8011B25
:10883000002AD9D1E2E700BF000000202821FF1F55
:10884000B486FF1F4421FF1F9838FF1F08B5FFF7AC
:10885000B5FF00BF70B40D4B00220726082501208C
:1088600002214FF4FA741E705D7158709A701A717B
:108870009A711A755A759A75DA75D9701C62986072
:108880001A619A61DA61D96070BC70477438FF1F51
:10889000304B314AF0B506219A65FA260A25082799
:1088A000C8244FF4967247F230505E61DD614FF498
:1088B0007A664FF4FA7583F8251083F8297005213C
:1088C0004FF4FA671C669A6401240022D8654FF4BD
:1088D0007A701E605E60DE639D601D635D631C6276
:1088E00083F8244083F82C40588540F2FF74D86404
:1088F0004FF4827E7826D96019619F619F634FF49F
:10890000C87583F8262083F8272083F8282083F869
:108910002D20A3F8402083F842205A6483F8542085
:10892000186547F6FF7083F8642083F82E2083F8DB
:10893000692083F86A20A3F86E10A3F86CE09E67A4
:10894000DD67A3F87040A3F87240A3F87400A3F8A1
:108950007600F0BDF037FF1FC0B85900F0B5514D9B
:108960005149524A41F238044FF480702B5943F474
:1089700000732B510860C8605369002043F008035E
:108980000825536104462E460A2156604FF47A7337
:1089900000BF013BFCD113699560DF0748BF01347C
:1089A0004FF47A7300BF013BFCD11369DB0758BF5A
:1089B00001300139E9D10A2C3B4C3A4B3C4EDFF8EF
:1089C00018E13C4F41F238024FF4E0652560E56064
:1089D0009C5818BF084644F4806437499C504FF4B3
:1089E00081754FF480740D65CC60756925F4801530
:1089F00075610E6D314D26F020060E650E6D46F048
:108A000002060E650E6D26F001060E65995841F4BA
:108A100000619950CEF83C40CEF840409E5828491D
:108A200046F480569E506E6946F040066E612E6890
:108A300026F040062E60BC619E58224D224F46F41F
:108A400000569E504A69214E42F004024A61AC60D1
:108A50002F666E660C681E4E1E4A41F22C0524F0ED
:108A600004040C605C59B6F8721044F480545C51F4
:108A700092F8213043F0800382F8213092F82130BF
:108A800008BF0A38C1F3032443F04003C9B282F897
:108A9000213008BFB0FA80F05470117008BF40094F
:108AA000F0BD00BF007004400090044000F00F4093
:108AB00040F00F4000C0044000A00440C0F00F4050
:108AC00000F10F4000D004400001090000010A003D
:108AD000F037FF1F00C00C4000B00440044B054AB3
:108AE000B3F87230C3F30321DBB2517013707047D7
:108AF000F037FF1F00C00C402DE9F04F974CDFF816
:108B00007CC2974EDFF878E29648DFF87882964B81
:108B10009649974F41F23C0541F23009625942F0C3
:108B20000062625154F8092042F0006244F80920C2
:108B30000022CCF824204FF00D0ACCF82C204FF066
:108B40001009F2614FF0040CCEF80420012604F560
:108B5000825EC0F808A0C8F808A0C0F80C90C8F859
:108B60000C90C0F820C0C8F820C04262C8F8242089
:108B70000660C8F80060DEF8009049F00209CEF8FF
:108B8000009054F805A003F5845941F2840E4AF090
:108B9000020A4FF0B60B44F805A00A7141F28C05A9
:108BA00081F804B041F29004C9F8007041F2940ACF
:108BB00041F2980923F80E606FF0030B41F2880E22
:108BC00043F805B00126185141F29E0523F80A200A
:108BD00041F2960443F8092041F2860041F29C09D3
:108BE00043F80E6003F5855E23F805C0614E23F857
:108BF00004C041F2A4051A5241F2AC0423F8092042
:108C000041F2B0004FF0A8094A7141F2B40A81F86C
:108C10000590CEF8006041F2B80941F2A80E564E18
:108C20005A531A5141F2BE051E5002206FF007063A
:108C300023F80A0041F2B60443F8096043F80E0035
:108C400048F6040E23F805E041F2A60948F20405AF
:108C50001D5341F2BC0E40F2011423F8094040F2CA
:108C6000224923F80E90D3F80CE0434E03F58659C1
:108C700067444EF0200E4FF0B80AC3F80CE00836F7
:108C80008A7141F2C40E81F806A0C9F8007041F261
:108C9000CC0734464FF0010623F80E6041F2D009AC
:108CA00043F807B041F2D40E41F2D80743F80980E7
:108CB00041F2C80A23F80E2041F2DE09DA5141F2EE
:108CC000D60841F2C60E41F2DC0701264FF0A90B8F
:108CD00043F80A6023F809C003F5875623F808C053
:108CE00041F2E40A23F80E2041F2EC09DA5341F292
:108CF000F008CA7181F807B001F51A2141F2F40CAD
:108D000041F2F80E41F2E8071031316041F2FE0BFA
:108D100023F80A2041F2F60643F8092041F2E60161
:108D200043F8084041F2FC0A6FF0070423F80C00F6
:108D300048F6044943F80E4040F22262D85140F20E
:108D4000011023F80B909D53585223F80A20DA683B
:108D500042F08002DA6062B6BDE8F08F0070044035
:108D600000A0044000B0034000800040001002401A
:108D70000800FF1F10B003406C21FF1F00B004402B
:108D800000C0044000B00B400249034A01230B60BD
:108D90001360704700B0034000B00B40704700BF45
:108DA000704700BF704700BF704700BF704700BFEB
:108DB000704700BF704700BF704700BF704700BFDB
:108DC00009490A4B4A6922F480124A611A6D22F05D
:108DD00020021A651A6D42F002021A651A6D42F0FD
:108DE00001021A65704700BF40F00F4000A0044028
:108DF00009490A4B4A6922F480124A611A6D22F02D
:108E000020021A651A6D42F002021A651A6D22F0EC
:108E100001021A65704700BF40F00F4000A00440F7
:108E2000094B0A4A596941F480115961116D21F0C9
:108E300002011165116D41F0200111651A6822F4DB
:108E400080121A60704700BF40F00F4000A004403D
:108E5000024B1869C0F30050704700BF40F00F404C
:108E60000020704701280ED008D3022804D1084BF7
:108E70001869C0F30050704700207047054B18690F
:108E8000C0F3C0307047034B1869C0F3004070470F
:108E900040F00F4080F00F40704700BF704700BFA8
:108EA0000020704705281CD8DFE800F0070B0F13DF
:108EB00017030D4B588880B270470B4B988980B2CE
:108EC0007047094B588980B27047074B188980B2A8
:108ED0007047054B188880B27047034BD88980B221
:108EE00070470020704700BF6C21FF1F03281BD86C
:108EF000DFE800F0140E08020C4A0D4B927A33F8AA
:108F000012007047094A0A4B527A33F81200704730
:108F1000064A074B127A33F812007047054A044B91
:108F2000127C33F812007047002070470800FF1FC2
:108F30009C38FF1F6C21FF1F032808D8DFE800F0D2
:108F4000140E08020B4A0C4B927A23F81210704749
:108F5000084A094B527A23F812107047054A064B0B
:108F6000127A23F812107047044A034B127C23F83C
:108F7000121070470800FF1F9C38FF1F6C21FF1F55
:108F80000E490B690A6910B50C699209C3F30023F5
:108F900002F00202E408134304F004041C4306D068
:108FA000072C04D0202000F02BFF204610BD012804
:108FB000F8D1202000F01CFFF7E700BF80F00F4041
:108FC00038B50D4C0D4DB4F87410687AFFF7B4FF46
:108FD000B4F87610A87AFFF7AFFFB4F87010287ACB
:108FE000FFF7AAFFB4F87230054AC3F30321DBB2DE
:108FF0005170137038BD00BFF037FF1F0800FF1F0E
:1090000000C00C40024B4FF480425A60704700BFD2
:1090100000F00F40024B4FF480429A60704700BF4F
:1090200000F00F40014B04225A60704700F10F40DE
:10903000014B04229A60704700F10F40024B186800
:10904000C0F38000704700BF00F10F40704700BFC1
:10905000704700BF704700BF704700BF024B4FF41E
:1090600080625A60704700BF40F00F40024B4FF4DF
:1090700080629A60704700BF40F00F40014B402271
:109080005A607047C0F00F40014B40229A60704711
:10909000C0F00F4070B5254A254B2648264C41F2BA
:1090A000380641F23C01955945F4007595515558E3
:1090B00045F480555550555825F4802555505A6C27
:1090C00042F400725A641A6C42F400721A64DA6B49
:1090D00042F40072DA639A6B42F480729A634369D5
:1090E000012243F4804343612260236843F000433C
:1090F00043F440632360FFF785FF4FF06053E36064
:10910000E36843F02003E360E36843F48033E36003
:10911000E36A43F08053E362236823F00103236092
:10912000236823F00063236070BD00BF007004401B
:109130000090044000F00F4000C00240F0B422490B
:10914000224A234C234B244E244D41F23807C85960
:1091500040F48060C85141F23C000F5847F400577A
:109160000F500F5827F480270F50516C41F40071B5
:109170005164116C41F400711164D16A41F40071C1
:10918000D162916A41F4807191626269012142F475
:109190008062626119601A6842F0004242F44062E3
:1091A0004FF480611A606160DE601D61DA6A42F02E
:1091B0008052DA621A6822F001021A601A6822F0FC
:1091C00000621A60F0BC70470070044000A00440C8
:1091D00040F00F4000D002400100523E0100F23E3C
:1091E00070B50C4616460546002833D001281ED11E
:1091F000FFF72EFF1B4BEEB144F000645C63DA6AAC
:10920000D200FCD5DA6A42F08052DA62DA6A12F0F1
:10921000F00FFBD09C6B1A6842F44062E4B21A6013
:10922000E5B1012D01D1FFF711FF204670BD0E4BB6
:10923000002EE1D144F000445C63DA6AC2F30332E9
:10924000032AFAD8DA6A12F0F00FFBD09C6BE4B272
:10925000204670BDFFF7DEFE034BCCE7FFF7D2FEE2
:10926000204670BD00D0024000C00240012870B509
:1092700005460C4616463AD035D3022820D1FFF7D2
:10928000EBFE214BFEB144F000645C63DA6AD2006D
:10929000FCD5DA6A42F08052DA62DA6A12F0F00F34
:1092A000FBD09C6B1A68012D42F44062A4B21A6094
:1092B00025D020D3022D01D1FFF7CCFE204670BD72
:1092C000124B002EDFD144F000445C63DA6AC2F333
:1092D0000332032AFAD8DA6A12F0F00FFBD09C6B43
:1092E000A4B2204670BDFFF795FE084BCAE7FFF712
:1092F000AFFE054BC6E7FFF785FE204670BDFFF7C2
:10930000A5FE204670BD00BF00D0024000C0024054
:10931000134AA8B14FF000635363D36ADB00FCD556
:10932000D36A0F4943F08053D362CB6A13F0F00F36
:10933000FBD0886B0B6843F4406380B20B607047CE
:109340004FF000435363D36AC3F30333032BFAD8BC
:10935000034AD36A13F0F00FFBD0906B80B27047D2
:1093600000D00240F8B5364B98423CD0354B98427D
:1093700041D0354B984253D0344B984258D0344B5F
:1093800098421DD0072A96BF324B4FF4165353F81C
:1093900022300029B8BF0F310911B1FBF3F1C1F33D
:1093A0000423C9B203704170C37843F02C03C37027
:1093B0002F20FFF763F8284B302283F82F23F8BDC6
:1093C000264F274C41F228064FF44075BB5943F411
:1093D0008063BB51256600236566C370837083710B
:1093E000C3724371CEE71D4D41F234042B5943F44F
:1093F00080632B51C6E7A3F5103341F2340641F2E6
:1094000038079C59164D44F400649C51DC594FF4C4
:10941000407644F40054DC512E6000236E60DCE79B
:109420000E4D41F234042B5943F480532B51A9E7DC
:109430000A4D41F234042B5943F400532B51A1E758
:1094400000A0064000B0064000C0064000D0064024
:1094500000A00E40C488010000E100E0007004405C
:1094600000D00440024602490248FFF77BBF00BF1C
:1094700000D8B80500B006400A4A136851680133A5
:10948000202B08BF00238B420AD010B41168064C71
:10949000114408721360E37843F08003E37010BC5A
:1094A000704700BF8021FF1F00B006400B4B996A38
:1094B000DA6A91420FD09A6A511C1A44996292F862
:1094C00030109A6A0170202A01D0012070470022D2
:1094D0009A62012070470020704700BF8021FF1F63
:1094E000044A137803F0FF0013B100231370012026
:1094F000704700BFA838FF1F014B1865704700BFB9
:109500008021FF1F684620F007018D4631B52A49AA
:109510000C79E4B2A00615D5284AD36A906A0133C3
:10952000202B08BF0023834206D0D06ACD791118C2
:10953000E8B281F83000D3622149224B052008604F
:10954000126D1A60620625D4230603D4BDE83140AB
:10955000854670471B4B1D68002DF7D1174C2268BC
:1095600063689A421ED0FFF75DFD6368124A591C7A
:10957000234461601B7ADBB2D37163680E4A202BEF
:1095800008BF6560D37843F04003D370BDE8314035
:1095900085467047FFF74CFD074AD37803F0BF03B9
:1095A000D370D1E7044AD37803F07F03D370BDE8CA
:1095B00031408546704700BF00B006408021FF1F44
:1095C000AC38FF1FB038FF1FF8B52D4C2D4F617020
:1095D000002241F23C062270BD592B4B45F000752C
:1095E000BD515D6D45F004055D651D6825F01805EC
:1095F0001D605D6D25F001055D65D3F8845001386F
:1096000045F0C005C3F88450DA645A609860D3F816
:10961000802042F00102C3F88020D3F8802049B3B3
:1096200022F02002C3F88020D3F8802022F010021C
:10963000C3F88020144A134D516D144B144E41F061
:1096400001015165116841F2380041F008011160D3
:109650002A584FF4C06142F4806240272A501960B2
:1096600058205960C3F8A0709E61FEF707FF0123E0
:109670002370F8BD42F02002C3F88020DAE700BF73
:10968000D421FF1F007004400090034000A004405C
:1096900000010900024A034B11801860704700BFA7
:1096A000B838FF1FB438FF1F014B1880704700BF48
:1096B000B838FF1F014B1860704700BFB438FF1F58
:1096C000084B187820B1084B586880B2C0EB0040B6
:1096D000064B074A1B881268B0FBF2F000FB03F050
:1096E00080B27047D421FF1F00900340B838FF1F9D
:1096F000B438FF1F034B187808B1034B586880B289
:10970000704700BFD421FF1F00900340014B5888D1
:10971000704700BFD421FF1F024B0022D8645A605B
:10972000DA64704700900340014B1879704700BF1E
:10973000D421FF1F014B00221A717047D421FF1F53
:10974000014B1870704700BF2000FF1F014B1878B5
:10975000704700BF2000FF1F014B9860704700BF9B
:10976000D421FF1F014B9868704700BFD421FF1F11
:10977000014B187B704700BFD421FF1F024B012211
:1097800018611A7358697047D421FF1F38B50C4C03
:1097900025690122290C0220FFF768FDA9B20122E8
:1097A0000220FFF763FD074B05465988012202207E
:1097B000FFF75CFD002340EA05402373606138BD7C
:1097C000D421FF1F2000FF1F704700BF014B1883EB
:1097D000704700BFD421FF1FF0B4114D114B41F26F
:1097E000380420272A59802642F400624FF4807101
:1097F0002A51C3F8A070C3F8A060C3F8A01030B914
:1098000059615920D961F0BC1962FEF737BE064A8A
:109810005A615920DA61F0BC1A62FEF72FBE00BF10
:109820000070044000B0044000010B0008B5FFF7D1
:10983000A7FB0138C0B205289ABF024B33F91000CC
:10984000002008BDE488010038B500F13B03762B09
:109850000B4C08D80020208042F6AA22094906F0C5
:1098600087F8208038BD2388074D01FB02F1800373
:1098700095FBF1F190FBF1F0181A00B22080EBE7B4
:10988000F421FF1F56D5FFFFE0930400014BB3F90D
:1098900000007047F421FF1F884210D0204B0022A7
:1098A00001381A80052808D8DFE800F033210327A3
:1098B0002D1A012932D0022916D0002070478B1EA4
:1098C000042BFAD801A252F823F000BFEF98000051
:1098D000B3980000FB98000007990000E198000091
:1098E00002291BD00429E8D14FF0FF30704703292B
:1098F00014D00629F8D00020704706290ED005297B
:10990000F2D000207047042908D00129ECD00020B3
:109910007047052902D00329CFD1E5E70120704720
:10992000F421FF1F014B5860704700BFF421FF1F57
:10993000014B5868704700BFF421FF1FFEF7B2BE0D
:10994000044B0548002207211A6058609A6019608C
:10995000704700BF10E000E000770100014B0022DB
:109960001A60704710E000E0014B1868704700BFB4
:10997000FC21FF1F684620F007018D460E490F4A63
:109980000B6801B5106801330B6020B11368013B0F
:10999000136013685BB10A4B1A6812B11A68013A76
:1099A0001A600AF0D1F8BDE8014085467047054BC2
:1099B00001221A70EFE700BFFC21FF1FAC38FF1F28
:1099C000B038FF1FA838FF1F044B00221A619A61AC
:1099D0001A629A621A639A63704700BF008003405C
:1099E0005D4AF8B541F23C0441F2380115595B4B30
:1099F00045F080751551155945F480051551545899
:109A000044F400645450545844F4805454505A6DF3
:109A100042F004025A65002879D1D3F884205049D5
:109A2000504C42F0C002C3F884205A6D40F6C31572
:109A300042F061025A659D60D864D3F88C2042F0F0
:109A40008002C3F88C209A6D42F002029A659A6DEA
:109A500042F080029A650A883F20024018665C66E0
:109A60009A66FFF7B1FF3D4B3F49DA683F48404EE9
:109A7000404C42F00802DA605A6942F008025A612A
:109A8000DA6942F00802DA615A6A42F008025A6260
:109A9000DA6A42F00802DA625A6B2A2742F00802B8
:109AA0004FF400755A631F67C3F89850DA6E42F09E
:109AB0004002DA665A6D42F002025A651D6840F2B1
:109AC0000442002745F008051D6042608260C260C4
:109AD000026132617261CF600A6842F40A6242F048
:109AE000010240F6C3100A6048601F661A683E20F3
:109AF00042F040021A60FEF7C1FC302384F83E3386
:109B00004820FEF7BBFC202384F84833F8BD5A6D8B
:109B10001349144842F061026FF49C6440F2E1453D
:109B20005A659D60DC649A6D42F002029A659A6DF6
:109B30003F2442F080029A651C665866088840F20D
:109B400071226FF41C712040986619619A61196244
:109B50009A6219639A6386E70070044000800340AC
:109B60001400FF1F737373000060034000B00440D3
:109B700000C0044000E100E0014B3F221A6670473C
:109B80000080034058B1064B6FF41C7140F2712203
:109B900019619A6119629A6219639A63704713E7AF
:109BA00000800340F0B444F2A8324DF6F00510FBFB
:109BB00002F310FB25F5EC1A2B445A1082B04FEA41
:109BC000640143D40029C0F2838002F51C52103294
:109BD000521A44BF02F57F3202F2FF32002CBCBFA2
:109BE00004F57F3404F2FF349214181EB8BF00F558
:109BF0007F3002F2E24292B2B8BF00F2FF3002EBD5
:109C0000A444A2EBA040A4B280B20225624B197812
:109C1000012907D16149624F0A8000264C80888063
:109C20003D701E705F4963085208400857425E420B
:109C300045424FF400748A610F618B620E62886343
:109C40000D63C1F8984002B0F0BC704700291DDBDD
:109C5000002D5EDDC5F51C5110318A1844BF02F598
:109C60007F3202F2FF329214002BB8BF03F57F332C
:109C700002F2E24292B2B8BF03F2FF33A2EBA34377
:109C800098B200EB65439CB20325BFE702F51C5276
:109C90001032521A44BF02F57F3202F2FF32002C1A
:109CA000BCBF04F57F3404F2FF349214002BB8BF1C
:109CB00003F57F3302F2E24292B2B8BF03F2FF3300
:109CC00002EBA444A2EBA343A4B298B205259DE7FE
:109CD000002D41DD05F51C521032521A231E4FEAA9
:109CE000A242B8BF03F57F3302F2E242B8BF03F2EB
:109CF000FF3392B2281EB8BF00F5FF3002EBA3433A
:109D00009CB2B8BF00F2FF10A4EB604080B2012506
:109D10007CE705F51C521032521A44BF02F57F321F
:109D200002F2FF329214231EB8BF03F57F3302F212
:109D3000E242B8BF03F2FF3392B2281EB8BF00F56B
:109D4000FF3002EBA3439CB2B8BF00F2FF10A4EBBC
:109D5000604080B2042559E7C5F51C5110310A4412
:109D6000002B4FEAA242B8BF03F57F3302F2E24272
:109D7000B8BF03F2FF3392B2002DB8BF05F5FF352F
:109D8000A2EBA343B8BF05F2FF1598B200EB654301
:109D90009CB206253AE700BF0022FF1FBC38FF1F18
:109DA0002A00FF1F00800340014B01221A707047F8
:109DB0000022FF1F014B33F810007047BC38FF1F13
:109DC000064A074B1088518892880844104483FB48
:109DD0000023A3EBE07080B2704700BFBC38FF1FC8
:109DE00056555555014B1878704700BF2A00FF1F84
:109DF000024A136818431060704700BF0422FF1F17
:109E0000024A136823EA0000106070470422FF1F13
:109E1000044A136819B923EA000010607047184318
:109E2000106070470422FF1F034B1B68034214BFDE
:109E300001200020704700BF0422FF1F024A136860
:109E400023F06D03136070470422FF1F034B186853
:109E50001A6822F06D021A60704700BF0422FF1FCB
:109E6000044B18681A6822F06D0200F06F001A6047
:109E7000704700BF0422FF1F2DE9F041174F184D16
:109E8000184E04463878FFF70DF880463878FFF70B
:109E90002DF8294647F6FF72A8EB000005F068FD93
:109EA00007B23078FEF7FEFF80463078FFF71EF8E5
:109EB0002946A8EB000047F6FF7205F059FD06B2EF
:109EC000B819294647F6FF72404205F051FD278038
:109ED000A08066802046BDE8F08100BF1100FF1F12
:109EE0000180FFFF1200FF1F38B5084C2078FEF7F5
:109EF000D9FF05462078FEF7F9FF47F6FF72281ACA
:109F00000021BDE8384005F033BD00BF1000FF1F41
:109F1000002210B5032104461046FFF761F9002224
:109F2000C4F307211046FFF75BF90022E1B21046A7
:109F3000FFF756F9002108460122BDE81040FFF75F
:109F40004FB900BF38B5012204460D460020062156
:109F5000FFF746F9002210460521FFF741F90021DD
:109F600001220846FFF73CF98207F3D5002210468C
:109F70000221FFF735F900221046C4F30721FFF74D
:109F80002FF90022E1B21046FFF72AF929460122F3
:109F90000020FFF725F9002210460521FFF720F9E0
:109FA000002108460122FFF71BF9C307F3D438BD8F
:109FB000F8B51646002204460D4610460321FFF769
:109FC0000FF90022C4F307211046FFF709F9002218
:109FD000E1B21046FFF704F97EB1013D771E00247F
:109FE0003A1B0021B2FA82F208465209FFF7F8F84C
:109FF0000134A64205F8010FF2D1F8BD2DE9F04178
:10A0000004460E461746062101220020FFF7E8F815
:10A01000002210460521FFF7E3F80021084601223F
:10A02000FFF7DEF88107F3D5002210460221FFF783
:10A03000D7F800221046C4F30721FFF7D1F8002219
:10A040001046E1B2FFF7CCF8002F4AD0013E0025C0
:10A0500007F1FF380AE0A8EB0502B2FA82F25209D2
:10A060000020FFF7BDF80135AF423AD0013414F0BB
:10A070003F0016F8011FEED10122FFF7B1F8A84505
:10A08000F1D9002210460521FFF7AAF80021084661
:10A090000122FFF7A5F810F00100F2D101220621FC
:10A0A000FFF79EF8002210460521FFF799F80021DE
:10A0B00001220846FFF794F88207F3D500221046E4
:10A0C0000221FFF78DF800221046C4F30721FFF7A5
:10A0D00087F800221046E1B20135FFF781F8AF4260
:10A0E000C4D1002210460521FFF77AF80021084666
:10A0F0000122FFF775F8C307F3D4BDE8F08100BF74
:10A1000038B50D46C0EBC00404F500600978FFF7D0
:10A1100019FF697804F60100FFF714FFA97804F627
:10A120000200FFF70FFF297904F60300FFF70AFF8B
:10A13000697904F60400FFF705FFA97904F6050024
:10A14000FFF700FFE97904F60600BDE83840FFF7A5
:10A15000F9BE00BF002238B50C46C0EBC005032194
:10A160001046FFF73DF805F500650022C5F307210D
:10A170001046FFF735F80022E9B21046FFF730F835
:10A18000002211461046FFF72BF8002211462070DE
:10A190001046FFF725F80022114660701046FFF7C1
:10A1A0001FF800221146A0701046FFF719F8002290
:10A1B000114620711046FFF713F800221146607116
:10A1C0001046FFF70DF80021A07101220846FFF7A5
:10A1D00007F8E07138BD00BFF0B5002283B00D462E
:10A1E000C0EBC00403211046FEF7FAFF04F500643B
:10A1F0000022C4F307211046FEF7F2FF0022E1B26D
:10A200001046FEF7EDFF002211461046FEF7E8FF6C
:10A210000022114606461046FEF7E2FF00221146D4
:10A2200004461046FEF7DCFF0022114607461046A2
:10A23000FEF7D6FF002211468DF804001046FEF707
:10A24000CFFF002211468DF805001046FEF7C8FF2B
:10A2500000218DF8060001220846FEF7C1FF8DF8A7
:10A2600000608DF80140BDF800202B888DF80700B4
:10A270009A4202D0002003B0F0BDAB78BB42F9D1C6
:10A280006B680198C01AB0FA80F04009F3E700BF8C
:10A2900038B54FF40065012206210020FEF7A0FF2B
:10A2A000002210460521FEF79BFF002101220846EF
:10A2B000FEF796FF8207F3D5002210460221FEF733
:10A2C0008FFF00221046C5F30721FEF789FF002209
:10A2D0001046E9B2FEF784FF0024A4F13F020021FA
:10A2E000B2FA82F2084652090134FEF779FF402C97
:10A2F000F3D1002210460521FEF772FF0021084627
:10A300000122FEF76DFFC307F3D44035B5F5804F4A
:10A31000C1D138BD70B5054640F2FF700C461646F7
:10A32000FFF7F6FD912821D0002140F2FF70FFF7E2
:10A3300009FEFFF7ADFF242229460020FFF75EFE4D
:10A34000214640208022FFF759FE912140F2FF7004
:10A35000FFF7F8FD294624220020FFF729FE2146B9
:10A3600080224020BDE87040FFF722BE002EDBD1E6
:10A37000F0E700BFF0B51D4C1D4FA569E369DFF89C
:10A3800074E003FB05F387FB0327421ADE17002A5C
:10A39000C6EB6736B8BF5242B242B8BF44F620633C
:10A3A000DEF80060B8BF5343114A334482FB0362B6
:10A3B000DF175213A2EB070C44F6206606FB1C3392
:10A3C000CEF8003085B1884208DB0EDD2168BA1A6C
:10A3D000494210448842B8BF0846F0BD2168604435
:10A3E0008842A8BF0846F0BD0846F0BDF037FF1F01
:10A3F000AD8BDB680822FF1F2DE9F84F5C4D95F807
:10A4000025E02E68BEF1060F0746884691461C4699
:10A4100002D0BEF1000F73D195F82900D7F800B033
:10A4200040080DF0F7FA5946824658460DF046FBB3
:10A4300050490DF043FB014650460DF03FFB82466C
:10A44000A869C0EB0010C0000DF0E4FA01465046C8
:10A450000DF0E8FB0DF086FDA4EB09024C45B8BFFA
:10A460007642002AB8BF524290424FEAE27371EB43
:10A4700003034FF48040A8BF0026FFF7D5FC012856
:10A4800058D030460DF0C6FA3C688046014620465A
:10A490000DF0B2FCC8B1002E38D1EB69A86903EB0E
:10A4A000830203EB420300FB03F00DF0B3FA3249E1
:10A4B0000DF0B8FB014620460DF0F8F9044638606F
:10A4C00020460DF0C1FCBDE8F88F414620460DF056
:10A4D000B1FC0028F4D00EB3AB69E86900FB03F0CF
:10A4E0000DF098FA25490DF09DFB014620460DF030
:10A4F000DBF90446386020460DF0A6FCBDE8F88F75
:10A50000BEF1070F20D000200021A5E7AB69E86964
:10A5100000FB03F00DF07EFA1849C9E7EB69A86962
:10A5200003EB830203EB420300FB03F00DF072FA2E
:10A530001149D8E740460DF06DFA044638602046D0
:10A540000DF082FCBDE8F88F016808460DF0B6FA00
:10A550000B490DF067FB0DF005FDEB6BAA698E460C
:10A56000A3FB000103FB0E11D3170DF093FC73E75F
:10A57000F037FF1F0000C0400050434800409C4699
:10A580000000F042014B1878704700BF0C22FF1FFB
:10A59000014B1870704700BF0C22FF1F38B50E4DDD
:10A5A000AB6C1361401A00231446536110600B49D1
:10A5B0004FF6FF7205F0DCF92369206003FB00F021
:10A5C00000282A68B8BFFF300012A0615142BDE8E0
:10A5D000384005F0CDB900BFF037FF1F0100FFFF85
:10A5E0002DE9F84F394FD7F84C803E6D5661C2F8CF
:10A5F0001080144697F82520054699464AB9B8F1C7
:10A600000003B8BF0733002EB8BF03364FEAE30894
:10A61000B610681A20602E494FF6FF7205F0A8F9AF
:10A62000D4E902AB616920601AEB000A4BEBE07BD6
:10A63000C4E902AB71B34FEA094292FBF6F2514210
:10A64000504605F095F92368824603FB08F34FEA6C
:10A65000E07B002BC4E902AB80FB06ABB8BFFF3345
:10A66000BAF1000F4FEA23207BF100031EDB4FEA13
:10A670001A4343EA0B431844A06197F82530082B8E
:10A680000ED1002D08DDB86BBD6F000290FBF5F018
:10A69000BDE8F88F0A46D3E710D12846BDE8F88F09
:10A6A0004A465142BDE8F84F05F062B94FF6FF72D5
:10A6B00000231AEB020A4BEB030BD8E7B86BBD6F14
:10A6C000000290FBF5F04042BDE8F88FF037FF1F25
:10A6D0000100FFFF2DE9F04114460E461A4659428B
:10A6E00005F046F9244A136B516B2361002BB8BF68
:10A6F0000733DD10D4E90223801B00298846B8BF48
:10A7000001F10308161843EBE077616120604FEA1E
:10A71000A808C4E9026739B3184A92FBF8F251421B
:10A72000304605F025F9236803FB05F3002B0646A8
:10A730004FEAE07780FB0801B8BF03F2FF3300283F
:10A7400071F10002C4E902674FEAA3230EDB000C9B
:10A7500040EA01401844A06140F6C312084905F0E0
:10A7600007F900B2BDE8F0810A46D9E74FF6FF7657
:10A77000002780197941EAE7F037FF1F0000C3097D
:10A780003DF6FFFFF8B514460D461A46594205F04E
:10A79000EFF8D4E902231F4E00B2451B716B306BFA
:10A7A0002061561943EBE57725606161C4E90267D2
:10A7B00039B3194A92FBF1F25142304605F0D8F80C
:10A7C0002269236803FB02F36269002B06464FEA05
:10A7D000E07780FB0201B8BFFF33002871F100026F
:10A7E000C4E902674FEA23230DDB000C40EA014075
:10A7F0001844A06147F6FF72084905F0B9F800B2A5
:10A80000F8BD0A46D9E74FF6FF760027801979414F
:10A81000EBE700BFF037FF1F0000FF7F0180FFFF65
:10A8200082B02DE9F04F1DB21C1487B005EBD57630
:10A8300004EBD475B94CDDF864E0139F01977610F2
:10A84000A680159E05966D10169EE5800296179EB1
:10A8500004968146189E606811930EEBDE7703968E
:10A86000DFF8CC82149D8A46934605F0D1F8019B0F
:10A870001E6898F82530A06006EBD676063B7F1060
:10A8800046F34F06032B00F22181DFE813F0B500F9
:10A89000F9005E0004000020FEF7C8FF98F82820A9
:10A8A000012A834600F070815846FFF73BF8029B6F
:10A8B0001B68029318460DF0C7FAD8F8142080EAF6
:10A8C000E07EAEEBE07E964580F20C8198F8293070
:10A8D000D8F820609249934A0EFB03F006FB00F083
:10A8E000000381FB0013C117C1EB6311236A1944F4
:10A8F00082FB01325211CB17D61A642000FB1610CE
:10A90000206200210298049303920DF093FA00282C
:10A9100000F01382039A049BE18BD8F838609B1AED
:10A920000B449BB203F58041E38309B23302F60185
:10A93000D8F8782093FBF2F3019A7B481360D8F89B
:10A94000783096FBF3F636B26BE0029BD3F800B09A
:10A9500058460DF079FA98F829307149714A80EA21
:10A96000E07EAEEBE07E03FB0EF0D8F8203003FB78
:10A9700000F0000381FB0013C117C1EB6311236AD0
:10A98000194482FB01325211CB17D01A4FF0640EDA
:10A990000EFB101E039000215846C4F820E00293DD
:10A9A00001920DF047FA002800F0A980019A029B5D
:10A9B000E18B9B1A0B449BB203F58041E38309B200
:10A9C000594805F015F9C0F30F4328806B8001202A
:10A9D000FEF72CFF98F82830012B00F0DB80FEF703
:10A9E000A1FFFEF76DFEA0F5FF407F3800B2FEF735
:10A9F000B3FE4FF0000B1CE00120FEF717FF98F8A4
:10AA00002E20012A834600F0CA8098F82820012AC7
:10AA10007ED05846FEF786FF0020FEF79DFE424896
:10AA2000594605F0E5F8C0F30F4328806B804FF0DE
:10AA3000000B3B464A46B5F900103046FFF7A2FE30
:10AA40003B46208252465846B5F90210FFF79AFE5F
:10AA5000237860827BBB238AA384344805F000F806
:10AA6000324805F027F82A886B88A06252005B0004
:10AA70002A806B8007B0BDE8F04F02B0FFF792B8B4
:10AA8000FEF764FE012855D0FEF71AFE98F82C3028
:10AA9000A0F5FF407F38012B0FFA80F800F04781C6
:10AAA0000020FEF73FFF4046FEF756FE41461E4897
:10AAB000A4F81E80B5E7A18C21820022002300218A
:10AAC000C9E902236182CAE90223C6E700211648C8
:10AAD00005F08EF84FF0000BC0F30F4328806B8019
:10AAE0005E46A6E75946104805F082F8C0F30F42CB
:10AAF000A4F81EB028806A804FF0000B99E75846F2
:10AB000000210DF079F9002857D1B4F91E1057E74C
:10AB10000BF5FF437F330FFA83FB7AE70C22FF1F0D
:10AB2000F11976051F85EB511422FF1F1C22FF1F10
:10AB3000F037FF1F4FF48060FFF776F9012811D03E
:10AB40004FF40070FFF770F9012801D1049B4BB955
:10AB50004FF40060FFF768F90128B7D1019B1B682B
:10AB6000002BB3D098F82C30012B00F03C81C0F0C2
:10AB7000FE80022B40F02C816369032B3FF657AF18
:10AB8000DFE803F0A445242400F5FF437F330FFAE8
:10AB900083FB89E600F5FF407F3000B21FE798F89D
:10ABA0002910D8F8202003984908FEF74DFEFEF73B
:10ABB0006DFE83440FFA8BFB27E7E38B039A1A445D
:10ABC00093B2A3F58041E38309B2F9E65846002623
:10ABD0002682668205F078F8484605F075F85046FA
:10ABE00005F072F80599626900230B600299022A48
:10ABF0000B6000F0B4818020FFF7FAF80020FEF728
:10AC000091FEA069FEF7A8FDB4F918105FE7D4F82B
:10AC100018B098F829308BEAEB715B08C3EB03425C
:10AC2000A1EBEB71914280F29581D8F86010D8F8D1
:10AC30002020CF4E01FB03F3C2EBC23202FB03F331
:10AC4000B8F8662086FB0316B2F5007F4FEAE3737F
:10AC5000C3EBA64600F09481B2F5806F00F09081BE
:10AC6000B2F5006F00F0AC81E368D8F83820C14835
:10AC7000D8F878104FEAC21B9BFBF1FB03FB0BFBE0
:10AC8000A0FB0B3B0020FEF74DFEA069FEF764FD24
:10AC9000B4F91810B84804F0ABFFB8F86630288053
:10ACA000B3F5007FC0F30F404BF34F3B688000F0DB
:10ACB0007981B3F5806F00F0758198F8423013F018
:10ACC000020332D102221E466261B2E6E26842F21B
:10ACD00010739A4200F23081D8F83830A548D8F87D
:10ACE000781001324FEAC31B9BFBF1FB02FB0BFB0D
:10ACF000A0FB0B3B0020E260FEF714FE0020FEF7F5
:10AD00002BFD00219C4804F073FFB8F866302880C2
:10AD1000B3F5007FC0F30F404BF34F3B688000F06A
:10AD20003C81B3F5806F00F03881002681E618463B
:10AD3000FEF77CFDFEF7F6FDB5E6029800210DF06A
:10AD40005BF820B90646B4F91E100346F0E5E28B25
:10AD5000D8F83800324492B2C0EB0063A2F58041CB
:10AD6000C0EB4060E28309B21B02C601E0E5E36884
:10AD700042F2107201339342E36000F2A180D8F8EE
:10AD800038207C48B8F86610D8F878604FEAC21BC3
:10AD90009BFBF6FB03FB0BFBA0FB0B3BB1F5007F22
:10ADA0004BF34F3B00F08780B1F5806F00F083805C
:10ADB0000020FEF7B7FD0020FEF7CEFC00216E4814
:10ADC00004F016FFC0F30F4328806B80002630E6A6
:10ADD0000021694804F00CFF0026C0F30F432880CF
:10ADE0006B80B34625E618460393FEF7C9F8014683
:10ADF0000290207FFEF750FD039B029A01901846B7
:10AE00002277FEF713FD98F82820012A034604BF95
:10AE100000F5FF437F3318460293FEF783FD019B45
:10AE2000002B029B76DB39D003F515435433B8F978
:10AE30003C1098F829205148520803FB01F393FB7A
:10AE4000F2F380FB03201844DB17C3EBE03080B241
:10AE5000FEF762FCFEF734FC00230FFA80F8584638
:10AE600023826382019304F02FFF484604F02CFFF5
:10AE7000504604F029FF019B1846FEF761FC4FF491
:10AE80000040FEF7B5FFA8F5FF437F3B0FFA83F8BC
:10AE90004046FEF761FC41463748C2E50120FEF717
:10AEA000C5FC98F82830012B41D000F5FF437F33D3
:10AEB0000FFA83F8E7E7019A4FEA4B03136077E74D
:10AEC00000231846E360FEF727FC98F82C302BBBD4
:10AED00098F8423043F0010388F8423058464FF06A
:10AEE000000BA4F810B0A4F812B004F0EDFE484630
:10AEF00004F0EAFE504604F0E7FE059A00231360D2
:10AF0000029A58461360FEF71BFC4FF40040FEF710
:10AF10006FFF8EE503F5D5432A3388E7022BDDD199
:10AF200098F8423043F0020388F84230D6E700F543
:10AF3000FF437F3318B2B8E70020FEF7EDFB98F827
:10AF40004230012243F0020388F8423062614FF040
:10AF5000000B6EE5032363614FF0000B69E530469B
:10AF6000FEF7EEFB4FF40040FEF742FF46E600BF5F
:10AF7000851DD96F5917B7D11422FF1F018000809A
:10AF8000029B1B680293184600210CF053FF029BA2
:10AF900060B1ABEB0606A66166E6019B0026C3F82E
:10AFA00000B046E5019BC3F800B086E618460021D4
:10AFB0000CF022FF00283FF457AE5E44A66153E632
:10AFC000019B1B68002BE4DC3FF44EAEF5E700BFAD
:10AFD000024B00225A61DA609A6170470C22FF1F0F
:10AFE000014BB3F91E0070470C22FF1F08B5054B3B
:10AFF000054918600422FEF7DBFF044B01221A709A
:10B0000008BD00BFEC3CFF1FF03CFF1F3822FF1FB4
:10B01000024A136801331360704700BFF03CFF1F02
:10B020002DE9F04B2D4B2E4D1E6ADA6D2D4C2E4F17
:10B0300080EAE07EAEEBE07E85FB0E314FEAEE73F8
:10B04000C3EB21130EFB03F085FB0013C017C0EB0D
:10B05000231306FB03F3D4E9020187FB037E02EB13
:10B060008207DB176268C3EBEE0310EB030B02F100
:10B0700001024FEA8707B7FBF6F6A5FB063641F15A
:10B08000000CB2EB561FC4E902BC626023DBD4F8AB
:10B090001080DFF85890676959F8286000234FF452
:10B0A000C872584661460CF045FF08F1010185FB66
:10B0B0000135CB17C3EB651500220023BE1BC4E985
:10B0C0000223642303FB15150644002349F82800D6
:10B0D000666125616360BDE8F08B00BFF037FF1F3C
:10B0E0001F85EB513822FF1F67666666F43CFF1F21
:10B0F000014B5869704700BF3822FF1F014B186889
:10B10000704700BFF03CFF1F014B1860704700BF45
:10B11000F03CFF1F054B1B78012B00D07047044B00
:10B12000044918680422FEF769BF00BF3822FF1FD8
:10B13000EC3CFF1FF03CFF1F044B93F8643003B15D
:10B1400070474FF40030FEF75BBE00BFF037FF1FC3
:10B15000431E18B100BF13F1FF33FBD2704700BF8D
:10B1600041F238010E480F4A435830B443F480632B
:10B170000D4C43504FF48075A56453694FF4802102
:10B180000B43536142F23413916000BF013BFCD189
:10B19000044A536923F48023536130BC704700BFD5
:10B1A0000070044040F00F4000A00440F8B5384D56
:10B1B000384C394F00232B70FEF7DEFCFDF730FED4
:10B1C00041F2380135486658354B364A46F4006638
:10B1D0006650665846F4805666504FF48071416060
:10B1E0008160C160016139617961596941F01E0175
:10B1F0005961516941F030015161196821F0020132
:10B200001960196821F008011960116821F0100116
:10B210001160196841F004011960196841F01001CA
:10B220001960136843F02003136042F2341300BF27
:10B23000013BFCD141F2380116481B4C43581B4AD4
:10B2400043F4806343504FF48076A66453694FF40F
:10B2500080210B43536142F23413916000BF013BE4
:10B26000FCD1124A536923F48023536142F2341310
:10B2700000BF013BFCD10A490C4A4B6923F004038F
:10B280004B615369012143F4802353612970F8BD58
:10B290005022FF1F0070044000C0044000B0044072
:10B2A00080F00F40C0F00F4000A0044040F00F407D
:10B2B000014B1878704700BF5022FF1F064B074A0A
:10B2C0001B691B0703D4936801339360704753686D
:10B2D00001335360704700BF40F00F405022FF1F02
:10B2E000084909484B688A681A44A0FB020203EB2C
:10B2F000830300205B0052094860B3FBF2F38860CF
:10B30000CB6070475022FF1F1F85EB51014BD8685F
:10B31000704700BF5022FF1F0023194640FA03F276
:10B3200012F0010F03F1010318BF01310F2BF5D10A
:10B33000CB0754BF40F40040C0F30E00704700BF7D
:10B340000023194640FA03F212F0010F03F1010342
:10B3500018BF01310F2BF5D181EAD03000F0010088
:10B36000704700BF204B2149F0B500224FF48025E3
:10B370001024DFF87CE09D60074626461046202515
:10B380004FF0010C47FA02F3DB078E6040F25233B4
:10B390004CBFCEF80450CEF8085000BF013BFCD1A2
:10B3A0004C6040F2A91300BF013BFCD10B695B0765
:10B3B00003D50CFA02F3184380B240F2A91300BF80
:10B3C000013BFCD10132102ADCD10849084B8A60CC
:10B3D00020229A6040F2523300BF013BFCD1024B65
:10B3E0004FF480225A60F0BD40F00F4080F00F40D3
:10B3F000C0F00F4038B5002485B22946234641FAF3
:10B4000003F212F0010F03F1010318BF01340F2BF7
:10B41000F5D1E30754BF45F40045C5F30E052846B2
:10B42000FFF7A0FF42F2341300BF013BFCD12846D6
:10B43000BDE83840FFF796BF0220FFF7DBBF00BF33
:10B440000320FFF7D7BF00BF0420FFF7D3BF00BF23
:10B4500070B520F48055ADB2002104460B4645F48A
:10B46000006040FA03F212F0010F03F1010318BF6C
:10B4700001310F2BF5D1C80745BF46F6FF752540B2
:10B4800045F4084545F400652846FFF76BFF6A4B15
:10B4900000BF013BFCD124F40066B6B246F48050F4
:10B4A0001A4640FA02F111F0010F02F1010218BF31
:10B4B00001330F2AF5D1D90745BF47F2FF7020406D
:10B4C00046F4104040F48050FFF74CFF002319462B
:10B4D00040FA03F212F0010F03F1010318BF01312A
:10B4E0000F2BF5D1C0F3CF364E40F643420406F0A1
:10B4F000010648BF46F0020683040BD4684046F0BC
:10B50000040610F4FE6FB6B202D046F00806B6B2DA
:10B51000304670BD2D0985EA10104006F5D1002E89
:10B52000F6D142F2341300BF013BFCD11A4644F479
:10B53000C05040FA02F111F0010F02F1010218BFF0
:10B5400001330F2AF5D1D9074ABFC4F30E0044F4E2
:10B55000184040F4C050FFF705FF00210B4640FAA9
:10B5600003F212F0010F03F1010318BF01310F2B99
:10B57000F5D181EAD03111F0010F08BF1026420445
:10B5800044BF46F02006B6B283040BD485EA1015FA
:10B5900046F040066906B6B2BAD046F08006B6B2AA
:10B5A000304670BD85EA10104206F6D1002EAFD1AC
:10B5B00042F2341300BF013BFCD124F4C0501A46C0
:10B5C00080B240FA02F111F0010F02F1010218BF3E
:10B5D00001330F2AF5D1DB074ABF46F2FF7040F472
:10B5E00000402040FFF7BEFE00210B4640FA03F268
:10B5F00012F0010F03F1010318BF01310F2BF5D138
:10B6000081EAD03111F0010F08BF4FF48076410478
:10B6100044BF46F40076B6B2820458BF46F4806652
:10B6200085EA101558BFB6B26B061CBF46F400661B
:10B63000B6B2304670BD00BF1C7E06004FF6FA73EE
:10B64000034043F00200FFF703BF00BF4FF6FB7358
:10B65000034043F00300FFF7FBBE00BF4FF6FC734F
:10B66000034043F00400FFF7F3BE00BF10B54B7872
:10B6700082B0FE2B00F2A986DFE813F04606CA0569
:10B68000BD05B3052304A7060F04FB03A706E703C4
:10B69000FA04E6047606DD04A706A706A706A706B1
:10B6A000A706A70679036A03A706A706A706FD054E
:10B6B000560359054B058A06A7064305A706A706A4
:10B6C000A706A706A706A706A706A706A706A70612
:10B6D000A706A706A706A706A706A706A706A70602
:10B6E0009B0625062F06AD039206E40553065B0470
:10B6F00011030803FF02A706A706A706A706A706C9
:10B70000A706A706A706A706A706A706A706A706D1
:10B71000A706A706A706A706A706A706A706A706C1
:10B72000A706A706A706A706A706A706A706A706B1
:10B73000A706A706A706A706A706A706A706A706A1
:10B74000A706A706A706A706A706A706A706A70691
:10B75000A706A706A706A706A706A706A706A70681
:10B76000A706A706A706A706A706A706A706A70671
:10B77000A706A706A706A706A706A706A706A70661
:10B78000A706A706A706EB028B05A706A706A7062E
:10B79000A706A706A706A706A706A706A706A70641
:10B7A0007705A706A706A7066D056305DE03A706AE
:10B7B000A706D203C903A706A706B503A706BE04BA
:10B7C000A706AA04A70679046504A706A706A70684
:10B7D000A706A706C9044203A7062E031A032F05CE
:10B7E0001B051106A706A706A706A706A706A70614
:10B7F000A706A706A706A7060E05D705A10395036A
:10B8000089034F044304F005370439069F05A90551
:10B81000E2027302A7065F02A706A706A2024B0276
:10B8200098018F019902A70687010702FD01D60240
:10B83000F1016901A706A706A706A706A706A7069E
:10B840006101A70690025901DD01A706A706A70618
:10B85000C9017C02A706B50123020F02A706370221
:10B86000A706A7067401A706A706A706A70646010E
:10B870003301A10120010D01FF00052800F084879C
:10B88000062800F0F087072801F09280082800F0D1
:10B890004F8702B010BD052800F0FA86062801F097
:10B8A0009680072801F0A2800828F2D1CE49012213
:10B8B000692002B0BDE81040FEF77ABB052800F011
:10B8C000B386062801F0FD80072801F01F810828B3
:10B8D000DFD1C64901226E2002B0BDE81040FEF75C
:10B8E00067BB052800F0C086062801F008810728FC
:10B8F00001F014810828CCD1BD4904227C2002B07B
:10B90000BDE81040FEF754BB052800F0DF8606288E
:10B9100000F0C787072801F0BD800828B9D1B549D4
:10B9200001226C2002B0BDE81040FEF741BB0628A2
:10B93000AFD1019203F05EFA019A5060A9E70628A0
:10B94000A7D1019202F03CFF019A5060A1E70528BF
:10B9500000F0348706289CD10192FFF775FD019A0B
:10B96000506096E7052800F0C586062801F084801F
:10B97000072801F04B8008288BD19F4902226A20BA
:10B9800002B0BDE81040FEF713BB062881D101923A
:10B99000FFF7BCFC019A50607BE706287FF479AF83
:10B9A0000192FDF7DFFE019A506072E706287FF4EE
:10B9B00070AF0192FDF7BCFF019A506069E705285E
:10B9C00000F0BE86062800F03987072801F01680AF
:10B9D00008287FF45EAF894901226D2002B0BDE8DE
:10B9E0001040FEF7E5BA052800F03486062801F07D
:10B9F0007F80072801F06C8008287FF44AAF8049D7
:10BA00000122AA2002B0BDE81040FEF7D1BA0528F5
:10BA100000F03486062800F0D387072801F0608004
:10BA200008287FF436AF774904228C2002B0BDE8A5
:10BA30001040FEF7BDBA052800F02B85062801F05E
:10BA40009380072801F0088008287FF422AF6E4910
:10BA50000422882002B0BDE81040FEF7A9BA0528EC
:10BA600000F0988606287FF414AF0192FFF7E8FCF7
:10BA7000019A50600DE705287FF40BAF03F0AAF997
:10BA800002B0BDE81040FFF791BB05287FF401AF7D
:10BA900002B0BDE81040FFF763BB052800F00C863C
:10BAA000062800F05187072800F03F8708287FF418
:10BAB000F0AE56490222AE2002B0BDE81040FEF7BB
:10BAC00077BA052800F0A685062800F0F387072836
:10BAD00001F0688008287FF4DCAE4D490222AC20DA
:10BAE00002B0BDE81040FEF763BA052800F0F88503
:10BAF000062800F0DD86072801F0DC8008287FF4A6
:10BB0000C8AE44490422A02002B0BDE81040FEF7B0
:10BB10004FBA052800F0C685062800F00E870728D2
:10BB200000F0AF8608287FF4B4AE3B490422BC2065
:10BB300002B0BDE81040FEF73BBA052800F097843C
:10BB4000062800F02087072800F0A38608287FF445
:10BB5000A0AE32490122A92002B0BDE81040FEF794
:10BB600027BA06287FF495AE019203F05BF9019A9B
:10BB700050608EE6052800F0C785062800F0838710
:10BB8000072800F08F8708287FF483AE2449042219
:10BB9000902002B0BDE81040FEF70ABA06287FF4F4
:10BBA00078AE019203F020F9019A506071E6062800
:10BBB0007FF46FAE0192FFF713FA019A506068E6C6
:10BBC000052800F0AB85062800F0EB86072800F07A
:10BBD0004B8708287FF45DAE12490422B82002B0DA
:10BBE000BDE81040FEF7E4B91938FF1F1E38FF1FEB
:10BBF0002C38FF1F1C38FF1F1A38FF1F1D38FF1F6E
:10BC00005A38FF1F3C38FF1F3838FF1F5E38FF1FB0
:10BC10005C38FF1F5038FF1F6C38FF1F5938FF1F5B
:10BC20004038FF1F6838FF1F052800F0F3850628FD
:10BC30007FF42FAE0192FFF7FFFB019A506028E6D8
:10BC400006287FF426AE019203F0E6F8019A5060D0
:10BC50001FE6052800F07184062801F024800728DB
:10BC600001F0308008287FF414AECB4904225C2018
:10BC700002B0BDE81040FEF79BB906287FF409AE7C
:10BC8000022002F04BF8C54B586002E606287FF40C
:10BC900000AE012002F042F8C04B5860F9E50628DA
:10BCA0007FF4F7AD002002F039F8BC4B5860F0E5A6
:10BCB000052800F0E583062800F06C86072800F0D0
:10BCC000FE8508287FF4E5ADB5490222B22002B016
:10BCD000BDE81040FEF76CB9052800F091840628F5
:10BCE00001F00F80072800F0FD8708287FF4D1AD10
:10BCF000AC490222B02002B0BDE81040FEF758B9AE
:10BD0000052800F03884062800F09A87072800F0FC
:10BD1000E18708287FF4BDADA3490422742002B056
:10BD2000BDE81040FEF744B9052800F0CD83062891
:10BD300000F0FC86072800F0CA8508287FF4A9AD2A
:10BD40009A490422982002B0BDE81040FEF730B9AD
:10BD5000974C94F82F309A0740F13B830120FDF770
:10BD600081F801280FD08D4B00225A6091E5904C4C
:10BD700094F82F3013F0010000F037830020FDF716
:10BD800071F80128EFD1854B01225A6081E5052821
:10BD900000F0488506287FF47CAD019203F0F8FBA3
:10BDA000019A506075E5052800F0D08406287FF4DC
:10BDB00070AD019203F0E6FB019A506069E5052839
:10BDC00000F0D08406287FF464AD019203F0D4FB28
:10BDD000019A50605DE506287FF45BADFDF7F0FF4A
:10BDE0006E4B586055E5052800F0F683062800F0F4
:10BDF0004C87072800F01C8708287FF44AAD6D495E
:10BE00000122652002B0BDE81040FEF7D1B8062837
:10BE10007FF43FAD0192FEF719F8019A506038E5C2
:10BE2000052800F0B28306287FF433AD019202F0BA
:10BE3000FFF9019A50602CE506287FF42AAD0192A3
:10BE400002F034FA019A506023E5052800F0A78338
:10BE5000062800F00487072800F0F98608287FF4F8
:10BE600018AD55490422502002B0BDE81040FEF73D
:10BE70009FB8052800F0BA83062800F03B87072802
:10BE800000F0808608287FF404AD4C490422482045
:10BE900002B0BDE81040FEF78BB8052800F0028321
:10BEA000062800F06886072800F0748608287FF4CA
:10BEB000F0AC43490422442002B0BDE81040FEF734
:10BEC00077B8052800F00983062800F03686072891
:10BED00000F03A8608287FF4DCAC35490422402083
:10BEE00002B0BDE81040FEF763B8052800F05A84A0
:10BEF00006287FF4CEAC019203F062FB019A5060F9
:10BF0000C7E4052800F0548406287FF4C2AC0192EF
:10BF100003F04AFB019A5060BBE4052800F05C8402
:10BF200006287FF4B6AC019203F038FB019A50600A
:10BF3000AFE406287FF4ADAC224B1878FCF7B2FFD3
:10BF4000164B5860A5E4052800F06382062800F02F
:10BF50007F82072800F0DC8608287FF49AAC1A4913
:10BF600001226F2002B0BDE81040FEF721B805287D
:10BF700000F07482062800F07D84072800F0EC852C
:10BF800008287FF486AC11490222802002B0BDE867
:10BF90001040FEF70DB800BF0C38FF1FD838FF1F48
:10BFA0006238FF1F6038FF1F2438FF1F4838FF1F0B
:10BFB000F037FF1F1538FF1F0038FF1FF837FF1F2E
:10BFC000F437FF1F1200FF1F1F38FF1F3038FF1FFD
:10BFD000052800F0D383062800F03E84072800F0EF
:10BFE0002F8208287FF455ACD3490122942002B057
:10BFF000BDE81040FDF7DCBF052800F0FF830628F0
:10C00000ECD1019203F088F9019A506041E40528CF
:10C0100000F0A782062800F0DC85072800F0CA851A
:10C0200008287FF436ACC5490422702002B0BDE870
:10C030001040FDF7BDBF06287FF42BAC019202F043
:10C0400027F9019A506024E4052800F0348206287C
:10C0500000F08A84072800F08E8408287FF419AC49
:10C06000B7490422582002B0BDE81040FDF7A0BF38
:10C07000052800F06C82062800F0A485072800F04F
:10C080003C8408287FF405ACAE4904224C2002B061
:10C09000BDE81040FDF78CBF052800F06983062835
:10C0A0007FF4F7AB019203F05BFA019A5060FFF75F
:10C0B000F0BB052800F0B681062800F04C84072864
:10C0C00000F02B8408287FF4E4AB9F490222B420BF
:10C0D00002B0BDE81040FDF76BBF052800F01882E4
:10C0E000062800F07D85072800F08A8508287FF45F
:10C0F000D0AB96490422782002B0BDE81040FDF78D
:10C1000057BF05287FF4C5AB02B0BDE8104002F070
:10C11000D7BA052800F08C83062800F096830728FC
:10C120007FF4B7AB02B0BDE81040FEF7F3BF0628BE
:10C130007FF4AFAB0192FEF7DBFF019A5060FFF78F
:10C14000A8BB06287FF4A5AB019202F0A9F8019ADA
:10C150005060FFF79EBB06287FF49BAB019202F074
:10C16000E9FA019A5060FFF794BB052800F02A8293
:10C17000062800F08385072800F0788508287FF4DA
:10C1800088AB73490122642002B0BDE81040FDF77E
:10C190000FBF052800F0AA81062800F0A083072819
:10C1A00000F03E8508287FF474AB6A4904226020C1
:10C1B00002B0BDE81040FDF7FBBE06287FF469AB76
:10C1C000019202F01DFE019A5060FFF762BB062843
:10C1D0007FF45FAB019202F019FE019A5060FFF705
:10C1E00058BB06287FF455AB019202F09DFA019AE4
:10C1F0005060FFF74EBB052800F0DB8106287FF476
:10C2000048AB019202F09EF9019A5060FFF741BBE2
:10C21000052800F0A18206287FF43BAB019202F0D2
:10C220008BF9019A5060FFF734BB052800F0CE82ED
:10C2300006287FF42EAB019203F098F9019A506022
:10C24000FFF727BB052800F0DB8006287FF421AB31
:10C25000FEF798F9404B5860FFF71BBB052800F02C
:10C26000C78206287FF415AB019203F0A3F9019A67
:10C270005060FFF70EBB052800F04181062800F052
:10C280003583072800F0418308287FF402AB334947
:10C2900004229C2002B0BDE81040FDF789BE0528AD
:10C2A00000F03F81062800F0A284072800F0968362
:10C2B00008287FF4EEAA2A490222B62002B0BDE87F
:10C2C0001040FDF775BE06287FF4E3AA0120FDF7B4
:10C2D00071FD214B5860FFF7DCBA06287FF4D9AA1C
:10C2E0000220FDF767FD1C4B5860FFF7D2BA052806
:10C2F00000F08A8206287FF4CCAA019203F066F946
:10C30000019A5060FFF7C5BA052800F06B82062835
:10C310007FF4BFAA019201F0B5FF019A5060FFF7C8
:10C32000B8BA06287FF4B5AA0E4B1878FCF7BAFD08
:10C33000094B5860FFF7ADBA4438FF1F2038FF1F84
:10C340000838FF1FFC37FF1F6438FF1F2838FF1F06
:10C350001438FF1F1038FF1FD838FF1F4C38FF1F3D
:10C360006638FF1F1100FF1F052800F0DD8006283A
:10C3700000F09284072800F04B8408287FF489AAF3
:10C38000AE490422542002B0BDE81040FDF710BEB3
:10C3900005287FF47EAA02B0BDE81040FEF7CCBEAF
:10C3A00006287FF476AAFDF71DFDA54B5860FFF720
:10C3B00070BA06287FF46DAAFDF7F6FC0020FDF7A1
:10C3C000F9FC9F4B5860FFF764BA03231370FFF723
:10C3D00060BA0120FCF746FD00283FF4D4AC94F885
:10C3E0002F309B077FF5BFACB8E4FCF73BFD00287E
:10C3F0003FF4C9AC94F82F30D9073FF5BFACB2E495
:10C400004868012840F28C848D4B04221A70FFF793
:10C4100040BA4B68032B0FD88A4B0A7983F82F2038
:10C42000FFF737BA884B01924968187803F04CF847
:10C43000019A00287FF42DAA04231370FFF729BA6C
:10C4400082490122942002B0BDE81040FDF7D6BD1C
:10C450007C4B93F82F305360FFF71BBA486801926A
:10C4600002F07EFD019A0028E6D0FFF712BA486874
:10C47000019202F0D3FF019A0028DDD0FFF709BA3C
:10C480004868019202F0FEFF019A0028D4D0FFF71D
:10C4900000BA4868019202F0F5FE019A0028CBD05C
:10C4A000FFF7F7B94868019202F0C8FC019A00282A
:10C4B000C2D0FFF7EEB94868019202F0CFFE019AB0
:10C4C0000028B9D0FFF7E5B94868019202F092FF61
:10C4D000019A0028B0D0FFF7DCB94868019202F059
:10C4E00023FE019A0028A7D0FFF7D3B9486801922C
:10C4F00002F0D0FD019A00289ED0FFF7CAB9486823
:10C50000019202F063FF019A002895D0FFF7C1B9AC
:10C510004868019202F0A6FC019A00288CD0FFF72F
:10C52000B8B901924A4B7FE74868019202F0E8FDF2
:10C53000019A002880D0FFF7ACB94868019202F058
:10C540001BFE019A00283FF477AFFFF7A2B94868B5
:10C55000019202F0BDFE019A00283FF46DAFFFF793
:10C5600098B94868019202F0A7FD019A00283FF4AB
:10C5700063AFFFF78EB94868019202F0AFFD019AF0
:10C5800000283FF459AFFFF784B94868019201F0E1
:10C590006DFE019A00283FF44FAFFFF77AB9486863
:10C5A000019202F0D5FD019A00283FF445AFFFF754
:10C5B00070B94868019201F0D5FD019A00287FF416
:10C5C00068A939E74868019202F032FE019A002812
:10C5D0003FF432AFFFF75DB94868019202F02CFDDD
:10C5E000019A00283FF428AFFFF753B94868019239
:10C5F00002F05AFE019A00283FF41EAFFFF749B936
:10C600004868019202F020FF019A00283FF414AF1D
:10C61000FFF73FB94868019202F0B0FE019A002886
:10C620003FF40AAFFFF735B94868019202F06CFC9D
:10C63000019A00283FF400AFFFF72BB90438FF1F21
:10C64000D838FF1FF037FF1F1100FF1F4438FF1FAE
:10C650001200FF1F4868019202F07EFE019A002836
:10C660003FF4EAAEFFF715B94868019202F05EFCAC
:10C67000019A00283FF4E0AEFFF70BB94868019239
:10C6800002F0B2FD019A00283FF4D6AEFFF701B9DF
:10C690004868019202F0FAFB019A00283FF4CCAE00
:10C6A000FFF7F7B84868019202F04EFF019A0028A0
:10C6B0003FF4C2AEFFF7EDB84868019202F074FE95
:10C6C000019A00283FF4B8AEFFF7E3B8486801923A
:10C6D00002F074FC019A00283FF4AEAEFFF7D9B81F
:10C6E0004868019202F07CFC019A00283FF4A4AE55
:10C6F000FFF7CFB84868019202F08AFC019A00283F
:10C700003FF49AAEFFF7C5B84868019202F07EFD8B
:10C71000019A00283FF490AEFFF7BBB84868019239
:10C7200002F0C6FE019A00283FF486AEFFF7B1B8CA
:10C73000BA490122682002B0BDE81040FDF738BCBC
:10C74000486802B0BDE8104002F01EBC486802B064
:10C75000BDE8104002F052BF486802B0BDE810408A
:10C7600001F0D2BF486802B0BDE8104002F040BFFF
:10C77000486802B0BDE8104002F02EBF486802B021
:10C78000BDE8104002F0D0BD486802B0BDE81040DE
:10C7900002F0A6BB88880192FEF758FF019A50600C
:10C7A000FFF777B8486802B0BDE8104002F044BF18
:10C7B000486802B0BDE8104002F032BF888801929C
:10C7C000FEF74CFF019A5060FFF763B8486802B06B
:10C7D000BDE8104002F006BF486802B0BDE8104056
:10C7E00002F018BF486802B0BDE8104001F0E8BC94
:10C7F000486802B0BDE8104002F018BF486802B0B7
:10C80000BDE8104002F078BD486802B0BDE81040B5
:10C8100002F018BF88880192FEF710FF019A50605D
:10C82000FFF737B8486802B0BDE8104002F0ECBE30
:10C83000486802B0BDE81040FEF766BC019202F005
:10C84000B3FB019A5060FFF724B80192FEF756FC43
:10C85000019A5060FFF71DB8019202F075FD019A30
:10C860005060FFF716B8019202F044FB019A506045
:10C87000FFF70FB8019202F081FB019A5060FFF7B9
:10C8800008B867490422BC2002B0BDE81040FDF79B
:10C89000B5BB64490122A92002B0BDE81040FDF7F4
:10C8A000ADBB019202F096FB019A5060FEF7F1BF1A
:10C8B000019202F0A7FB019A5060FEF7EABF5A49C5
:10C8C0000222B22002B0BDE81040FDF797BB5749E5
:10C8D0000422982002B0BDE81040FDF78FBB019202
:10C8E00002F0E4FB019A5060FEF7D3BF019202F020
:10C8F0007BFD019A5060FEF7CCBF4D4904224C20CD
:10C9000002B0BDE81040FDF779BB4A4904229C20E3
:10C9100002B0BDE81040FDF771BB47490222B420C8
:10C9200002B0BDE81040FDF769BB44490222AE20C9
:10C9300002B0BDE81040FDF761BB019202F00AFEB3
:10C94000019A5060FEF7A5BF019202F039FD019AED
:10C950005060FEF79EBF3A4B0192187802F0DCFD62
:10C96000019A5060FEF795BF019202F085FC019A92
:10C970005060FEF78EBF33490422582002B0BDE854
:10C980001040FDF73BBB019202F054FD019A50604C
:10C99000FEF77FBF019202F085FD019A5060FEF71D
:10C9A00078BF019202F08AFD019A5060FEF771BFD4
:10C9B0001A490122682002B0BDE81040FDF71EBBF5
:10C9C000019202F01DFC019A5060FEF762BF0192D5
:10C9D00002F056FA019A5060FEF75BBF1A49022234
:10C9E000B62002B0BDE81040FDF708BB1749012290
:10C9F000692002B0BDE81040FDF700BB14490122D8
:10CA00006D2002B0BDE81040FDF7F8BA11490222CE
:10CA10006A2002B0BDE81040FDF7F0BA1838FF1FD9
:10CA20006C38FF1F5938FF1F6238FF1F4838FF1F3F
:10CA3000FC37FF1F4C38FF1F6438FF1F5E38FF1F95
:10CA40001100FF1F0838FF1F6638FF1F1938FF1F2E
:10CA50001D38FF1F1A38FF1FB4490422882002B076
:10CA6000BDE81040FDF7CABAB1490422B82002B0AF
:10CA7000BDE81040FDF7C2BA019202F0D7FA019A60
:10CA80005060FEF706BF019202F0CCFB019A5060A5
:10CA9000FEF7FFBEA74901226C2002B0BDE810409E
:10CAA000FDF7ACBAA4490422902002B0BDE81040C2
:10CAB000FDF7A4BA019202F071FC019A5060FEF7F2
:10CAC000E8BE019202F02CFA019A5060FEF7E1BE36
:10CAD0009A490122AA2002B0BDE81040FDF78EBAA3
:10CAE000974904228C2002B0BDE81040FDF786BAB9
:10CAF000019202F03DFC019A5060FEF7CABE01921D
:10CB000002F028FA019A5060FEF7C3BE8D49012257
:10CB10006E2002B0BDE81040FDF770BA8A490422C9
:10CB20007C2002B0BDE81040FDF768BA019202F027
:10CB30006FFC019A5060FEF7ACBE019202F002FB5E
:10CB4000019A5060FEF7A5BE80490422402002B041
:10CB5000BDE81040FDF752BA7D490222802002B0A4
:10CB6000BDE81040FDF74ABA019202F097FB019A26
:10CB70005060FEF78EBE019202F05AF9019A5060A1
:10CB8000FEF787BE73490422482002B0BDE810407A
:10CB9000FDF734BA70490422442002B0BDE81040C9
:10CBA000FDF72CBA6D490222AC2002B0BDE810405E
:10CBB000FDF724BA6A490422702002B0BDE8104093
:10CBC000FDF71CBA019202F091FB019A5060FEF74A
:10CBD00060BE019202F07CFA019A5060FEF759BEE5
:10CBE000019202F039F9019A5060FEF752BE5D4B96
:10CBF0000192187802F090FC019A5060FEF749BE4D
:10CC000059490422782002B0BDE81040FDF7F6B97A
:10CC100056490422542002B0BDE81040FDF7EEB999
:10CC200053490422602002B0BDE81040FDF7E6B988
:10CC300050490122652002B0BDE81040FDF7DEB981
:10CC4000019202F057FA019A5060FEF722BE4A495B
:10CC50000422502002B0BDE81040FDF7CFB9019288
:10CC600002F084FA019A5060FEF713BE4349012294
:10CC7000642002B0BDE81040FDF7C0B9019202F097
:10CC8000E3FA019A5060FEF704BE019202F0E6F961
:10CC9000019A5060FEF7FDBD019202F03FFA019A41
:10CCA0005060FEF7F6BD019202F098FA019A5060CA
:10CCB000FEF7EFBD32490422A02002B0BDE81040CB
:10CCC000FDF79CB92F4904225C2002B0BDE810405A
:10CCD000FDF794B92C490422742002B0BDE810403D
:10CCE000FDF78CB929490222B02002B0BDE81040FE
:10CCF000FDF784B9019202F0E5FA019A5060FEF75F
:10CD0000C8BD019202F0B8FB019A5060FEF7C1BDA8
:10CD10001F4901226F2002B0BDE81040FDF76EB937
:10CD2000C0B202B0BDE81040FDF732BC3838FF1F7A
:10CD30006838FF1F1C38FF1F4038FF1F5A38FF1F7D
:10CD40003C38FF1F1E38FF1F2C38FF1FF037FF1F16
:10CD50003038FF1FF837FF1FF437FF1F5C38FF1F05
:10CD60002038FF1F1200FF1F2838FF1F0438FF1F45
:10CD70001038FF1F1538FF1F0038FF1F1438FF1F22
:10CD80005038FF1F0C38FF1F2438FF1F6038FF1F6B
:10CD90001F38FF1F70B51049104C114B00224FF483
:10CDA00080700880227003F5806143F8042F8B4265
:10CDB000FBD10C4BDB7D73B90B4E40F21A7440F281
:10CDC000FA75A4F21A710422204631441444FDF786
:10CDD000EFF8AC42F5D170BD8846FF1F863EFF1FBD
:10CDE000E838FF1F7438FF1FEC38FF1F014B18781D
:10CDF000704700BF843EFF1F8B780BB9FEF736BC2F
:10CE000010B40423137010BC704700BF08B5874AE4
:10CE10009378002B40F0C7805378403BBF2B00F243
:10CE2000CE80DFE813F0BF018601A401CC004001F1
:10CE3000CC00CC00CC00CC006601CC0057017701BF
:10CE40002301EE01CC00CC00CC00CC009501CC003D
:10CE5000CC01CC003101CC00CC00DF01CC00CC00F7
:10CE6000CC00CC00CC00CC00CC00CC00CC00CC0062
:10CE7000CC00CC00CC00CC00CC00CC00CC00CC0052
:10CE8000CC00CC00CC00CC00CC00CC00CC00CC0042
:10CE9000CC00CC00CC00CC00CC00CC00CC00CC0032
:10CEA000CC00CC00CC004F01B201CC0019010F0125
:10CEB000CC00CC00CC00CC00CC00CC00CC00CC0012
:10CEC000CC00CC00CC00CC00CC00CC00CC00CC0002
:10CED000CC00CC00CC00CC00CC00CC00CC00CC00F2
:10CEE000CC00CC00CC00CC00CC00CC00CC00CC00E2
:10CEF000CC00CC00CC00CC00CC00CC00CC00CC00D2
:10CF0000CC00CC00CC00CC00CC00CC00CC00CC00C1
:10CF1000CC00CC00CC00CC00CC00CC00CC00CC00B1
:10CF2000CC00CC00CC00CC00CC00CC00CC00CC00A1
:10CF3000CC00CC00CC00CC00CC00CC00CC00CC0091
:10CF4000CC00CC00CC00CC00CC00CC00CC00CC0081
:10CF5000CC00CC00CC00CC00CC00CC00CC00CC0071
:10CF6000CC00CC00CC00CC00CC00CC00CC00CC0061
:10CF7000CC00CC00CC00CC00CC00CC00CC00CC0051
:10CF8000CC00CC00CC00E900CC00CC00CC00CC0024
:10CF9000CC00CC00CC00CC00CC00CC00CC00CC0031
:10CFA000CC00E900FA00012B0CD0022B0BD0204B57
:10CFB00004221A7008BD1F490988994223D81C4BC6
:10CFC00003221A7008BD5378372BF4D80A2800F0D2
:10CFD000268109281CD00B2800F082810C28F1D171
:10CFE0001549042240F21A7001EB830102FB030091
:10CFF000BDE80840FCF7DCBF0A28E3D10F4A0C4B20
:10D0000012785A6008BD0A2800F009810928D9D190
:10D010000949526841F8232008BD0A2800F04981D7
:10D020000928CFD1064B12791A7008BDE438FF1FCA
:10D03000D838FF1F8846FF1FEC38FF1F7038FF1FCE
:10D04000D138FF1F0A2800F0FF800928BAD1AE4A64
:10D05000AE4B52681A6008BD0A2800F01D810928ED
:10D06000B0D1A94AAA4B52681A6008BD0A2800F03C
:10D07000FF800928A6D11379A64A537519461520B1
:10D08000BDE80840FCF75EBF0A2800F0D3800928FD
:10D0900098D1A049137901F8023F01220220BDE88E
:10D0A0000840FCF7ABBF0A2800F0D880092889D1D6
:10D0B0009849536841F8183F04221820BDE80840F9
:10D0C000FCF79CBF0A287FF47DAF934A8E4B127801
:10D0D0005A6008BD0A2800F0DA8009287FF472AF90
:10D0E00013798C4A137119460420BDE80840FCF7F7
:10D0F00029BF0A2800F0D58009287FF463AF117991
:10D10000002940F0E780834B99751620BDE8084060
:10D11000FCF718BF0A2800F0888009287FF452AF76
:10D1200013797C4AD37019460320BDE80840FCF708
:10D1300009BF0A2800F0A18009287FF443AF1379C2
:10D14000744A137019460020BDE80840FCF7FABE87
:10D150000A2874D009287FF435AF6E49536841F826
:10D16000103F04221020BDE80840FCF747BF0A2802
:10D170006FD009287FF426AF1379664A5370194699
:10D180000120BDE80840FCF7DDBE0A287FF41AAF95
:10D19000614B5D4A1B78A3F10403B3FA83F35B0987
:10D1A000536008BD0A2800F0A78009287FF40AAF61
:10D1B000117940F2FF70BDE80840FCF7C3BE0A28B1
:10D1C00051D009287FF4FEAE5368012B3FF6EFAE35
:10D1D0005049137901F8173F01221720BDE8084094
:10D1E000FCF70CBF0A284DD009287FF4EBAE494963
:10D1F000536841F8203F04222020BDE80840FCF796
:10D20000FDBE0A285DD0092860D00B287FF4DAAE75
:10D21000404B0720D979BDE80840FCF793BE3F4951
:10D22000394A51F82330536008BD3A4A364BD27818
:10D230005A6008BD374A344B92785A6008BD354A67
:10D24000314B12695A6008BD304A2F4B12685A6040
:10D2500008BD304A2C4B52785A6008BD2D4A2A4BE3
:10D2600092695A6008BD2B4A274BD27D5A6008BD8F
:10D27000284A254B527D5A6008BD264A224B127817
:10D280005A6008BD234A204B126A5A6008BD214AE1
:10D290001D4B12795A6008BD1D4A1B4B12685A601B
:10D2A00008BD1C4B184A9B7D003318BF01235360F7
:10D2B00008BD1B4B144A1B78003318BF0123536071
:10D2C00008BD144A104BD2795A6008BD114B12792F
:10D2D000DA7108BD0F4A0C4B01219175596014E7B2
:10D2E0000E49042240F21A7001EB830102FB030095
:10D2F000BDE80840FCF782BE40F2FF70FCF708FE74
:10D30000014B586008BD00BFD838FF1F8C46FF1F77
:10D310009046FF1F7438FF1FD238FF1FEC38FF1FE5
:10D32000D138FF1F074B9A78022A04D15A685878DF
:10D330002AB9FBF7B1BD044B04221A707047FBF702
:10D34000ADBD00BFE438FF1FD838FF1F38B5184BFC
:10D350009A78012A14D00BD3022A05D15878FBF70A
:10D360009FFD144B586038BD124B04221A7038BD13
:10D370005878FF280AD0FBF775FD0E4B586038BD72
:10D380005878FBF78FFD0B4B586038BD0120FBF739
:10D3900069FD05460020FBF765FD44000220FBF710
:10D3A00061FD44EA8504034B2043586038BD00BF4B
:10D3B000E438FF1FD838FF1F034B9A7802B170473B
:10D3C0005868404200F0CEBEE438FF1F034B9A7805
:10D3D00002B17047586800F0C5BE00BFE438FF1FB7
:10D3E000024B987800B1704700F0BCBEE438FF1FD4
:10D3F0000A4B9A7832B95A7862B1012A06D1586834
:10D4000000F00EBF064B04221A707047044B032233
:10D410001A707047586800F0D3BE00BFE438FF1F91
:10D42000D838FF1F10B4114B5B789BB91049114BD2
:10D430000868114A1149DB7802F8013B0124431EB8
:10D440000C70073013F8011F02F8011B8342F9D159
:10D4500010BC7047012BFBD1094AC1246020042174
:10D460001371D4719071517110BC7047E438FF1F73
:10D470001C00FF1F7438FF1FC838FF1FC438FF1F70
:10D48000D838FF1FF8B50D490D4B01E08B4207D08E
:10D4900053F8042F0132F9D00A4B08221A70F8BD54
:10D4A000094C0A4F04F50066C4F5FE25281954F806
:10D4B000041FB847B442F9D1F8BD00BFFCF707001C
:10D4C000FCEF0700D838FF1F843EFF1F5DA8010056
:10D4D0000C4A5378012B10D009D3FF2B06D1536887
:10D4E000094A03F5FE231B685360704770474FF4E9
:10D4F000FE22054B12685A607047044A024B1268BC
:10D500005A607047E438FF1FD838FF1F04F0070047
:10D510004FF0E02318B9044AC3F80C2D7047034AB2
:10D52000C3F80C2D704700BF0100FA050400FA058E
:10D53000194A1A4938B5136823F07F4323F0FF03D3
:10D540008B4203D0164B04221A7038BD5268154B1B
:10D550009A42F7D1FBF74CFC72B6FCF7FFF9124C7C
:10D56000124B134D13484FF0E0214FF0FF32C3F838
:10D570008020C3F88021C3F88420C3F88421C3F835
:10D580008820C3F88821C3F88C20C3F88C2125603B
:10D59000C1F80C0D38BD00BFE438FF1F00819200B8
:10D5A000D838FF1FD6C5B4A30000FF1F00E100E07C
:10D5B000785634120400FA05044B5A6840F2D243FC
:10D5C0009A4202D1024B01221A707047E438FF1FC1
:10D5D000863EFF1F10B52D4B98785A7882B040B127
:10D5E000032A10D0042A4CD0294B04221A7002B00E
:10D5F00010BD0A2A41D8DFE802F012171C064421A8
:10D60000242E32373B0002AA002142F8041D0146B5
:10D61000586802F091F81E4B019A5A60E7E702F051
:10D6200085F81B4B5860E2E702F07CF8184B586015
:10D63000DDE702F07FF8164B5860D8E702F016F8E5
:10D64000D5E702F01BF8044602F01EF8104B204309
:10D65000C0B25860CBE7586802F082F8C7E702F022
:10D660009FF80B4B5860C2E7586802F09FF8BEE77E
:10D6700002F0A2F8064B5860B9E7054B03221A7076
:10D68000B5E7596801F0E4FFB1E700BFE438FF1FD8
:10D69000D838FF1F10B54849484A08784B68507081
:10D6A00064240E281470536079D00ED98E2837D098
:10D6B0001BD9D2286FD021D9F22868D0FF281AD1DF
:10D6C00040F2D242934272D010BD042838D02FD8F5
:10D6D000022819D038D801280DD18A78002AF3D130
:10D6E0001846BDE8104000F03DBD882814D08928B8
:10D6F00036D00F2818D002231370E5E7D128FAD1CD
:10D70000BDE81040FFF7BEBE8A78002ADCD158423F
:10D71000BDE8104000F026BDBDE81040FFF782BE16
:10D72000BDE81040FFF756BFBDE81040FFF70EBE42
:10D73000082810D90C28DED8BDE81040FFF766BBDA
:10D74000BDE81040FFF754BE88780028BCD1BDE882
:10D75000104000F007BD8B782BB30423137010BD6D
:10D76000096821F07F4121F0FF010029ACD140F28E
:10D77000D2429342A8D140F2FF70FCF7E3FBFCF7E2
:10D7800087FD4FF0E0230E4AC3F80C2D10BDBDE815
:10D790001040FFF7CDBEBDE81040FFF799BEBDE8D1
:10D7A0001040FFF7BFBDBDE81040FDF75FBF054B60
:10D7B00001221A7010BD00BFE438FF1FD838FF1FC8
:10D7C0000400FA05863EFF1F2DE9F043954B964D68
:10D7D0001B7883B053B92B7843B9944C2378032B2F
:10D7E00033D0042B00F0AD80914E07E0914B1B78B5
:10D7F000063BDBB2192B1FD98C4C8D4E8E4B1A7801
:10D800000023237033702B7022B14FF0E0238B4A3A
:10D81000C3F80C2D0DF10700FBF748FE002850D18E
:10D82000874B1B78042B7BD02278082A41D9FFF73D
:10D8300031FF03B0BDE8F083824A22FA03F3DA072E
:10D84000DAD57A4C2378032BCBD1794E3378002B61
:10D8500000F0A580012BD1D17B4F07F1090817F803
:10D86000010FFBF709FE4745F9D1C7E7714D637911
:10D87000617AA27AA779E679207A2B70E37AA97186
:10D880006A712B716F70AE70E871FCF76DF86C4ABD
:10D890006E4B12786E491860042A4FF000004FF06A
:10D8A000030308702370C2D195F90020002A3DDAE5
:10D8B0001A4640F25113D340DB07B8D503B0BDE898
:10D8C000F083FBF70DFE002835D162789DF8071034
:10D8D000531CDBB22244092B63701171A0D15D4B44
:10D8E00021795A7860708A429B7800F09680002BEC
:10D8F00096D0994294D101232B70574A0023D01D12
:10D9000001E012F8011B0B448242DBB2F9D1227B09
:10D910009A42ABD04A4B1B78042293422270CDD15D
:10D92000444B93F90030002BFFF67EAF01F052FA22
:10D9300003B0BDE8F08301229DF8073062702371C7
:10D940006EE7DFF81091454F99F8030099F80180D0
:10D95000374E01233B7000237B707B608044FBF7D4
:10D960008BFD99F80100FBF787FD3878FBF784FD04
:10D970007878FBF781FDF879FBF77EFDB879FBF746
:10D980007BFD08F101087879FBF776FD5FFA88F8EE
:10D990003879FBF771FD4046FBF76EFD2EE7DFF8A7
:10D9A000B490DFF8B88099F8030099F8017098F8FE
:10D9B000002098F801300744174498F807201F44C6
:10D9C00098F80630174498F805201F4498F804305A
:10D9D00017441F44FBF750FD99F80100FBF74CFD7D
:10D9E00098F80000FBF748FD98F80100FBF744FDAC
:10D9F00098F80700FBF740FD98F80600FBF73CFDA0
:10DA000098F80500FBF738FDFFB298F80400FBF723
:10DA100033FD3846FBF730FDF0E68B427FF46DAF07
:10DA200069E700BFD138FF1F853EFF1F6022FF1F3F
:10DA3000C438FF1FE438FF1F863EFF1F0400FA05AD
:10DA4000D238FF1F11020002C738FF1FD438FF1F52
:10DA5000E038FF1F7438FF1F6522FF1FD838FF1FF3
:10DA6000F0B5254B254C0246007992F801E09678F6
:10DA7000D778D871507998710D469179597194E899
:10DA8000030083B0D2795E7083F800E09F701A7152
:10DA90008DE80300FFF7FEFD194B1B786E46B3B10E
:10DAA000012B05D096E8030084E8030003B0F0BD25
:10DAB000144A6B1E073512F8011B03F8011FAB4215
:10DAC000F9D196E8030084E8030003B0F0BD2B70A1
:10DAD0006B7063782278AA70EB70E3792B71A3796D
:10DAE0006B716379AB7196E803002379EB7184E87D
:10DAF000030003B0F0BD00BFE438FF1FD838FF1F9C
:10DB0000C438FF1FC938FF1FF0B50D4C0D4E054638
:10DB10000F4694E8030083B03570B27073608DE8EF
:10DB200003007770FFF7B6FD9DE803006368257872
:10DB3000054A84E803001846157003B0F0BD00BF25
:10DB4000D838FF1FE438FF1F843EFF1F08B50C4B79
:10DB5000196821F07F4121F0FF0121B95A6840F294
:10DB6000D2439A4200D008BD40F2FF70FCF7EAF9B8
:10DB7000FCF78EFB4FF0E023024AC3F80C2D08BDE2
:10DB8000E438FF1F0400FA0510B50D4CFBF7B2FD99
:10DB900094F82920E36B21465208B3FBF2F3B0FB63
:10DBA000F3F202FB130021F8400F02228020FCF761
:10DBB00025FA94F8423023F0010384F8423010BD76
:10DBC000F037FF1F10B5064CB4F84000FBF7A4FD7A
:10DBD00094F8423023F0020384F8423010BD00BFB5
:10DBE000F037FF1F38B50020FBF7CAF90B4B93F84D
:10DBF0002520092A054602D9094C257038BD40F276
:10DC00004123D340DB07064CF7D501462078FBF7CC
:10DC100043FE636825701844606038BDF037FF1F0D
:10DC20007022FF1F684620F007018D4619B5164B7C
:10DC3000D3F8A030590609D5144C94F82530072B99
:10DC400008D0114A936943F080739361BDE819408D
:10DC50008546704794F84230DA0703D5FFF794FF02
:10DC600094F84230980701D5FFF7ACFF94F8543090
:10DC7000D907E6D5064A002151605A07E1D523F0BD
:10DC8000010384F85430DCE700A00440F037FF1FA4
:10DC90007022FF1F1A4B6846D3F8A02020F007011E
:10DCA0008D46910601B503D4D3F8A020120617D5EE
:10DCB000FFF798FF0020FBF763F904281BD0104BF7
:10DCC0005A6942F080725A61DA6942F08072DA6110
:10DCD0001A6A42F080721A62BDE8014085467047B8
:10DCE000D3F8A030DB05F7D5FFF77CFF0020FBF76A
:10DCF00047F90428E3D101210220FBF75FF8DEE7B2
:10DD000000B004400346044A00EBD070C0F34F005B
:10DD100082F82930FBF7C8BCF037FF1F01280CD070
:10DD200007D3022803D1074BB3F904007047002042
:10DD30007047044BB3F900007047024BB3F902007F
:10DD4000704700BFF846FF1FFBF73AB800B585B033
:10DD500001F094FC10B905B05DF804FB01F020FD62
:10DD60000328F8D10020FBF79DF800900120FBF775
:10DD700099F801900420FBF795F802900520FBF735
:10DD800091F804AB039013E90F0001F099FCE2E76E
:10DD900070B50A4C0A4DE06909F038FE01460948A1
:10DDA00009F040FF064694F8290009F02FFE0146CD
:10DDB000304609F037FF286070BD00BFF037FF1F05
:10DDC0002C00FF1F0050C34870B5094C094DE06995
:10DDD00009F01CFE0146084809F024FF0646E06BE6
:10DDE00009F014FE0146304609F01CFF686070BD62
:10DDF000F037FF1F2C00FF1F007C924938B5054605
:10DE000000200C46FBF7BCF8314B93F8283013B1D7
:10DE100080F00700C0B214B980F00700C0B22D4BEB
:10DE20000022C3F8902007280FD8DFE800F01D215A
:10DE30002B313C47041D274B27490C24002202208C
:10DE40001C6688609D619A629A63224B9A6D4FF4BA
:10DE5000007042F004029A650021C3F89800022085
:10DE6000BDE83840FAF7AABF1A4B3F221A66ECE722
:10DE7000184B194900220C2018668A609A619A6230
:10DE80009D63E2E7134B1449302400220120D7E7B9
:10DE9000104B11490022032401201C6688609A61FE
:10DEA0009A629D63D1E70B4B0B49002203240220A9
:10DEB0001C6688609A619D629A63C6E7054B0649B5
:10DEC0000022302018668A609A619D629A63BCE7DE
:10DED000F037FF1F008003407022FF1FF8B5554840
:10DEE000554C564E01F0F0FE554801F0EDFE5548F8
:10DEF00001F0EAFE94F82500FBF772FDE06909F0F5
:10DF000085FD01460546504809F08CFE074694F809
:10DF1000290009F07BFD0146384609F083FE2946B9
:10DF200030604A4809F07EFE0546E06B09F06EFD60
:10DF30000146284609F076FE94F825507060062DBB
:10DF400030D0072D3CD0082D5BD0092D12D06DB9F3
:10DF50004FF40040FBF74CFF8020FBF751FF0120FE
:10DF6000FBF73AFC29462846FFF748FFBDE8F84092
:10DF7000FAF726BF4FF40040FBF73AFF8020FBF78B
:10DF80003FFF0120FBF728FC94F82D10E06BFBF716
:10DF90001BFB94F82910E06B4908FBF77BFB94F816
:10DFA0002550D4E74FF40040FBF722FF8020FBF719
:10DFB00027FF0120FBF710FC94F82550072DC2D154
:10DFC0004FF40040FBF71CFF8020FBF719FF94F88B
:10DFD0002C30012B2AD094F82D10E06BFBF7F4FACB
:10DFE00094F82910E06B4908FBF754FBFBF7A2FB00
:10DFF000FCF7EEFF0120FBF7A3FB94F82550082D5A
:10E00000A3D14FF40040FBF7F3FE0020FBF7E4FB45
:10E0100094F82D10E06BFBF7D7FA94F82910E06B19
:10E020004908FBF737FB94F825508EE70020FBF7F3
:10E03000D3FBD0E7C046FF1FF037FF1F2C00FF1FA8
:10E040002847FF1FA046FF1F0050C348007C92498D
:10E05000014B01221A7370477022FF1FB0F5007F39
:10E0600010B504464AD02CDDB0F5806F1CD0B0F559
:10E07000006F16D1FBF7BCFE4FF48070FBF7C0FEBB
:10E080004FF48060FBF7BCFE4FF40070FBF7B8FE66
:10E090004FF48040FBF7B4FE1D4BA3F86640FAF73F
:10E0A00083FE1C4B1C6010BDFBF7A2FE4FF480707A
:10E0B000FBF7A6FE4FF40070FBF7A2FE4FF40060E2
:10E0C000E4E7B0F5807FECD1FBF792FE4FF480607F
:10E0D000FBF796FE4FF40070FBF792FE4FF40060E2
:10E0E000FBF78EFE4FF48040FBF78AFE084BA3F847
:10E0F0006640FAF75BFE074B1C6010BDFBF778FE2D
:10E100004FF48070FBF77CFE4FF48060D4E700BFD3
:10E11000F037FF1FE846FF1F08B50F4B93F8252087
:10E1200012B993F8692082B90C4A9B6F000290FBE8
:10E13000F3F010604FF40060FFF790FF084B0022EF
:10E140001A60FAF73DFE012008BD044ADB6F0002A9
:10E1500090FBF3F01060EDE7F037FF1FF046FF1F74
:10E160002047FF1F00F54333104A03F5A073934285
:10E1700001D9002070470E4A0E4B10B51468186084
:10E180004FF40070FFF76AFFB4F5006F03D0FAF7A1
:10E1900017FE012010BD084B084C186809F03AFC26
:10E1A0002060FAF70DFE012010BD00BF801A0600A6
:10E1B000E846FF1F5847FF1FE446FF1F2047FF1F89
:10E1C000124A134B10B510611C684FF48060FFF7C2
:10E1D00045FF4FF48040FBF713FEB4F5007F0CD0F1
:10E1E000B4F5006F05D10B4B0B4C186809F012FC0D
:10E1F0002060BDE81040FAF7E3BD084A064B1268FC
:10E200001A60BDE81040FAF7DBBD00BF7022FF1FA7
:10E21000E846FF1FE446FF1F9846FF1F2047FF1FE9
:10E22000024B5B681844FFF7CBBF00BF7022FF1F93
:10E230000C4B93F8252012B993F8692042B90A4A89
:10E240009B6F106800FB03F0002808DB001270478A
:10E25000054ADB6F106800FB03F00028F6DAFF3098
:10E2600000127047F037FF1FE046FF1F00F5AF3385
:10E27000034A03F5C873934200D84DE70020704766
:10E2800020BF0200014B1869704700BF7022FF1FBA
:10E2900008B5024B186809F0D7FD08BD2047FF1FDD
:10E2A000014B5869704700BF7022FF1F014B9869EE
:10E2B000704700BF7022FF1F10B5164B164C187820
:10E2C000FAF7F0FD4FF4C673144A03FB00F082FB2B
:10E2D00000320244C017C0EBE230B0F58C7F6061C1
:10E2E0004FF004000ADBFBF783FD63693C2B4FF022
:10E2F00002000ADDBDE81040FBF782BDFBF780FDA0
:10E3000063693C2B4FF00200F4DCBDE81040FBF7E2
:10E310006FBD00BF1700FF1F7022FF1F018000802C
:10E3200010B5454B454C1878FAF7BCFDC0F30F10FB
:10E3300009F070FB08F060FF02460B4632A1D1E9FC
:10E34000000109F0D7F832A3D3E9002308F0F4FD67
:10E3500009F056FA3A4909F065FC08F04DFF0AF059
:10E3600031F82DA3D3E9002308F09AFF2CA3D3E9B9
:10E37000002308F0E3FD02460B462BA1D1E9000182
:10E3800009F0B8F82AA3D3E9002308F0D5FD09F075
:10E3900037FA09F059FDA0610820FBF745FDA36994
:10E3A00048B9772B4FF0080022DCFBF729FDFAF77C
:10E3B0004FFD48B110BD6D2BFCDC0820FBF720FDA4
:10E3C000FAF746FD0028F5D1FBF74AFD0028F1D108
:10E3D0004FF40050FBF728FD0028EBD14FF480707C
:10E3E000FBF722FD0028E5D1BDE81040FAF7E8BCB4
:10E3F000FBF7FEFCFAF7FCFC4FF48070BDE8104020
:10E40000FFF72CBEAFF300809A9999999999C14072
:10E410009A999999999901400000000000A07240D2
:10E420000000000000D4AA4000000000C83A2F41BC
:10E4300000000000001071401600FF1F7022FF1F37
:10E440000000204138B5374DFBF78EFAEB69C31A4F
:10E45000002BB8BF5B42B3F57A7F50DA324CFFF73E
:10E460002BFFFCF72BFFFCF743FEA36D98422DD842
:10E47000FBF77AFA6B6AE26DC01A0028B8BF404217
:10E4800090420ED394F86420012A03D001F0FCF8E6
:10E4900098B938BD0023254984F86430A420FBF7DF
:10E4A000ADFD94F86430012BF0D14FF40030FBF750
:10E4B0009FFC01F0E9F80028EBD01D4A1D4B1068C5
:10E4C00019686A68BDE8384001F07CB9FBF74CFA7E
:10E4D0002B6AC01A0028B8BF4042B0F57A7FC7DB6C
:10E4E000FCF796FD4FF40030FBF782FC94F86430A3
:10E4F00063B1FCF70FFEFBF737FA2862B8E7044672
:10E50000FCF7EEFEFFF70CFFEC61A7E721460122C6
:10E5100001F8642FA420FBF771FDFBF725FA686270
:10E52000E7E700BF7022FF1FF037FF1F5438FF1FBF
:10E53000EC46FF1FE446FF1F014B5868704700BFC1
:10E540007022FF1F014B1868704700BF5847FF1F1C
:10E550002DE9F041414C94F8253082B00546092B55
:10E5600025D8DFE803F0322424242424320527327E
:10E57000FBF7C0F8E16B3A4C8A10904202EB42067E
:10E58000636B2CDA9E422ADAC31A0B44354E61685B
:10E5900032686063C91AD01A3060616013B1324AC0
:10E5A0005B429360002D3FD0304BA26A1A6002B0EC
:10E5B000BDE8F0812E4B186809F046FC2B4A284B29
:10E5C0001060986202B0BDE8F08178B1244B274A10
:10E5D0005868996AD862116002B0BDE8F081B04213
:10E5E00020DD9A421EDDC31A5B1ACFE71C4C1F4D7B
:10E5F000E36A60682E68C01A09F00CFA1A4B1968B1
:10E6000009F05CFA09F020FC082301460093324629
:10E61000052304F1300001F0EDF963682860A06281
:10E62000E362C4E7C31AB1E709F0F4F90E4B0F4FE8
:10E630005968D7F8008009F041FA09F005FC082371
:10E640000146424600930B48022301F0D3F90A4BDE
:10E6500032683860A0621A603560A8E7F037FF1FA3
:10E660007022FF1F4847FF1F2C00FF1FE446FF1FBB
:10E670002047FF1FA022FF1FF446FF1F08B50120FF
:10E68000FFF766FFFFF72AFC0120FFF761FF034A4F
:10E69000034B92F825201A7308BD00BFF037FF1F07
:10E6A0002C00FF1F044A054B92F825201B7B9A4241
:10E6B00000D0E3E7704700BFF037FF1F2C00FF1FBB
:10E6C000F8B50B4B0B4F58680B4E0C4D0C4C0D49CD
:10E6D00018610022002301203B6033602B60226020
:10E6E0000A60FFF735FFBDE8F840FFF7F7BB00BF52
:10E6F0007022FF1F5847FF1FE046FF1FF046FF1F15
:10E700009846FF1F2047FF1F10B504464FF4804076
:10E71000FBF776FB034B01205C601C61BDE81040F9
:10E72000FFF716BF7022FF1F014B1868704700BF2C
:10E73000E446FF1F0C4B93F8252012B993F869208B
:10E7400042B90A4A986F136800FB03F0002808DBFF
:10E7500000127047054AD86F136800FB03F00028C9
:10E76000F6DAFF3000127047F037FF1FEC46FF1F4C
:10E77000034A92F8423023EA000082F842007047D0
:10E78000F037FF1F034B93F84230184214BF0120AB
:10E7900000207047F037FF1F034A92F8543023EAF5
:10E7A000000082F854007047F037FF1F034B93F8C6
:10E7B0005430184214BF012000207047F037FF1F6B
:10E7C000014B1868704700BF0047FF1F684620F0E4
:10E7D00007018D462DE9F147B94D8FB00121002089
:10E7E000FAF7ECFA95F82530002B35D1B54CB64A3E
:10E7F000B4F9381081EAE173A3EBE1739B10D360A5
:10E80000136843F001031360B048E26B0168236CA6
:10E8100021F080010160217B01320133E263236436
:10E8200051B1AB4A95F82510127B914202D0FFF707
:10E8300025FF236C00222273EA699A4240D92A6A92
:10E84000E36B9A4211D900210846FAF7B7FA0FB0E4
:10E85000BDE8F147854670479B4B9A4C0022DA6031
:10E860001A6842F001021A60CEE70023E36301F068
:10E870007BFA4FF48060FBF7D7FA002800F03E8166
:10E8800095F82560002E40F0668195F86930012BDF
:10E8900000F0838008A8FBF7EFFAA2688D4B089878
:10E8A000BDF824109980012A186000F0FB81022A2B
:10E8B00000F0F481002A73D11E88764236B26FE0F0
:10E8C0000026854F266401F05FFA3046FFF740FED0
:10E8D0003A682B6982EAE271A1EBE27183EAE372A2
:10E8E000A2EBE37291424FF0100053DDFBF788FA80
:10E8F0004FF48060FBF798FA002840F0858195F886
:10E900002430012B00F0A4812A68744B744E1868DF
:10E91000514201F02DF809F07DF830604FF400709D
:10E92000FBF782FA002800F0678195F82530002B6C
:10E9300040F0B98095F86930002B00F0B4806B6826
:10E94000EE6F1B0293FBF6F6DFF89481D7F8009088
:10E95000D8F8000009F078FA33464946614AFBF7D7
:10E960003FFE614B186000F089FE00283FF467AF5E
:10E9700000F016FF01287FF462AFD8F8000009F01C
:10E9800063FA3B680B930A900EAB13E90F0000F09B
:10E9900097FE54E7FBF72CFAAAE7FBF7A5FA06B2B5
:10E9A00094F84430012B95F8693004BF764236B2B2
:10E9B000002B7ED06B68EA6F1B0293FBF2F34A4F89
:10E9C0004A4A38683146FBF785FE494B3A6820874A
:10E9D00000281A60C0F25781002384F84430454F64
:10E9E00045483A68082331460093042301F002F8B1
:10E9F000B4F93830386083EAE37094F84410A0EB3F
:10EA0000E370FFF7FBF900F039FE002840F0928038
:10EA1000FFF79CF995F82530002B40D195F8693027
:10EA2000002B3CD039686B68EA6F81EAE176A6EB8F
:10EA3000E1761B0293FBF2F39E42D4BF002601262F
:10EA400031460120FBF7E4F93046FAF7ABF995F8C7
:10EA50006A3053B16269B5F86C30934240F3178164
:10EA6000B5F86E105B1A9A4205DAFAF70DFB4FF40F
:10EA70008020FBF7C5F9FFF75DFEFCF7D1FA4FF4F4
:10EA80000030FBF7D1F9002850D1FAF7E1F900285E
:10EA90007FF4D9AE4FF48070FFF7E0FAD3E639681F
:10EAA0006B68AA6FC1E76B68AE6F1B0293FBF6F64B
:10EAB0004AE76B68AA6F1B0293FBF2F37FE700BF84
:10EAC000F037FF1F7022FF1F0060034000800340EB
:10EAD0002C00FF1FF846FF1FE446FF1F5847FF1F8B
:10EAE0002047FF1FC046FF1FF046FF1F2847FF1F9C
:10EAF000E046FF1FEC46FF1FB822FF1F4FF40070D7
:10EB0000FBF792F900287FF4BBAE4FF40060FBF7EF
:10EB10008BF9064600287FF4B3AE4FF48070FBF704
:10EB200083F9002840F0DC807C4F73E70020FFF77A
:10EB3000F3FAAAE700F034FE00287FF469AFFFF78C
:10EB400077FB0A90FFF7F6FD0EAB0B9013E90F0071
:10EB500000F0B6FD5CE7DFF8FCA1714EDFF8F8913C
:10EB6000DFF8F8816D4F08A8FBF786F9089A6D4821
:10EB7000BDF82430CAF800206B496A680068AAF81A
:10EB800004300968BAF804E006901202A86F92FBFC
:10EB9000F0F266480792664ADAF80030ADF800E015
:10EBA000059104900392CDF80490624A624963484B
:10EBB0000296FBF735FE624BD9F800E0C3F800E09F
:10EBC0004FF00809B6F90010D8F800205D48CDF8DC
:10EBD0000090022300F00EFFB6F90230B6F90010E3
:10EBE000C8F800003A685848CDF80090194404234A
:10EBF00000F000FF386006E74FF48060FBF714F97F
:10EC000000287FF492AE1AE6504A61682069FBF74B
:10EC1000C5FC454B186000F031FD002846D1236942
:10EC20006168EA68591A81EAE173A3EBE1739342E0
:10EC30003FF765AE3B68AA6883EAE371A1EBE37135
:10EC400091423FF75CAE4FF48040FBF7D1F856E6B7
:10EC50004FF48060FBF7E8F8002835D14FF40070DE
:10EC6000FBF7E2F800283FF459AE2F4B2F4ED3F8B4
:10EC70000080306809F0E8F84146FBF77BFB08F0BC
:10EC8000C9FE30604AE6012384F84430A7E6FAF76B
:10EC9000F5F94FF48020FBF7ABF8ECE69E8876425E
:10ECA00036B27DE65E88764236B279E600F078FDCF
:10ECB0000228B4D1226963680B930A920EAB13E960
:10ECC0000F0000F0FDFCAAE7174A236911681848F5
:10ECD0006268164EFBF790FB08F09CFE3060BDE7C3
:10ECE00014480E4F00F0F0FF184800F0EDFF1348F5
:10ECF00000F0EAFF104800F0E7FF0C4B104995F8D0
:10ED000025000E6000221A603E60FAF73BFF104BB0
:10ED10004FF40072C3F898207AE600BFEC46FF1F5C
:10ED20004C47FF1FE446FF1F5847FF1F2047FF1FA8
:10ED30009846FF1FC046FF1FA046FF1F2847FF1F22
:10ED4000E046FF1FBC22FF1FC022FF1F0047FF1F1E
:10ED500000800340F846FF1FF046FF1F5047FF1F8B
:10ED6000684620F007018D4601B5FAF70DF8044A10
:10ED7000BDE80140136823F04003136085467047E7
:10ED800000600340034B93F84230DB0701D5FEF7E8
:10ED9000FBBE7047F037FF1F034B93F842309B07D1
:10EDA00001D5FEF70FBF7047F037FF1F074A92F8F3
:10EDB0005430D80708D5064900204860590744BF99
:10EDC00023F0010382F85430704700BFF037FF1F73
:10EDD0007022FF1F08B5FAF70BF84FF48070BDE8FA
:10EDE0000840FFF73BB900BF014B1868704700BFF0
:10EDF000C046FF1F014B9868704700BFC046FF1F09
:10EE0000014B1868704700BF2847FF1F014B9868E7
:10EE1000704700BF2847FF1F014B1868704700BFAD
:10EE2000A046FF1F014B9868704700BFA046FF1F18
:10EE3000014B5868704700BFF037FF1F044A9042EB
:10EE400098BF044A03469ABF5360012000207047D0
:10EE5000905F0100F037FF1F014B986B704700BFB8
:10EE6000F037FF1F044A904298BF044A03469ABFF6
:10EE70009363012000207047905F0100F037FF1F6F
:10EE8000014B93F829007047F037FF1F831EFC2BBE
:10EE900002D900231846704770B50E4C0E4D84F809
:10EEA0002900C0F34F00FAF7FFFBE06908F0AEFD60
:10EEB00001460A4808F0B6FE064694F8290008F014
:10EEC000A5FD0146304608F0ADFE01232860184636
:10EED00070BD00BFF037FF1F2C00FF1F0050C3485C
:10EEE0000030034B18BF012083F82800704700BF93
:10EEF000F037FF1F034B93F82800003018BF0120A4
:10EF0000704700BFF037FF1F012898BF034A034630
:10EF10009ABF82F82E30012000207047F037FF1F83
:10EF2000014B93F82E007047F037FF1FB0F5803F7C
:10EF30000BD208B5064BDA6BD863904203D0FFF7CB
:10EF4000BFFB012008BD012008BD0020704700BFA5
:10EF5000F037FF1F014BD86B704700BFF037FF1F22
:10EF6000B0F5803F38BF044A03463ABFA2F84030AC
:10EF700001200020704700BFF037FF1F014BB3F89E
:10EF800040007047F037FF1F064B003093F82D20EC
:10EF900018BF0120824283F82D0001D0FFF790BBFB
:10EFA000704700BFF037FF1F034B93F82D00003070
:10EFB00018BF0120704700BFF037FF1F022898BF1D
:10EFC000034A03469ABF82F82C3001200020704784
:10EFD000F037FF1F014B93F82C007047F037FF1FED
:10EFE00000F54333054903F5A0738B4298BF044BEA
:10EFF00002469ABF1A66012000207047801A060058
:10F00000F037FF1F014B186E704700BFF037FF1F2E
:10F0100042F21072904298BF034A03469ABF53854A
:10F0200001200020704700BFF037FF1F014BB3F9EC
:10F030002A007047F037FF1F831F032B00D930B918
:10F04000044A054B82F82500012018737047002000
:10F05000704700BFF037FF1F7022FF1F014B93F86E
:10F0600025007047F037FF1F094BB3F86630B3F542
:10F07000806F08D0B3F5006F07D0B3F5007F0CBFE9
:10F08000022000207047032070470120704700BF16
:10F09000F037FF1F0A2898BF034A03469ABF13623E
:10F0A00001200020704700BFF037FF1F014B186A96
:10F0B000704700BFF037FF1FB0F5803F38BF034AED
:10F0C00003463ABF1363012000207047F037FF1F4B
:10F0D000014B186B704700BFF037FF1FB0F5803F42
:10F0E00038BF034A03463ABF5363012000207047EC
:10F0F000F037FF1F014B586B704700BFF037FF1F01
:10F10000044A904298BF044A03469ABF53610120C3
:10F1100000207047400D0300F037FF1F014B586976
:10F12000704700BFF037FF1F044A904298BF044A5F
:10F1300003469ABF1360012000207047400D030072
:10F14000F037FF1F014B1868704700BFF037FF1FF3
:10F15000044A904298BF044A03469ABF13610120B3
:10F1600000207047400D0300F037FF1F014B186966
:10F17000704700BFF037FF1F1428F8B523D8134C91
:10F18000134DE06108F042FC01460646114808F0C4
:10F1900049FD074694F8290008F038FC0146384636
:10F1A00008F040FD314628600B4808F03BFD06465C
:10F1B000E06B08F02BFC0146304608F033FD0123DC
:10F1C00068601846F8BD00231846F8BDF037FF1FE9
:10F1D0002C00FF1F0050C348007C9249014BD869A6
:10F1E000704700BFF037FF1FB0F5803F38BF034ABC
:10F1F00003463ABFD364012000207047F037FF1F59
:10F20000014BD86C704700BFF037FF1FB0F5803F4F
:10F2100038BF034A03463ABF1365012000207047F8
:10F22000F037FF1F014B186D704700BFF037FF1F0D
:10F23000012898BF034A03469ABF82F82430012070
:10F2400000207047F037FF1F034B93F82400003075
:10F2500018BF0120704700BFF037FF1F044A9042DB
:10F2600098BF044A03469ABF93610120002070476B
:10F27000A0860100F037FF1F014B9869704700BF5F
:10F28000F037FF1FB0F5803F38BF034A03463ABF4F
:10F290009364012000207047F037FF1F014B986CEA
:10F2A000704700BFF037FF1F044A904298BF044ADE
:10F2B00003469ABF9360012000207047400D030071
:10F2C000F037FF1F014B9868704700BFF037FF1FF2
:10F2D000044A904298BF044A03469ABFD360012073
:10F2E00000207047A0860100F037FF1F014BD8684F
:10F2F000704700BFF037FF1F064A92F8543020B91C
:10F3000023F0010382F85430704743F0010382F880
:10F3100054307047F037FF1F024B93F8540000F051
:10F3200001007047F037FF1F064A92F8543020B9A9
:10F3300023F0040382F85430704743F0040382F84A
:10F3400054307047F037FF1F024B93F85400C0F35E
:10F3500080007047F037FF1F012898BF034A03461B
:10F360009ABF82F86A30012000207047F037FF1FF3
:10F37000014B93F86A007047F037FF1FA0F132028B
:10F38000B2F5D77F98BF044A03469ABFA2F86C3003
:10F3900001200020704700BFF037FF1F014BB3F87A
:10F3A0006C007047F037FF1F322898BF034A0346AE
:10F3B0009ABFA2F86E30012000207047F037FF1F7F
:10F3C000014BB3F86E007047F037FF1F044A9042BC
:10F3D00098BF044A03469ABFD365012000207047B6
:10F3E000E0930400F037FF1F014BD86D704700BF5A
:10F3F000F037FF1F044A904298BF044A03469ABF61
:10F40000936501200020704780DF1710F037FF1F41
:10F41000014B986D704700BFF037FF1F012898BF60
:10F42000034A03469ABF82F86930012000207047E2
:10F43000F037FF1F034B93F86900003018BF01201D
:10F44000704700BFF037FF1F08B54FF6FE739842B4
:10F4500001D9002008BD03460549064A08789BB239
:10F460001946A2F87030F9F767FD012008BD00BF0A
:10F470001000FF1FF037FF1F014BB3F870007047FB
:10F48000F037FF1FB0F5805F01D30020704708B54B
:10F49000034BA3F87200F9F721FB012008BD00BF60
:10F4A000F037FF1F014BB3F872007047F037FF1FB2
:10F4B000014B986701207047F037FF1F014B986F91
:10F4C000704700BFF037FF1FB1F5803F0AD208B583
:10F4D0000E4A1278824210D00D4A1278824203D02E
:10F4E000002008BD002070478BB20A4A1946A2F8D6
:10F4F0007630F9F721FD012008BD8BB2054A194687
:10F50000A2F87430F9F718FD012008BD1100FF1FA3
:10F510001200FF1FF037FF1F084B1B78834208D0F3
:10F52000074B1B78834206BF064BB3F876000020DA
:10F530007047044BB3F87400704700BF1100FF1F01
:10F540001200FF1FF037FF1F014BD86701207047E3
:10F55000F037FF1F014BD86F704700BFF037FF1F18
:10F56000014B1868704700BF0086FF1F014B1868E9
:10F57000704700BFF885FF1F014B1868704700BF38
:10F58000F485FF1F014B1868704700BFEC85FF1F13
:10F59000014B1868704700BFFC85FF1F014B1868BE
:10F5A000704700BFE085FF1F014B1868704700BF20
:10F5B000E885FF1F014B1868704700BFE485FF1FF7
:10F5C000014B1868704700BFF085FF1F014B18689A
:10F5D000704700BF5C47FF1F014B1860704700BFBA
:10F5E0000086FF1F014B1860704700BFF885FF1FA2
:10F5F000014B1860704700BFF485FF1F014B186076
:10F60000704700BFEC85FF1F014B1860704700BFBB
:10F61000FC85FF1F014B1860704700BFE085FF1F8E
:10F62000014B1860704700BFE885FF1F014B186051
:10F63000704700BFE485FF1F014B1860704700BF93
:10F64000F085FF1F014B1860704700BF5C47FF1F2C
:10F65000054B10B40022012418705C721A725960B4
:10F66000DA6010BC704700BFC822FF1F024B0022A7
:10F670005A721A72DA607047C822FF1F014B187A5B
:10F68000704700BFC822FF1F014B587A704700BF68
:10F69000C822FF1F014BD868704700BFC822FF1F58
:10F6A000064BDA6801320021B2F57A7FDA6019611F
:10F6B00002D159721972D960704700BFC822FF1F6A
:10F6C000F0B4154D154E2C693668013484B004AF82
:10F6D000B44207E90F002C6117DB2B7AABB1EB6862
:10F6E000B3F57A7F11DA1F010D4A009ED65101331E
:10F6F0003A44019C02980399EB600026B3F57A7FA7
:10F7000054609060D1602E6102D004B0F0BC7047AC
:10F710006E722E72EE60F8E7C822FF1F3C00FF1FDA
:10F720006047FF1F4FF47A70704700BF4FF47A5064
:10F73000704700BF04207047B0F57A7F0BDA0329C9
:10F7400001DD0220704701EB8001044B53F82130AA
:10F750001360002070470120704700BF6047FF1F03
:10F760000A2807D8DFE800F00611150A0E0E060673
:10F7700006060E00094B00225A617047074B032210
:10F780005A617047054B58617047044B01225A611A
:10F790007047024B02225A61704700BFC822FF1F08
:10F7A000014B5869704700BFC822FF1F014B18600A
:10F7B000704700BF3C00FF1F014B1868704700BF37
:10F7C0003C00FF1F10B5144B1C78062C08D8DFE84E
:10F7D00004F00713171B1F0C04005A68904207DD42
:10F7E00001221A7200225A7210BD5A688242F7DC56
:10F7F0001A7A012AF6D010BD59689142F8DDEFE778
:10F8000059688A42ECDCF3E75A688A42E8DCEFE7A1
:10F810005A689142E4DCEBE7C822FF1FB0F5803F55
:10F820001DDBB0F1807F33DBB0F1805F3BDAB0F1FC
:10F83000806F3A4A4FDB0315D35C9B015A1C90FB47
:10F84000F3F31A445210531C90FBF2F213445B1072
:10F8500003FB03F2904209DA013B18467047FF2888
:10F8600006DC002857DB2D4B1B5C1B091846704734
:10F87000B0F5805F294A26DBB0F5804F41DB0312EB
:10F88000D35C013303FB03F29042E5DB184670477B
:10F89000B0F5801F214A0FDBB0F5800F29DB031480
:10F8A000D25C1201CFE7B0F1804F18DB1C4B9842BD
:10F8B0002CDD4FF6FF73D9E7B0F5802F1DDB031366
:10F8C000D25C9200BFE7B0F5806F0DDB0311D35C13
:10F8D0009B080133D6E78314D35C5B01AEE70F4A84
:10F8E0008315D35CDB01A9E78310D35CDB0801330C
:10F8F000C8E78313D25CD200A5E78312D25C520022
:10F90000A1E78311D35C5B080133BBE7034A03160D
:10F91000D35C1B0292E74FF0FF33A7E7F0880100AA
:10F920000080FE7FB0F5806F14D2B0F5007F08D262
:10F93000FF2895BF0A4B0B4BC018181A90F800010E
:10F940007047B0F5407F07D3074B181A90F80001B5
:10F950004042704700207047044BC05C40427047F3
:10F96000F0880100EF8A0100EF8C0100F0870100B0
:10F97000904203DC8842B8BF084670471046704783
:10F98000904203D8884238BF0846704710467047F7
:10F9900030B5DDE90345844275EB010E07DB90428B
:10F9A00071EB030400DB30BD1046194630BD204624
:10F9B000294630BD70B514460E4608F02BF80546B2
:10F9C000204608F023F804460146284608F02AF9A4
:10F9D0000146284607F068FF0546304608F01AF849
:10F9E000214608F01FF90146284607F05FFF08F09E
:10F9F0002BFA70BD30B4029C0568E31A8A1A02FA29
:10FA000003F32B44036043FA04F030BC704700BF9B
:10FA100044F6E612030C13FB02F3002B00B2B8BF4E
:10FA200003F5FF4310FB02F2B8BF7F33002A84B016
:10FA3000B8BF02F5FF42C3F3CF33B8BF7F32ADF892
:10FA40000C0003EBE2321344BDF80C205B420020B3
:10FA50009BB262F30F0063F31F4004B0704700BF16
:10FA6000B0F90210B0F9003010B401FB01F20F4CF4
:10FA700003FB0322A24216D9120E3A3A0C4C34F878
:10FA8000122002FB03F3002B02FB01F2BCBF03F5C3
:10FA9000FF437F33002ABCBF02F5FF427F32DB13F6
:10FAA000D2130380428010BC704700BF0044FA3A72
:10FAB000F08A01001F49B0F90020B1F90030B1F916
:10FAC000021010B4B0F9024002FB03F00028B8BFE6
:10FAD00000F5FF4002FB01F204FB01F1B8BF7F30EB
:10FAE0000029B8BF01F5FF4103FB04F3B8BF7F3124
:10FAF000002B83B0B8BF03F5FF434FEAE03000EBC3
:10FB0000E131B8BF7F33002AB8BF02F5FF42ADF83C
:10FB10000410B8BF7F32BDF80410DB13A3EBD2335F
:10FB200000209BB261F30F0063F31F4003B010BCD1
:10FB3000704700BFE022FF1FA0F50040C0F389100E
:10FB400000F44073B3F5807F82B03FD029D9B3F57C
:10FB5000007F19D0B3F5407F35D1244BC0B203EB01
:10FB60004002400080F4FF70B2F88C2018445242EA
:10FB7000B0F98C3012B292B200209BB262F30F0047
:10FB800063F31F4002B07047C0B2184A430083F4C9
:10FB9000FF73134402EB4000B3F98C20B0F98C30B2
:10FBA000E9E783B9C0B2114A430083F4FF731344F9
:10FBB00002EB4000B3F88C20B0F88C3052425B422C
:10FBC00012B21BB2D7E700231A46D4E7C0B2074AE5
:10FBD000430083F4FF73134402EB4000B3F88C300E
:10FBE000B0F98C205B421BB2C5E700BFF08A010070
:10FBF00010B5044682B00846FFF79EFF1C4AB4F9D0
:10FC00000030106002B203FB02F1B4F90240002997
:10FC10004FEA2040B8BF01F5FF4103FB00F304FBAE
:10FC200000F0B8BF7F310028BCBF00F5FF407F3037
:10FC3000002BB8BF03F5FF4302FB04F24FEAE131AA
:10FC4000A1EBE030B8BF7F33002AADF80400BCBFA1
:10FC500002F5FF427F32BDF80410DB1303EBD23311
:10FC600000209BB261F30F0063F31F4002B010BD90
:10FC7000E022FF1F032923D8DFE801F01C140C0247
:10FC8000104B400080F4FF701844B0F88C004042E4
:10FC900000B270470B4B03EB4000B0F88C004042C1
:10FCA00000B27047074B400080F4FF701844B0F971
:10FCB0008C007047034B03EB4000B0F98C00704799
:10FCC00000207047F08A010000230022C0E90223CF
:10FCD000002303608361704770B5124C2368C31A18
:10FCE000002BB8BF5B42B3F57A7F1ADB054660682C
:10FCF0000026FFF771FCA0686660FFF773FCE06800
:10FD0000A660FFF775FC2069E660FFF777FC606985
:10FD10002661FFF779FCA0696661FFF77BFCA661AD
:10FD2000256070BDE422FF1F024A5368013353600F
:10FD3000704700BFE422FF1F024A936801339360BB
:10FD4000704700BFE422FF1F024AD3680133D3602B
:10FD5000704700BFE422FF1F024A13690133136199
:10FD6000704700BFE422FF1F024A53690133536109
:10FD7000704700BFE422FF1F024B586900EB800070
:10FD800040007047E422FF1F024A936901339361E8
:10FD9000704700BFE422FF1F024B986900EB800010
:10FDA00040007047E422FF1F124B1A88013A12B23A
:10FDB000002A02DA00231846704770B45E680021FA
:10FDC000541804EBD474641004EB440506EB85036B
:10FDD00036F82550854209D004F1FF3304F10104BF
:10FDE0008CBF1AB221B28A42EADA0023184670BCEC
:10FDF000704700BF4423FF1FCB071DD5002A18BF43
:10FE000001301F4B00EBC00040009A68135A591E86
:10FE100010441D2912D8DFE801F01E1E201C1E20F0
:10FE20001C1C22221111111111111111111111118A
:10FE3000111111111111111E1044E2E71E2B17D8D8
:10FE40000120104A00FA03F3134205D113F4C87FCE
:10FE500010D00420704701207047022070470379BA
:10FE6000C289022B0CBF084B084B53F82200704785
:10FE70000020704713F0480F0CBF0020022070478D
:10FE80004423FF1F260000409C14FF1F9493010091
:10FE9000F8B50C4615461E46FFF786FF00283DD0F4
:10FEA0000279A242034602D84FF48170F8BD027A6B
:10FEB000D20736D4B0F802C0BD4904EB0C0202EB05
:10FEC000C20288685200811891F804E0CF88BEF120
:10FED000000F39D1835A1E2B3DD8DFE813F02301E0
:10FEE0004701410161015A0154014D0134012901C9
:10FEF0003C003C003C003C003C003C003C003C0022
:10FF00003C003C003C003C003C003C003C003C0011
:10FF10003C003C003C003C003C003B0140F2011036
:10FF2000F8BD4288A249002C0CBF1346531C03EBBA
:10FF3000C30388685B00C11891F804E0CF88BEF164
:10FF4000000F0BD1C35AC6E7BEF1020F00F0A48028
:10FF5000BEF1010F18D000232B60A5E7002C0CBFC9
:10FF60001146511C01EBC101490043181B79022BBA
:10FF70004ED0002C0CBF1446541C04EBC404620089
:10FF800083181B79012BE6D1835A1E2BE3D801A2DB
:10FF900052F823F025010100770201006B020100F5
:10FFA0005D0201004F0201005703010049030100F7
:10FFB0003B0301002D0301001D0301000D0301009F
:10FFC00057FF000057FF000057FF000057FF0000D9
:10FFD00057FF000057FF000057FF000057FF0000C9
:10FFE00057FF000057FF000057FF000057FF0000B9
:10FFF00057FF000057FF000057FF000057FF0000A9
:020000021000EC
:1000000057FF000057FF000057FF000001030100E9
:10001000435A1E2B9FD801A252F823F0250101005C
:100020002F0201002B020100270201002302010020
:100030001F0201000702010003020100EB010100A1
:1000400057FF000057FF000057FF000057FF000058
:1000500057FF000057FF000057FF000057FF000048
:1000600057FF000057FF000057FF000057FF000038
:1000700057FF000057FF000057FF000057FF000028
:1000800057FF000057FF000057FF000057FF000018
:1000900057FF0000D9010100825A1E2A3FF65BAFCC
:1000A00001A151F822F000BF25010100E502010085
:1000B000D7020100C9020100BB020100AD0201002C
:1000C0009F02010091020100830201004B02010026
:1000D0003302010057FF000057FF000057FF0000E8
:1000E00057FF000057FF000057FF000057FF0000B8
:1000F00057FF000057FF000057FF000057FF0000A8
:1001000057FF000057FF000057FF000057FF000097
:1001100057FF000057FF000057FF000057FF000087
:10012000F302010000232B6040F215203360F8BD7C
:10013000204B042203EB87032B603260002B3FF43B
:10014000B3AE0020F8BD1C4B042203EB87032B60E9
:100150003260F3E7194B01223B442B603260EDE73C
:10016000174B01223B442B603260E7E7154B01221D
:100170003B442B603260E1E7134B022203EB470361
:100180002B603260DAE7114B01223B442B60326076
:10019000D4E70F4B042203EB87032B603260CDE7DB
:1001A0000C4B022203EB47032B603260C6E700BF13
:1001B0004423FF1F3423FF1F9C14FF1F2C23FF1F0A
:1001C0004023FF1F3023FF1F2415FF1F4415FF1F6F
:1001D0003823FF1F3C23FF1F624B53F82730013C9D
:1001E000234401222B603260A8E75F4B53F827308D
:1001F00004F18044013C03EB840304222B60326051
:100200009CE75A4BF2E75A4B53F8273004F100446D
:10021000013C03EB440302222B6032608EE7554B16
:10022000DBE7554BE2E7554BEEE7554BD5E7554B32
:10023000D3E7554A52F827702F60197A2246604654
:10024000FFF7DAFD3B46306078E7504AF2E7504B63
:10025000042203EB87032B6032606FE74D4B0222D1
:1002600003EB47032B60326068E74B4B01223B44B2
:100270002B60326062E7494B01223B442B603260C5
:100280005CE7394B042253F827302B60326055E786
:10029000364B042253F827302B6032604EE7344B44
:1002A000022253F827302B60326047E7314B01229E
:1002B00053F827302B60326040E72F4B042253F86D
:1002C00027302B60326039E72C4B022253F827305D
:1002D0002B60326032E72A4B012253F827302B6023
:1002E00032602BE7274B012253F827302B60326016
:1002F00024E71C4B012253F827302B6032601DE7A6
:10030000274B01223B442B60326017E7254B53F803
:100310002700286006F004FE306012E7224B53F8F5
:100320002700286006F0FCFD30600AE71F4B04221E
:1003300003EB87032B60326000E71D4B042203EBC5
:1003400087032B603260F9E61A4B022203EB470366
:100350002B603260F2E6184B01223B442B60326086
:10036000ECE600BFD8910100E0910100E4910100AA
:1003700064920100A0920100C49201004493010024
:100380006C930100DC910100C8910100CC91010047
:100390003494010054940100689401008C9301008E
:1003A00088930100789301007C93010090930100F1
:1003B0009493010008940100249401001E2807D89A
:1003C00001230A4A03FA00F0104203D008207047C4
:1003D0000020704710F4C87F01D02020704710F033
:1003E000480F0CBF00201020704700BF26000040BF
:1003F00038B50D461446FFF7D7FCC0B1037A184A4A
:1004000013F0010F438813D15919936801EBC1010F
:1004100003EB41014888082C06D8DFE804F0081CEB
:100420001C0518050505140020F03F0080B238BDFA
:10043000002D0CBF1946591C936801EBC10103EB59
:1004400041014888E7E720F01B0080B238BD20F06A
:100450002D0080B238BD20F0360080B238BD00BF1C
:100460004423FF1F2DE9F04182B0154601AA06463C
:100470000F469846FFF70CFD044618B1204602B01F
:10048000BDE8F08100F06AFE394602463046FFF7CB
:10049000AFFFC30405D4019B2B60204602B0BDE82A
:1004A000F081D8F800200199284607F077FFE5E7AA
:1004B0002DE9F04383B000240E46914698460194FE
:1004C0000746FFF771FC48B10379B34204460BD8E5
:1004D0004FF48175284603B0BDE8F08340F2011562
:1004E000284603B0BDE8F08301AB6A463146384682
:1004F000FFF7CEFC05460028ECD100F02FFE314678
:1005000002463846FFF774FFC30409D43246217A05
:100510006088FFF771FC804523D940F20315D9E7C5
:10052000237A194A13F0010F638822D0002E0CBFE2
:100530001E465E1C06EBC606936833F816301E2B6B
:1005400015D80122114902FA03F30B4218D113F412
:10055000C87F17D113F0480F0CBF00230223984522
:10056000DBD142464946009807F018FFB2E7002366
:10057000F5E71E4406EBC606936833F81630DEE74F
:100580001346ECE70423EAE74423FF1F260000405C
:1005900070B50C4615461E46FFF706FC40B30379BE
:1005A000A34203D84FF48173184670BD037A418883
:1005B00013F0010F2A4B1FD10C4404EBC4049B68B9
:1005C00064001A191B5B1289013B1D2B45D8DFE81B
:1005D00003F042403E3C3A3230281F4444444444F5
:1005E00044444444444444444444444444444418F7
:1005F00040F20113184670BD002C0CBF0C464C1C79
:10060000DBE7184B1A4401212A6000233160CBE755
:10061000154B53F82200286006F082FC002330605E
:10062000C2E7124B03EB820204212A6000233160EF
:10063000BAE70F4BF6E70F4B03EB420202212A60A9
:1006400000233160B0E70C4BDCE70C4BEAE70C4BC6
:10065000F2E70C4BD6E70C4BD4E700232B60A3E763
:100660004423FF1F889301007C93010090930100B5
:100670009493010008940100249401003494010033
:1006800054940100689401008C93010038B50D4624
:100690001446FFF789FB50B14289074B53F82200FB
:1006A000286006F03DFC00232080184638BD40F24B
:1006B0000113184638BD00BF9490010070B50E4676
:1006C00015461C46FFF770FB08B3037A124A13F075
:1006D000010F438810D19919936801EBC10103EB15
:1006E00041010A8A0D4B53F82200286006F018FCDD
:1006F00000232080184670BD002E0CBF1946591CDF
:10070000936801EBC10103EB41010A8AEAE740F279
:1007100001132860184670BD4423FF1F7C8D010023
:1007200001282DE9F04F59D0DFF85CB1BBF80C80FF
:10073000BBF800A0D04543D2DBF80430DBF80860FA
:1007400008EB480903EB89094FF6FF7C99F804E0B0
:10075000BEF1000F2CD099F80870B9F802500020B3
:1007600007F00107044609E001306145528883B271
:1007700019D031EA020216D0734518D282B2002A8B
:100780000CBF2A466A1C2B1802EBC20203EBC30300
:1007900006EB420206EB4303002FE5D10130614531
:1007A0005A8883B2E5D101347345A4B2E6D364B963
:1007B00008F101081FFA88F8D04509F10C09C5D1E4
:1007C0004FF000084046BDE8F08F08F10108ABF893
:1007D0000C80B9F800804046BDE8F08F4FF6FF73FB
:1007E000DFF8A4B09942BBF8008047D0B8F1000F01
:1007F00044D008F1FF391FFA89F909F10109DBF842
:1008000004C0DBF8086009EB49090CEB89094FF0DB
:1008100000089CF804E0BEF1000F2BD09CF8080003
:10082000BCF80250002400F0010027460BE052887B
:1008300031EA020204F1010408BF0137A3B208BF84
:10084000BFB2734511D2A2B2002A0CBF2A466A1C5D
:100850002B1902EBC20203EBC30306EB420206EBC9
:1008600043030028E3D15A88E2E71FB108F10108E9
:100870001FFA88F80CF10C0CE145CAD10023ABF843
:100880000C304046BDE8F08F4423FF1F70B50E4684
:1008900015461C46FFF788FA40B1C288437932807A
:1008A0002B700279013A2270002070BD40F20110D5
:1008B00070BD00BF70B50C4615461E46FFF774FAB2
:1008C00028B30379A34202D84FF4817070BD037A34
:1008D000184913F0010F43881CD1234403EBC302D2
:1008E0008B6833F812202A80027A4188D2071AD501
:1008F000002C0CBF0C464C1C04EBC40403EB44045A
:10090000638833802B88002BDED0002070BD40F23E
:10091000011070BD002C18BF013303EBC3028B68BC
:1009200033F81220DFE70C4404EBC40403EB440467
:100930006388E6E74423FF1F30B5A0F5E052103A84
:10094000032A83B01D4603D8E9B9002003B030BDA7
:1009500000F47F43B3F5B05F044602D0B3F5D05F37
:10096000F3D10029F1D0002DEFD101AB294620466B
:100970000DF10302FFF776FD9DF80330002BE4D064
:100980004FF48570E2E701AB0DF103020021FFF7A0
:1009900069FD9DF80330002BD7D0002DD5D140F252
:1009A0000910D3E7044A054B10880549054A188009
:1009B00099605A6000207047C401FF1F4423FF1F45
:1009C0005805FF1FC801FF1F2DE9F0415A4E8768E7
:1009D00032783B7A012A054603F0E0012DD0092A3E
:1009E00002D00020BDE8F081B9BB4288092A40F25C
:1009F0008780C3F34201033A521A746892B2D94312
:100A0000A242C9B2C3F3001353DC4C4F97F800E085
:100A10009E4508D0B2EB040E01F0010118BF4FF063
:100A2000010E8E457FD00A240022284634701146DC
:100A3000434BBDE8F04102F01FB9602931D82029AD
:100A40001ED051BB6B88092B33D80B23284633703B
:100A50000821BDE8F04101F0C9B8602933D14288CE
:100A6000092A4DD9354A1178C3F300139942DAD0D7
:100A7000072471683470BDE8F041137002F084BC43
:100A800013F00204438827D00A2BDED102233370EF
:100A90001146BDE8F04102F03BB940293AD0602947
:100AA000D0D00B23284633700521BDE8F04101F07A
:100AB0009DB80A240022284634701146214BBDE817
:100AC000F04102F0D9B80B22002332707360052187
:100AD000BDE8F04101F08AB8092BB6D917490323C4
:100AE00007F10C0033700A7001F054F96B880A3B6F
:100AF000C31A214628467360BDE8F04102F008B9E8
:100B00000B2200232846327073600821BDE8F041B3
:100B100001F06CB843880A2B97D106233370BDE8E7
:100B2000F04102F047BCA21A042172603B703170A0
:100B3000BDE8F04102F068BC5423FF1F5B15FF1FA6
:100B40000000030501000405034B1A7812B90121C6
:100B50005A601970704700BF5423FF1F0C490B786F
:100B6000013BDBB20A2B0FD8012202FA03F340F259
:100B700001121A4009D113F4C06004D113F0FE0F22
:100B800002D0087070470A70704700230B707047DE
:100B90005423FF1F0D4B1A780A2A02D00B2A02D0C9
:100BA00070475A6812B901221A707047B2F1004FAB
:100BB00002D009221A7070479A681AB901215A6046
:100BC0001970704708221A7002F03AB85423FF1FB8
:100BD00010B504468068063001F0DAF82E4A137822
:100BE000012B00F4704003D0092B24D0022010BD4B
:100BF000B0F5005F37D0B0F5004F07D020460B238B
:100C00000521BDE81040137000F0F0BFA3681B7A07
:100C100003F07F03012B2AD0032B19D0052BEDD134
:100C200063880A2B2ED020460B230821BDE81040F4
:100C3000137000F0DBBFB0F5005F14D020460B242A
:100C4000002314700521BDE81040536000F0CEBFB2
:100C50006388082BE7D120460021BDE810401370BF
:100C6000916001F0A7BD2046BDE81040ACE6638866
:100C7000082BD8D120460021BDE8104013709160A8
:100C800001F070BC204600210823BDE810409160AF
:100C9000137001F051BE00BF5423FF1F154B68B104
:100CA0001A78062A0DD0072A12D0082A01D1062860
:100CB00017D0082810D00A221A70704701221A7023
:100CC00070470428F5D10C4A596001211170F2E7F0
:100CD0000528EED15960EEE700225A600A221A7008
:100CE00070470029CCBF4FF00042002299605A6043
:100CF000E1E700BF5423FF1F5B15FF1F044B1B7868
:100D000003F0F703012B14BF02200020704700BF3F
:100D10005423FF1F0349044A044B0020087010802D
:100D2000188070476023FF1F0486FF1F0686FF1F81
:100D300010B54FF4186082B002F016FC40F2013397
:100D40001840B0F5407F35D01C48002400F8044B13
:100D500002F0A6FE019402F0D5FD01280ABF22236D
:100D60000123ADF80000ADF802306A464FF00203EF
:100D70004FF0010141F6324018BFADF80040FFF7D7
:100D800097FB01AA0423022141F63240FFF790FBB2
:100D900002230DEB0302012141F63340FFF788FBEC
:100DA00001AA0423022141F63340FFF781FB022010
:100DB00002B010BD002002B010BD00BF6023FF1FB5
:100DC0002DE9F041394F82B0381D02F069FE042050
:100DD00000F096FC364A374B0025022401264FF4DA
:100DE0001A6015801D803E70ADF80240ADF80040DD
:100DF00002F0C8FBBDF8021003460246BDF8000031
:100E0000019305F05DFF40B323466A46314641F643
:100E100032403D70ADF80250ADF800500195FFF73B
:100E200047FB01AA2146042341F63240FFF740FB6D
:100E3000234631460DEB040241F63340FFF738FB01
:100E400001AA2146042341F63340FFF731FB40F26B
:100E50000E28404602B0BDE8F081804623466A462F
:100E6000314641F63240FFF723FB01AA2146042315
:100E700041F63240FFF71CFB23460DF102023146DA
:100E800041F63340FFF714FB01AA2146042341F643
:100E90003340FFF70DFB812242F21071381D02F042
:100EA000FBFD40463E7502B0BDE8F0816023FF1FA8
:100EB0000486FF1F0686FF1F38B50C4B1B784BB10D
:100EC0000B4A13889BB23BB10A4C238800250A2B9E
:100ED000158003D8012038BD002038BD00F03EF950
:100EE0000828F9D02580012038BD00BF6023FF1FEE
:100EF0000486FF1F0686FF1F10B51F4C231D83426B
:100F000000D010BD00F02AF90828FAD1237DC3B122
:100F10001A4B1B889BB2002BF3D000234FF41860B0
:100F2000237502F021FBC30516D442F21074144855
:100F300002F0B6FD214681221148BDE8104002F0C2
:100F4000ABBDFFF7B9FF0028DBD105F0B5FE2C20C3
:100F5000BDE8104000F00EB94FF41A6002F012FB29
:100F6000084B0409A3FB0434E40942F210739C42C9
:100F700038BF1C46DBE700BF6023FF1F0486FF1F4E
:100F80006423FF1FC55A7C0A024B1A1D1A605A645B
:100F9000002070477823FF1FF0B51C4A91F800E04D
:100FA00013684F788E78CD780C7983B0ADF8000057
:100FB000506C8DF802E0191A3F298DF803708DF8F6
:100FC00004608DF805508DF8064016DC92F8481044
:100FD000012910D00E49581A3F2812DC6C4603CC68
:100FE0000C4C1860012003F10805207000205960A6
:100FF000156003B0F0BD8342ECD140F2092003B08C
:10100000F0BD01200B4682F84800E7E77823FF1F78
:101010007C23FF1F0986FF1FF0B587B0FFF76EFE28
:1010200018B10124204607B0F0BD01A800F058FD1A
:1010300018B10224204607B0F0BD314D2A686B6C10
:10104000D11A3F293CDD2F4A991A3F2904DD00219E
:101050006A64134685F84810019A186859689468BC
:1010600000260A2704AB03C357809680A01D967103
:101070004FF4805100F090FE019BBDF8101098686D
:10108000083000F089FE314602AB03AA41F20100AC
:10109000FEF7FEFE0198039A836812789A7206ABF7
:1010A000826853F8061DC2F80B101B79D373032115
:1010B00000F02EFD044670B1019B02241E70B1E7C2
:1010C0009A42C0D195F84820002ABCD1019B40F239
:1010D00003241A70A6E701460720FFF7DFFD6B6CBB
:1010E0002A680833D11A3F296B649BDC9A4299D154
:1010F00095F84830002B95D1034B1C7092E700BF48
:101100007823FF1F7C23FF1F0986FF1F70B50E4C3D
:1011100010F010030D4600F00F06218018BF0123C8
:1011200001464FF49870E370A67002F043FA294626
:101130004FF49A7002F03EFA2A46E1783046BDE854
:10114000704005F08FBD00BFC223FF1F0123024A7C
:10115000184600219370D9E7C223FF1F014B9878EE
:10116000704700BFC223FF1F014B1888704700BFA4
:10117000C223FF1F10B5194CA378A080013B072B99
:101180002AD8DFE803F02119291129292904142379
:101190000120E38000F080FEA088E3880146184625
:1011A000FFF7B4FF002010BD142301461846E3806A
:1011B000FFF7ACFF002010BD122301461846E38064
:1011C000FFF7A4FF002010BD112301461846E3805D
:1011D000FFF79CFF002010BD022010BDC223FF1F9F
:1011E000F8B588B1A34CA378013B0546072B08D876
:1011F000DFE803F00438072607070741012D00F058
:10120000078102263046F8BD9A4C4FF4907002F0E8
:10121000ABF9A378013B072BF3D801A252F823F0D6
:101220009B1201001113010003120100EB120100D7
:10123000031201000312010003120100C112010098
:10124000012800F07F81022DDBD1E378002BD8D17B
:1012500028461B221423A280E38002F00FFAE088C4
:10126000A1883DE00128CCD1E578002D00F0448133
:10127000002EC7D132E0012D00F04D81022DC0D1EA
:10128000E378002BBDD11B2214230120A280E38030
:1012900000F002FEE088A18822E010F010014AD0A0
:1012A00000F00F000138072800F21C81DFE810F081
:1012B0009B00A500A00077001A011A011A0177000F
:1012C000E37800F00F00002B4ED0022800F0D4800D
:1012D000042800F05881012800F04881E088A188A6
:1012E0000026FFF713FF3046F8BD10F0100349D079
:1012F00000F00F000138072800F2F980DFE810F055
:101300009A0091008C00B000F700F700F700A500EC
:1013100010F010031BD000F00F000138072800F276
:10132000DB80DFE810F0420050004B005500D90090
:10133000D900D9004B00E37800F00F00002BB1D0AA
:10134000012852D011202188E080A180C8E7E278EE
:1013500000F00F00002AE0D0012800F05281122096
:101360002188E080A180BBE7431E072B00F2D180DB
:10137000DFE813F09A008E00AB00A100CF00CF0091
:10138000CF00AD00E27800F00F00002AB2D00128B3
:1013900000F03E8114202188E080A180A0E7112385
:1013A0001946A380E38018469AE701220023E280D1
:1013B000A38000F083FBE088A18891E7112112202F
:1013C000A180E0808CE702200021E080A18087E7F7
:1013D000032000F07BFD002800F0E8801E21122091
:1013E000A180E0807CE701200021E080A18077E7F8
:1013F00013211120A180E08072E7022000F000FBA1
:10140000002800F0F68016211120A180E08067E717
:1014100002F048FA0226F5E611211420A180E080AE
:101420005EE702220023E280A38000F045FDE08811
:10143000A18855E701220023E280A38000F03EFB53
:1014400000F03AFDE088A1884AE7637A002B00F0BB
:10145000A480FFF731FD002840F09F800126D1E6EF
:10146000042200230220E280A38002F0F9F8E08841
:10147000A18835E7C223FF1F2388A3800120122300
:10148000E38000F009FD00F017FDE088A18827E760
:1014900002220023E280A38000F00EFD012000F074
:1014A000FBFCE088A1881BE701250023E580A380E1
:1014B00000F004FBF0E7002304221846A380E2803A
:1014C00000F0EAFCE088A1880AE71122DCE60823A4
:1014D0000021E380A18003E712231946A380E38063
:1014E0001846FDE612211120A180E080F8E61221C5
:1014F0001420A180E080F3E6022000F081FA0028A9
:1015000040F0B680022602F0CDF9002E7FF47AAECC
:10151000E4E61222B8E6E778002F7FF4A9AE0220B5
:1015200000F06EFA064600284AD0162211232846FB
:10153000A280E3803E4600F0AFFC00F0BDFC00F06E
:10154000BDFAE0E7E578002D7FF4C8AE022000F098
:1015500057FA0646002841D016221123A280E380C4
:101560002E4600F0A9FC00F0A9FACCE72388A3805E
:101570001123E38000F090FC00F09EFC00F09EFA46
:10158000E088A188ACE62388A38001201423E380AF
:1015900000F082FCE088A188A2E608220023E28015
:1015A000A38000F001FEE088A18899E6022000F007
:1015B0008DFC002843D01D211220A180E0808FE601
:1015C000032000F083FC28B31E221223A280E380B4
:1015D00000F072FC284600F05FFC94E7032000F066
:1015E00075FCF8B11E221223A280E38000F064FC97
:1015F00089E70223A080E38000F044FAE088A18814
:101600006EE6E080A38000F059FAE088A18867E6E2
:10161000E08012E7022000F059FC00283FF472AF8E
:101620001D22D2E7022000F051FC00283FF46AAFEF
:101630001D221223A280E38000F03EFC63E7FFF747
:1016400077FB10B9FFF7BCFBD0B9FFF771FB08B10E
:10165000237AABB9FFF76CFBB8B90123637204229C
:101660000023E280A38000F0EDFDE088A18837E64A
:10167000162211232E46A280E38000F01FFA42E7D3
:1016800036211220A180E0802AE600236372E6E77B
:1016900010B5FFF787F9044608B1204610BD01F0E8
:1016A000A5FF00F093F904460028F6D1FFF74EFDA0
:1016B000FFF76AFC04460028EFD1FFF72BFB044636
:1016C0000028EAD14FF4A77001F04EFFC30701D5FF
:1016D0000224E2E7034B21464FF401701C6001F045
:1016E00075FFDAE7CC23FF1F044A1368034319464A
:1016F0004FF40170136001F069BF00BFCC23FF1FDE
:10170000044A136823EA000319464FF4017013607A
:1017100001F05CBFCC23FF1F10B582B005F0C0FA0A
:10172000044640F68E1001F01FFF0B4BADF806008B
:101730001A78BDF806101AB908490A8803320A80D7
:1017400007490120002208801A7014B1032002F01A
:1017500033F802B010BD00BF0886FF1F0686FF1FCA
:101760000486FF1F38B51D4B1D4D1C684FF40870D3
:1017700001F008FF0440620504D52B78D3B902209C
:1017800002F01AF8230511D52B781BB914F4406F19
:101790001AD138BD02F0B6F8022807D1114A124911
:1017A0001388012008700BB1013B13802B78002BAC
:1017B000ECD038BD0B4A0C49138801200870002B6F
:1017C000DDD0013B1380DAE705F06AFA0028E0D0AB
:1017D0000320BDE8384001F0EFBF00BFCC23FF1F5E
:1017E0006023FF1F0686FF1F0886FF1F38B54FF4D2
:1017F000087001F0C7FE434D6C6808B9002C6CD02E
:101800000443600626D42B7A012B71D0E30758D409
:10181000A0054BD4E1053ED4E20632D43A4C4FF455
:10182000887001F0A1FE23888342054602D005F0AE
:1018300045FA2580354B1A783AB9354B1B7803B9F0
:1018400038BDBDE83840FFF7E7BB00221A7002F050
:10185000BBF8F2E74FF4886001F086FEC1072B7AEF
:10186000D2D4002BD0D101232B7205F023FA00280B
:10187000C9D1FFF773FC0828C5D10220FFF7B0FCDF
:10188000C1E7FFF771FC0028C8D102F017F801206A
:10189000FFF7A6FCC2E700F0DBF96B6801280CBF7C
:1018A00043F4807323F480736B60B5E700F066F94E
:1018B0006B6801280CBF43F4007323F400736B6062
:1018C000A8E70020FFF78CFC6B6801280CBF43F0F1
:1018D000010323F001036B609AE740F6050001F075
:1018E00035FE03079AD56B6843F480736B6095E708
:1018F0004FF4886001F038FEC20744BF00232B720A
:1019000084E700BFCC23FF1F5C15FF1F4136FF1F7C
:101910000986FF1F2DE9F04182B000268DF807608F
:10192000C0B1022304460370012001F0B5FE8046D9
:10193000012001F0C9FE0E4A63881568A1689C1D4C
:10194000A4B24544074622462846334601F04AFEE3
:10195000A74202D802B0BDE8F081781E2844334681
:1019600001220DF1070101F03DFE02B0BDE8F0815A
:101970000C86FF1F38B5044601200D4601F0A4FE79
:1019800063885A1D824202DB40F2022038BDA26801
:101990000D4913701B0A5370A288A0680B788270DF
:1019A000120AC270A268A0791071072BA26845EADA
:1019B00003151ABF0133DBB20123204655710B70AA
:1019C000FFF7A8FF002038BD5E15FF1F70B40A4B5B
:1019D0000A4AFF21002003F1280603F2EA5503F624
:1019E000AC345170DE609D615C62187018711874BF
:1019F000187770BC704700BFD823FF1F5E15FF1F0C
:101A00000238012801D90220704708B5002001F0F2
:101A10005BFE21282FD940F6060001F097FDC20792
:101A20002CD5002001F038FEB0F5805F1AD30120DC
:101A300001F04AFE21281ED940F60E0001F086FD75
:101A4000C3071BD5012001F027FEB0F5805F09D345
:101A5000002001F051FE012001F04EFE002001F0B7
:101A60006FFE10B140F20D2008BD012001F068FEAC
:101A70000028F7D108BD40F20B2008BD4FF40370D9
:101A800008BD00BF10B50B4C2378012B10D00023EC
:101A9000094A23711846FF2123742377517001F0FE
:101AA000DFFD012001F0DCFD01232370FFF74CF87E
:101AB000002010BDD823FF1F5E15FF1F10B5074C77
:101AC00023784BB1FFF74AF8002001F0D7FD012041
:101AD00001F0D4FD0023237010BD00BFD823FF1FE9
:101AE0000A4A137C63B1137F23B1002303600223EE
:101AF00018467047012102F81C1F02601846704703
:101B0000012102F8101F026018467047D823FF1FFA
:101B1000064B1B7813B94FF4007070470378012B04
:101B200002D040F20120704724E700BFD823FF1FF6
:101B300010B5114C237C032B1AD0237F032B00D02C
:101B400010BD012304F81C3F012140F60F0001F0F5
:101B500025FD40F60D0001F0F9FC10F00801F8D168
:101B600040F60F0001F01AFD2046BDE81040D1E616
:101B7000012304F8103FE7E7D823FF1F30B5194CC5
:101B800083B0237800228DF8072013B9022003B018
:101B900030BD154B01201D6801F07EFD01231A4662
:101BA00028440DF1070101F01DFD237C022B07D015
:101BB000227F022A11D0FEF7EDFF002003B030BDD6
:101BC00003232374237F0222032BF4D102EB42026E
:101BD00004EB820400232371EDE703222277012224
:101BE000F2E700BFD823FF1F0C86FF1F38B5174B45
:101BF0001A7CC2B91C46012204F8102F8288A280E8
:101C0000042565808079A268A07101250020957166
:101C1000D0711A78A3680D0A19725D723AB900235F
:101C20002370022038BD1A7F5AB1022038BD2378B4
:101C3000012BF4D101462046FFF79CFE0028EED18F
:101C400038BD1C46012204F81C2FD7E7D823FF1FFC
:101C50002DE9F047484C82B0237800208DF805002C
:101C60001BB9022002B0BDE8F087444B1E6801F0AA
:101C700013FD371800F5805539460DF10600012394
:101C80000222354401F0B0FC26791EB1012002B0D9
:101C9000BDE8F0874FF00108304684F8048001F079
:101CA00013FDA5F6FB7A8146434601A842465146FC
:101CB00001F09AFC9DF80400DFF8D0E0C0F30210B8
:101CC0008DF8040018B19EF80130834238D001230A
:101CD0001A468EF8010051460DF1030001F084FC14
:101CE000BDF806209DF80360E0680632002392B23A
:101CF00006F00F0639468DF8036001F075FCBDF85B
:101D0000063099452CD81E48E38002220123A5F60F
:101D1000FE7101F069FC01231A46A5F6FC71194811
:101D200001F062FC9DF80330032B15D00221164808
:101D3000FFF75CFF01284FF0000093D0207191E77E
:101D400009F1FF310DF1060039444346424601F0E6
:101D50004BFC2671022085E70B48FEF739FFE9E7C7
:101D6000012309F1FF311A4639440DF1050001F054
:101D70003BFCBDF80630C6E7D823FF1F0C86FF1FCB
:101D8000E023FF1FE223FF1FDC23FF1F5E15FF1F61
:101D900000887047006870470B0A017043707047F5
:101DA00010B40A0C0C0A0B0E447001708270C370E0
:101DB00010BC704749B942B9012826D0354B998DDE
:101DC00009293AD940F207207047F0B50E4683B092
:101DD00014461F46054601AB6A4621463046FEF7CB
:101DE00057F818B140F2011003B0F0BD019B3B80E1
:101DF000082221463046FEF7FBFA012D10D00106DD
:101E000016D440F2072003B0F0BD224B19880529F3
:101E1000D8D803EBC100013142601980002070471F
:101E20004406EED510F0380F24D140F20510DBE760
:101E3000420709D14FF48270D6E703EBC1000131AC
:101E40000263998500207047214630460422FEF740
:101E5000CFFA4307EED00F4B998D0929D1D80098BE
:101E600003EBC102106308B138889086013199856F
:101E70000020B9E7074B19880529C2D8009803EB61
:101E8000C102506008B138881081013119800020EA
:101E9000AAE700BF4835FF1F10B50446054801F00A
:101EA000FFFD012C01D0002010BD022001F0E6FB57
:101EB000002010BDC035FF1F08B5032001F0DEFB78
:101EC000022001F0DBFB002008BD00BF2DE9F04F30
:101ED00083468FB04FF48060FFF712FC4FF4006030
:101EE000FFF70EFC0BAB09AA00214FF4E050FEF700
:101EF000B9FA28B140F2062528460FB0BDE8F08FA8
:101F0000BBF1030F054609D0BBF1020FF2D1844BA0
:101F1000188001234FF0030A039305E0804B988556
:101F200002234FF0040A03939DF82430022B40F261
:101F3000E7800BF58073DB009A1D07330192029353
:101F40000324049506E001349DF82430E4B2A34252
:101F5000C0F0D5800BAB0DF1250221464FF4E050C7
:101F6000FEF780FA0028C5D19DF825305345EAD107
:101F7000584601F091FBB0F5805FC0F0CD80584627
:101F800001F0A2FB0546019801F0E0FAC20702D475
:101F9000002D40F0C180029801F0D8FA10F0010F36
:101FA00058464FD101F0A8FB584601F0C9FB054641
:101FB000002D40F0B18004F5E0570F3738460BABE9
:101FC0000DF126022946FEF74DFA002892D101981C
:101FD00001F0BCFAC307B6D5584601F075FB9DF871
:101FE0002630814600283AD1002BACD00125CDF80F
:101FF00014A0DDF80CA006940BAB0AAA29463846BB
:10200000FEF730FA00287FF475AFBDF82880ADF8F0
:102010002A0028F4FF73BAF1010F23F0010323D043
:10202000B3F5D05F23D041460DF12A03002250467C
:10203000FFF7C0FE00286CD040F2072528460FB0FD
:10204000BDE8F08F01F00CFB584601F055FB5846F7
:1020500001F076FB0546584601F010FBA8E7002B7F
:102060005AD0A9460125C2E7B3F5B05FDBD10DAB6D
:102070000DF1270200214046FEF7F4F90028DBD1DC
:102080009DF8274044B30446064607950136F6B24C
:102090000DAB31460CAA4046FEF7E4F90DF12A03D8
:1020A0000028C9D10C995046C1F3C405C1F30722D9
:1020B000090CADF82A500D95FFF77CFE0028BBD126
:1020C000BDF82A300D9A1C449342A4B2B4D19DF8B5
:1020D0002730B342DAD8079D9DF826300135EDB29E
:1020E000A144AB421FFA89F986D25846DDF814A004
:1020F000069C01F0E9FA81457FF625AF9CE7049D37
:102100004FF48060FFF7F0FA4FF40060FFF7ECFA4D
:10211000F2E6BDF82A40DFE74FF40275ECE600BFB7
:102120004835FF1F2DE9F047DFF870A0DFF8709009
:10213000DFF87080DAF80070B9F80C30B8F80050A9
:1021400082B01F449DB10024254608EBC40601233C
:1021500032897068394601F047FA01343389B8F89A
:102160000020E4B21D44A242ADB21F44EDD8B9F83C
:102170000E30AB420CD9B9F80C20DAF80010134439
:102180005A1E012311440DF107001A4601F02CFAE2
:1021900004F012FD02B0BDE8F08700BF0C86FF1FFF
:1021A0001086FF1F4835FF1F08B5822242F21071CA
:1021B000034801F071FCFFF7B5FF002008BD00BF28
:1021C000C035FF1F2DE9F047DFF86CA0DFF86C90F9
:1021D000DFF86C80DAF80070B9F81230B8F82C50DB
:1021E00082B01F449DB10024254608EBC40601239C
:1021F000B28E316B384601F0F5F90134B38EB8F880
:102200002C20A4B21D44A242ADB21F44EDD8B9F8AF
:102210001430AB420CD9B9F81220DAF8000013449C
:102220005A1E012310440DF107011A4601F0DAF994
:1022300002B0BDE8F08700BF0C86FF1F1086FF1FAD
:102240004835FF1F08B5FFF7BDFF022001F008FA6F
:10225000032001F005FA4FF48060FFF751FA4FF4C4
:102260000060FFF74DFA022001F02EFA40B902207B
:1022700001F042FB4FF40060FFF736FA002008BD82
:10228000012001F039FB4FF48060FFF72DFA0020A8
:1022900008BD00BF2DE9F04F89B0884693460193F1
:1022A000074600285AD18DF810200025AA465C4622
:1022B0004FF0010906AB07AA21464046FDF7E8FDAD
:1022C000012F064603461BD0B6BB05AB0DF112022B
:1022D00021464046FEF7EEFABDF8143013F4805F55
:1022E00008BF4FF00009012F11D0069B9DF8102068
:1022F0001D44B246ADB20134E4B29442DAD913E0DF
:1023000040F215229042DFD19DF81020F3E7BDF88E
:102310001230012B14D0B246069B1D44ADB29DF87D
:102320001020002CE7D1B2B9B9F1010F129B2BD0CC
:10233000AB422BD940F20313184609B0BDE8F08F29
:10234000BAF1080F1ED00AF1010A5FFA8AFABAF14F
:10235000010FE4D8E0E70135ADB2CCE704AB0DF1F5
:102360000F020DF112014046FEF790FA03460028D5
:10237000E2D19DF810305B4597D2129B002BD9D14A
:102380000023D9E7BA46C7E7AB42D3D15A45F7D3C2
:10239000DFF84091DDF804A001265C4606AB07AAF1
:1023A00021464046FDF774FD012F15D0002873D15A
:1023B000FEF7D4FE214602464046FEF719F810F01B
:1023C000380FADF8140012D1002F38D140F20513A8
:1023D000184609B0BDE8F08F40F215239842E5D1C8
:1023E00001349DF81030E4B2A342D7D2C8E75FBBF6
:1023F000BDF81850D34601263B465A462146404672
:10240000FEF79AFA002847D1BDF8143013F4805F24
:10241000079B39D159462A46184605F0BFFF224688
:102420004146384604F0CEFB002842D1069B9A4430
:10243000002FD5D0002CD3D10AF1010AD0E7069B9A
:102440009A44002CCCD1F7E70DF116030DF11202DE
:1024500021464046FEF72EFAF0B9BDF81250012D84
:10246000C6D1012E1ED01AF8013C1E4214BF012312
:102470000023802E0AF1FF3A8DF811300ED076003D
:10248000F6B20DF1110BB7E719462A4648460193FB
:1024900005F084FF019BBDE703464DE72E460DF195
:1024A000110BA9E79AF8003003F001038DF8113001
:1024B000E5E7012803463FF43FAFBDF81420D204FE
:1024C0007FF53AAF01902A460249079805F066FF6A
:1024D000019B31E7D035FF1F70B582B0054601A8DA
:1024E0000E46FFF7FDFA38B100210846FEF7D6FB8D
:1024F0000225284602B070BD019BAA889A800A2254
:1025000004465A809868AA799A7106304FF40041BF
:10251000FFF742FC019B9A68072111729A68947236
:10252000986821460A30FFF737FC019B98683146CE
:102530000C30FFF735FC03210198FFF7E9FA054657
:1025400048B1019B204621461C70FEF7A7FB0225DF
:10255000284602B070BD01460820FEF79FFB2846C2
:1025600002B070BD2DE9F041904D2B8982B05BB96E
:10257000044680680C30FFF70BFC0528688167D89B
:10258000A288A379AA81EB8101A8FFF7A9FA0446E2
:1025900040B100210846FEF781FB0224204602B02C
:1025A000BDE8F081019BA9899868EA899980062194
:1025B00059809A7108444FF40041FFF7EDFB019AEE
:1025C0002B8991684FF0020881F8088091688C721D
:1025D000976807F10C06002B48D0013B2B816B89D3
:1025E00023B1E98A0020FEF79BF8E0B9019B298915
:1025F0005A88986814445C800A30FFF7CDFB2B8919
:102600000198EBB92B760321FFF782FA044640B319
:10261000019B002108461970FEF740FB022420466A
:1026200002B0BDE8F08101463046FFF7B5FB023449
:102630002B69A4B2B4EB430F06F10206D1D1D5E762
:102640008268137A012163F07F0313722976DAE737
:1026500020465749FFF740FF0446204602B0BDE838
:10266000F08129890620FEF719FB97E7012001F088
:102670002BF80C38430869892B613046FFF78CFB37
:102680006C8907F10E0634B3012C64D0022C0ED0F5
:10269000032C6BD0042C72D0052C7BD0A88A444626
:1026A0002B69421C9A420AD800232B8197E74021CC
:1026B0000120FEF735F84023A882EB82F0E7C3F152
:1026C00001021044B0FBF3F203FB120392B203B118
:1026D00001322A8183E705234FF6FF710120AB8287
:1026E000FEF71EF8034601463046AB82FFF754FB67
:1026F00040210120FEF714F80346014607F11000BF
:10270000AB82FFF749FB80210120FEF709F8034661
:10271000014607F11200AB82FFF73EFB4FF48071D8
:102720000120FDF7FDFF0346014607F11400AB82CF
:10273000FFF732FB4FF400710120FDF7F1FF034674
:10274000014607F11600AB8207F11806FFF724FBDC
:102750000C24A88AA4E720464FF6FF71FDF7E0FF9E
:102760004FF6FF734446A882EB8299E7802101204F
:10277000FDF7D6FF80234446A882EB8290E74FF412
:1027800080710120FDF7CCFF4FF480734446A8828E
:10279000EB8285E74FF400710120FDF7C1FF4FF494
:1027A00000734446A882EB827AE700BFD035FF1F52
:1027B000430004062DE9F0415D4C638B82B03BBBC6
:1027C000054680680C30FFF7E3FA0DF101036A4615
:1027D0000DF10201A083FEF759F838B904F11E0289
:1027E00004F12001A08BFDF751FF40B1284651496B
:1027F000FFF772FE0546284602B0BDE8F081AA88C0
:10280000AB79A2840120E38400F05EFF0C38A06263
:1028100001A8FFF765F9054640B100210846FEF71B
:102820003DFA0225284602B0BDE8F081019BA18C4B
:102830009868E28C9980062159809A7108444FF477
:102840000041FFF7A9FA019B668B9A680421117277
:102850009A6895729F6807F10C00002E3BD0013EEC
:10286000B6B26683A846A26AE38B216A551B9D42D5
:1028700028BF1D462A4605F091FD019F226A7B88EC
:10288000B8681FFA85FE43441544E28B2562734401
:102890007B800A30A2EB0E033146E383FFF77CFA1C
:1028A000638B0198002B39D08268137A022163F080
:1028B0007F03137221760321FFF72AF9054678B3C7
:1028C000019B002108461970FEF7E8F90225284609
:1028D00002B0BDE8F081E38BA26A991D914208D94C
:1028E0009B1A0633B3FBF2F102FB113389B2E3B951
:1028F0006183A18BFFF750FA07F10E00BDF80210BB
:10290000FFF74AFA06259DF801209DF800303A7439
:102910007B7407F11200A846668BA4E72376CAE70A
:10292000618B0620FEF7BAF97CE70131E0E700BFD2
:10293000D035FF1F000002062DE9F041B04DAC8DEF
:1029400086B0002C41D1064680680C30FFF720FA93
:10295000B368E885997BDF7B85F8301005F1320399
:102960000DF1060285F83170FDF7A4FFC0B1A5494D
:10297000234640F2031205E00133172B00F00181DA
:1029800031F833209042F7D19E4A02EBC3035968D5
:102990003046FFF7A1FD0446204606B0BDE8F081B1
:1029A0006B8EB188B279A98613F4805F95F83130C7
:1029B000EA8608BF03F08F0323F06003012085F847
:1029C000313000F081FE0C38A86302A8FFF788F8C8
:1029D000044640B100210846FEF760F90224204673
:1029E00006B0BDE8F081029BA98E9868EA8E9980B6
:1029F00006269A715E8030444FF40041FFF7CCF90F
:102A0000029AAB8D91680E7291688C72976807F18B
:102A10000C06002B46D0013BAB8595F831301907E9
:102A200004D5AA6B271D974240F2CC80DA0629D440
:102A3000002B00F0AE80029BA98D5A889868144440
:102A40005C800A30FFF7A8F9AB8D0298002B00F0EC
:102A500096808268137A032163F07F0313722976CC
:102A60000321FFF755F80446002800F08D80029BF3
:102A7000002108461970FEF711F90224204606B01D
:102A8000BDE8F08103AB05AA95F83010E88DFDF79D
:102A90007FFD039AAB6BA118994240F2B78095F87D
:102AA0003130C5E73046E98DFFF776F995F83020EB
:102AB00095F83130BA7307F11000FB73BDF80610BA
:102AC000FFF76AF9BDF80600012807F1120875D072
:102AD000FDF774FC04460490002840F0AA8005AE7F
:102AE000324604AB95F83010E88DFDF7D1F9002897
:102AF00040F0A280BDF810104046FFF74DF9698EF6
:102B000007F11400C1F30901FFF746F9002432462A
:102B100003AB95F83010E88DAC87FDF7B9F995F85F
:102B200031301A0707F1160602D5AA8F0432AA8798
:102B3000DF0603D5A98F039A0A44AA879C0603D50A
:102B4000A98F039A0A44AA87580603D5AA8F039B24
:102B50001344AB872C4B95F83010E88D9A1CFDF789
:102B6000ADFDAB8FE98FAA6B0B449BB203F10A0159
:102B70009142AB8736D80023AB850A244DE72B76EC
:102B80006EE74FF0006103E7A98D0620FEF786F897
:102B900025E7AB6BEA8F296C1F1B974228BF1746AE
:102BA0003A46304605F0FAFBAA8F2B6CB9B20C44BA
:102BB000521A1F44A4B2AA872F643CE7049001462E
:102BC00005AE99E730460021FFF7EAF8AA8F95F89D
:102BD0003130043A03F0F703BCB20436AA8785F813
:102BE000313023E7C2F10A011944B1FBF2F302FBD1
:102BF00013129BB202B10133AB850A240DE700BF6B
:102C0000D035FF1F709401000E36FF1F0599304626
:102C100005F0C4FB0399AA8F95F8313088B20444BB
:102C2000121A03F0EF030E44A4B2AA8785F83130DC
:102C3000FEE681B205AE5FE7049421465CE700BF83
:102C400010B50C4C237E012B09D0022B0DD0032B89
:102C500000D010BD0020BDE81040FFF76DBE002081
:102C6000FFF780FC237E022BF1D10020FFF7A2FDAD
:102C7000237EECE7D035FF1F2DE9F04182B00446FA
:102C800001A8884617461E46FEF72AFF40B10021DC
:102C90000846FEF703F80224204602B0BDE8F081A2
:102CA000019BA2889A800A225A8005469868A279D8
:102CB0009A7106304FF40051FFF76EF8019B9A6845
:102CC00080211172986841460930FFF765F8019B31
:102CD0009A68D772986831460C30FFF761F8032183
:102CE0000198FEF715FF044650B1019B284629467E
:102CF0001D70FDF7D3FF0224204602B0BDE8F0812D
:102D000001460820FDF7CAFF204602B0BDE8F08169
:102D10002DE9F0430446806885B009308846FFF706
:102D200037F8A3681A7ADD7A12F01007064602D047
:102D3000012D4DD80127B8F1010F30D003F10C005F
:102D4000B4F80290FFF726F8A36802461033B8F1F2
:102D5000000F05D1A9F10A0E1FFA8EFE704543D867
:102D6000009231462A463846FFF794FA20B3444988
:102D700040F20312002304E00133172B31D031F865
:102D800033208242F8D13E4A02EBC3035B682A46F5
:102D900031462046FFF770FF05B0BDE8F083C2F36F
:102DA0008102C2F1040200920C332A4631463846B1
:102DB000FFF770FA0028DAD103A8FEF791FE50B3AE
:102DC00000210846FDF76AFF022005B0BDE8F08348
:102DD00001462A4620462B4BFFF74EFF05B0BDE8C3
:102DE000F0834FF00063D2E7DFF89CC01946CCF8BF
:102DF00048200CF155007246ACF844608CF84650FF
:102E0000CCF84CE08CF8547005F0C8FA03A8FEF733
:102E100067FE0028D4D1039BA2889A800A225A8098
:102E20009868A2799A714FF440510630FEF7B4FFCA
:102E3000039B9A6860211172E7B99868314609309E
:102E4000FEF7AAFF03988368DD7283680024DC60C4
:102E50000321FEF75DFE38B1039B204621461C701E
:102E6000FDF71CFF022097E701200021FDF716FF68
:102E7000002091E799680A7A42F010020A72DCE7B2
:102E80007094010043000406D035FF1F2DE9F04F78
:102E900091B0164603939DF8703004939DF87430FA
:102EA0000790DDF8688000930D46002940F04F81BF
:102EB0009DF80C308DF82B304FF0000ACDF868806B
:102EC000039C0DF138090DF1340BD0460CE00028BD
:102ED00040F02581BAF1010F40F21E8101349DF8C6
:102EE0002B30E4B2A34228D34B465A462146304603
:102EF000FCF7CEFF012D0746E9D140F21523984299
:102F0000ECD0002840F00B810CAB0DF12E022146D5
:102F10003046FDF7CFFCBDF82E30012B00F00A81C2
:102F2000BA460E9B9844002CD8D101349DF82B3022
:102F3000E4B2A34208F10108D6D201204446CDF8FC
:102F40002080DDF8688000F0BFFB042C834640F24F
:102F50001581103883B209930FA800230693FEF75A
:102F6000BFFD0590002840F01781049B052B00F061
:102F70002381089B042B0F9B9A6800F27E8102F14B
:102F80000C0A9DF82B2003998A4238BF00277AD378
:102F90000DF1340B0023CDF804B0039CDDF824B010
:102FA00002931F460DF138094B46019A21463046DF
:102FB000FCF76EFF012D00F0F980002840F06081E1
:102FC000B8F1000F06D00D9A0E9B4244A3EB080304
:102FD0000D920E93FEF7C2F8214602463046FDF7E9
:102FE00007FA4207ADF8300040F0EB80002D00F00A
:102FF000A181009B012B00F0F5804FF001080DF13D
:1030000032030DF12E0221463046FDF753FC002815
:1030100040F03681BDF82E30012B00F00C810D9967
:103020000E9A0290BB185B4511D9AD4BA3F84460D2
:1030300083F8464083F85450049BABEB0702052B02
:103040000E92A74B00F0F0801A6500230693B8F1AA
:10305000000F40F0C280504605F0A0F90E9B1F44BF
:10306000BFB29A4425B11CB901370AF8014BBFB26F
:10307000BB4507D04FF0000801349DF82B30E4B277
:10308000A34291D20F9B079998688A889A800A2256
:103090005A808A799A7106304FF44051FEF77CFECF
:1030A000049B052B00F022810F9B9A68402111722E
:1030B00099680A7A012D42F001020A7200F03E81FD
:1030C000069A002A00F0E98099680A7A42F0020222
:1030D0000A72089A9968C2F10402087A920002F012
:1030E0000C0202430A72986831460930FEF754FE1A
:1030F0000F989DF80C2083680321DA72FEF708FD13
:10310000002800F0E9800F9B002119700846FDF7A8
:10311000C5FD0223059309E00E9B9844DEE6224696
:10312000314607986F4BFFF7A7FD0590059811B042
:10313000BDE8F08FBAF1080F00F09D800AF1010A96
:103140005FFA8AFABAF1010F7FF6EBAEEBE60DF10A
:103150002B030BAA0DF12E013046FDF797FB03461A
:10316000002840F098809DF82B2003998A42BFF4F4
:10317000A3AE0120089300F0A7FA8346ABF10C0B35
:103180001FFA8BF309930FA801230693FEF7A8FCFF
:10319000059000283FF4E9AE00210846FDF77EFDCA
:1031A00002230593059811B0BDE8F08F40F2152376
:1031B00098427FF402AF5FE70F9B9A6802F1090A19
:1031C000DFE6009B012B00F0D480002D40F0CE8084
:1031D0000D990E9A0295A84624E70021504605F065
:1031E000E8F83BE722463146284603F023FD002855
:1031F0003FF403AF0F9A3C490023137040F20312CF
:1032000005E00133172B00F0AE8031F83320824205
:10321000F7D1354A02EBC3035B6807982246314673
:10322000FFF72AFD059081E71B6D2D4813440365C8
:10323000002306930BE70D9A02981278003218BF0C
:10324000012210F0F70F8DF82D20014611D01AF849
:10325000013C824001311A43013FCBB2BFB202931D
:103260008DF82D200AF1FF3A01220E920DF12D0169
:10327000D8E60293F8E7AA4653E602F1100A80E680
:103280000F9D0798174B0027224631462F70FFF7F6
:10329000F3FC05904AE7039A42E75A889868089930
:1032A0003A445A800C30FEF77BFD0F9B98683146FC
:1032B0000930FEF771FD0F989DF80C2083680321FB
:1032C000DA72FEF725FC00287FF41DAF089B04206E
:1032D000D91BFDF7E3FC29E701460320F9E700BF0E
:1032E000D035FF1F11000906709401000F98836804
:1032F00000221A72079B9B681B7ADB0604D5826842
:10330000137A43F0100313721B9B9F4225D0072FA3
:103310001AD94388073B3B4443800321FEF7F8FB5F
:10332000059000287FF4EFAE1B9B0520D91BFDF70D
:10333000B5FCFBE60F9A134B15706EE799680A7A95
:1033400042F010020A72BBE68268FB1F117A5B0032
:1033500003F00E030B431372DFE78268137A43F026
:1033600001031372D3E74FF0006356E74FF00008F4
:1033700045E622463146284603F05CFC00283FF42F
:1033800024AF37E70100010630B585B0084C019144
:1033900094F84630B4F8442094F85410246D009406
:1033A0000025052403950294FFF770FD05B030BD9C
:1033B000D035FF1FF0B50546806885B00930FEF7AF
:1033C000E7FCAB681C7ADB7A14F0100418D0012BF0
:1033D0000DD8012100240127042602460397284620
:1033E000029601940094FFF751FD05B0F0BD1A4616
:1033F000044B0146284605B0BDE8F040FFF73CBC51
:103400002146E7E74300040670B544880A2C84B0DF
:1034100006465AD0033CA4B2494DE86C23180A2B47
:1034200043D8B168284422465530093104F0B6FF2C
:10343000EB6CB2681C44EC64137ADA070CD403A872
:10344000FEF74EFB002845D000210846FDF726FC7C
:103450000224204604B070BDAB6C95F84620B5F848
:10346000441095F85400009305F15503FEF712FF40
:103470000028E4D0B5F8441095F84620314D40F2CC
:103480000314002304E00133172B51D035F83340E7
:10349000A042F8D12B4800EBC3035B683046FFF72E
:1034A000EBFB0446204604B070BD00210846FDF742
:1034B000F5FB3046244B95F84620B5F84410FFF74D
:1034C000DBFB0446204604B070BD83681C7AC4F35D
:1034D0004204A1E7039BB2889A800A225A80986826
:1034E000B2799A7106304FF44051FEF755FC0398BB
:1034F000836820221A72B3681B7ADB0604D58268BF
:10350000137A43F01003137283680025C3F809503F
:103510000321DD60FEF7FCFA044660B1039B2846F8
:1035200029461D70FDF7BAFB0224204604B070BD89
:103530004FF00063B2E701460220FDF7AFFB88E7DA
:10354000D035FF1F709401000500040500B583B05D
:10355000014601220DF1070000F04EFB9DF8070027
:1035600003B05DF804FB00BF00B583B00146022242
:103570000DF1060000F040FBBDF8060003B05DF859
:1035800004FB00BF00B5042283B001460DEB02002E
:1035900000F032FB019803B05DF804FB00B583B086
:1035A00002AB012203F8011D194600F05FFB03B0D6
:1035B0005DF804FB00B583B002AB022223F8021DC4
:1035C000194600F053FB03B05DF804FB00B583B06F
:1035D00002AB042243F8041D194600F047FB03B078
:1035E0005DF804FB00F042BB00F006BBF8B5052017
:1035F000FFF7ACFF184E0428307029D9042333702C
:10360000164F002403E00134E4B29C421FD204F5BB
:103610008075ED00E81D0121FFF7C0FF3378A3425C
:10362000F1D92846FFF7A0FF337804EB4402A34208
:1036300027F8120005F1020007EB4205E3D9FFF776
:1036400093FF013433786880E4B29C42DFD3F8BD45
:103650000028D5D1FBE700BF3036FF1F1086FF1FC3
:10366000054B1B78834200D87047C00000F6070066
:103670000021FFF793BF00BF3036FF1F054B1B78BB
:10368000834200D87047C00000F607000121FFF711
:1036900085BF00BF3036FF1F094B1B78834201D81E
:1036A0000020704710B5044600F58070C000FFF799
:1036B0005BFF04EB4404034B23F8140010BD00BF70
:1036C0003036FF1F1086FF1F094B1B78834201D83D
:1036D0000020704710B50446C00000F60200FFF756
:1036E00043FF044B04EB440403EB4404608010BD2F
:1036F0003036FF1F1086FF1FF8B500F58076F60004
:1037000005463046FFF730FF0746B01CFFF72CFF99
:103710000446301DFFF71AFF830708BF04EB44047B
:10372000064B07F1FF3008BFA4B205EB4505044482
:1037300003EB4505A0B2A880F8BD00BF1086FF1FAF
:103740002DE9F0411A4F3B785BB31A4D00EB40086E
:10375000064605EB48080024E00000F60600FFF7E7
:10376000F5FEA64204F1010217D06300191910F00A
:10377000010F05EB410010D035F81130B8F80010FA
:103780009942044602D3808888420DD2B8F80410CA
:103790008B4202D8A3888B4206D23B78D4B2A34294
:1037A000DAD80020BDE8F0810220BDE8F08100BF3A
:1037B0003036FF1F1086FF1F70B5044682B0FDF73C
:1037C000CDFC022C23D0032C1ED1234B9A78022A45
:1037D00004BF01225A70082836D0042834D01F4B69
:1037E0001F4D1C686B8A1C4401231A4620460DF1AC
:1037F0000701FFF7F7FEA88A0123013820440DF1E5
:1038000007011A46FFF7EEFE002002B070BD124B12
:10381000012408285C701CD0114E104B1D68B38920
:103820001D4429460DF1070023462246FFF7DCFE22
:10383000F18901390DF10700294423462246FFF79B
:10384000D3FE002002B070BDFEF7BCFC002002B029
:1038500070BDFEF767FCD7E73036FF1F0C86FF1FF1
:103860001086FF1F0320FFF7A7BF00BF70B50C4CE9
:103870006368012B06D063780BB1012363600023DA
:10388000637070BD6678002EF7D1054603F010FA1C
:103890000220FDF7A5FC284600F002F96660EAE781
:1038A0003036FF1F38B540F6060440F68605204640
:1038B0000834FFF74BFEAC42F9D138BD10B540F6E5
:1038C0000E00FFF743FE10F001030FD0094C237ADE
:1038D00000F0020083420BD02072FEF729F9217A12
:1038E00040F60F00BDE81040FFF758BE014A1372C2
:1038F00010BD00BF3036FF1F014B9870704700BFEE
:103900003036FF1F014B9878704700BF3036FF1FDD
:1039100030B42B4D2C6844B1844203D148E0984226
:1039200013D01C462368002BF9D122F02003037327
:1039300012F0200308BF4381224B41601B88B1EB8A
:10394000C33F0BD9022030BC70470368236090F955
:103950000C30002BA4BF00234381E6E744890C44CC
:10396000A34221D2B4FBF3F103FB114389B243819B
:1039700001811BB113065CBF013189B22B792A6822
:10398000194489B20181B2B113898B4204D912E082
:103990001C89A14203D31A461368002BF8D1036097
:1039A00030BC106000207047002343810121E5E70F
:1039B00003682B60CBE7026028600020C3E700BFEC
:1039C0003C36FF1F6015FF1F70B5324E34683379E7
:1039D000002C5DD0DBB2228999B2914255D3307967
:1039E000C31ADBB233712546002000E02A898A42DF
:1039F0002ABF521A28812A812D68002DF6D12389E9
:103A0000EBB9207B20F08003012B2AD0022B03D1BD
:103A10002046FFF72BFF207B316849B3A14231D00C
:103A20000A4602E0A3420BD01A461368002BF9D1D4
:103A300010F0C00F0CD10C462389002BE1D070BDD3
:103A400023681360030658BF658110F0C00F04D0CF
:103A5000616800F0BF00207371B93468002CCED1CA
:103A600070BD2046FDF748FA3168207B0029D5D18A
:103A700010F0C00FECD170BD40F020022046FFF7DF
:103A800047FFEAE723683360DCE7092BA7D870BD5E
:103A9000347170BD3C36FF1F01B139E7012070471A
:103AA0000C4B1A684AB1824203D110E0984205D00B
:103AB0001A461368002BF9D17047704703681360EA
:103AC00090F90C30002BF8DB00234381704702682B
:103AD0001A60F5E73C36FF1F70B5104E336813B916
:103AE00011E01B687BB19842FBD10D460C4903895C
:103AF000098803FB01F1044659B901203279656058
:103B00009B1A238170BD09B9012070BDBDE87040CA
:103B1000FEE62046FFF7FCFE2389EFE73C36FF1F59
:103B20006015FF1F074B1B683BB1834202D106E0C3
:103B3000984204D01B68002BFAD118467047012028
:103B4000704700BF3C36FF1F034A13790133DBB2D5
:103B500001211371517170473C36FF1F70B5054646
:103B60000E46F5F783FAC5F3471343F000431F4AA7
:103B700043F480335363D36A002BFCDA936BD16A2E
:103B80001B4B1A4CE80000F0F80041F010410343D1
:103B9000D1625363E36A002BFCDA2B0A23F01F0384
:103BA00043EA8603A26BE16A104ADBB243F00043AA
:103BB00043F4803341F01041E1626363D36A002B28
:103BC000FCDA936BD36A032E43F01043D36200D028
:103BD00070BD084B05495363CB6A002BFCDA8B6B35
:103BE000CB6A43F01043CB6270BD00BF00D00240EF
:103BF00006000180FF00018070B50E4605461446A0
:103C000000F01CF9B0B20321FFF7A8FF0CB3144970
:103C1000144A012C0DD04A63CB6A002BFCDA8B6B63
:103C200005F8013BCB6A013C43F01043A4B2CB62E0
:103C3000EFE70B4B0C4A5A63DA6A002AFCDA084BAE
:103C4000DA6AD200FCD59A6B2A70DA6A42F0104226
:103C5000DA62F5F703FABDE8704000F0DFB800BFA4
:103C600000D0024000000180FF00010870B5064648
:103C70000D46144600F0E2F8B0B20421FFF76EFFE3
:103C800034B3164A16482946012C0ED00B7813433C
:103C900043630131C36A002BFCDA836BC36A013CC6
:103CA00043F01043A4B2C362EEE70B780C4A43F032
:103CB000006343F480335363D36A002BFCDA084B70
:103CC000DA6AD200FCD59A6BDA6A42F01042DA6204
:103CD000F5F7C4F9BDE8704000F0A0B8000001801D
:103CE00000D00240F8B5154B154C164E00275B204E
:103CF0001F70F4F7C3FB03CC134B144AB4F800C095
:103D0000402583F85B537160306003CA104D114B3E
:103D10002860696003CB1C880F4BB2F800E00F4AA3
:103D2000A5F808E01C810E4D18606FF00044A6F85D
:103D300008C0596038469564D464F8BD4236FF1F08
:103D40001CA80100B801FF1F00E100E028A8010045
:103D5000AC01FF1F34A80100A001FF1F4000FF1F9E
:103D600001000080014B0020186070470C86FF1F87
:103D700008B54FF4A070FFF7F7FBC0B208BD00BF55
:103D800008B54FF4A070FFF7EFFBC0B2A0F105003B
:103D9000B0FA80F0400908BD1E4B6846D3F8A02059
:103DA00020F007018D46D10131B51DD4194BD3F850
:103DB000A020920114D55A6E174C012142F0807256
:103DC0000D4608465A66F4F7F9FF2570FBF7BCFF6D
:103DD000FDF7C8FC0023284619462370F4F7EEFFD0
:103DE000BDE83140854670471A6E0B4C012142F008
:103DF00080720D461A660846F4F7E0FF2570FBF75F
:103E0000ABFFFDF789FC0023284619462370F4F721
:103E1000D5FFCBE700D004404236FF1F08B5054B65
:103E20001B7833B95B20F4F729FB034B402283F85E
:103E30005B2308BD4236FF1F00E100E0034B1B7807
:103E400003B170475B20F4F763BB00BF4236FF1F2E
:103E500010B5002003F04CF8002000F0CDFB00F07E
:103E60005FFC012000F0BAFA012000F085FB012080
:103E700000F030FF002000F0B1FA002001F0AAFCB1
:103E8000002000F079FB002001F0B0F80E4C00207B
:103E900000F020FF0D4B626E1A6000F0D3FF00208F
:103EA00001F00AFD638803F06F033BB9002001F0C5
:103EB0001DFB638803F06F03002BF7D002F0B4FF03
:103EC000BDE8104000F03CBC4000FF1F8486FF1F8F
:103ED00030B583B0FDF78AFC012000F04BF802F00A
:103EE0000FFF02F097FF38B9002000F043F80020E0
:103EF00001F0FCFA03B030BD164C00F079FFFFF77B
:103F0000B1FC2378002BEFD002AD134B45F8043DF4
:103F100003212A46042341F63340FCF7C9FA2A4616
:103F20000423062141F63340FCF7C2FA2A46042353
:103F3000092141F63340FCF7BBFA02AA002522F81A
:103F4000065D0223082141F63340FCF7B1FA2570E3
:103F5000CAE700BF9286FF1FA0860100044B588865
:103F600000F06F00A0F10800B0FA80F0400970473F
:103F70004000FF1F2DE9F047CD4EC700F319D3E9EC
:103F8000002352EA030182B024D0840006EB040827
:103F9000D8F8BC50E90700F1888015F0020100F064
:103FA0008F8030B1C349D1E9002342F00072C1E9EA
:103FB000002396F8B8E096F8B930344425F00205AD
:103FC0007345C4F8BC504FF0000939D1484602B0DF
:103FD000BDE8F087B74DB8493D443944D5E90045BF
:103FE000D1E900894D4508BF444521D0002188EA28
:103FF000040889EA05094FF03F0E4FF0010CAEF1BD
:104000002005CEF120040CFA05F32CFA04F4234326
:104010000CFA0EF208EA020409EA030501310EF176
:10402000FF3E2C43C9B25FFA8EFE2CD14029E6D167
:1040300096F8B8E096F8B9304FF001097345C5D04D
:104040009E4906EBCE0301EBCE010231188AFCF744
:10405000A3FF04460028B9D102AA014602F8010DC7
:10406000012341F20100FCF723FA96F8B830142B33
:1040700018BF013348460CBF86F8B84086F8B83000
:1040800002B0BDE8F0878E4C4FF0000E2146D1E91A
:1040900000894B4508BF424501F120015FD00EF178
:1040A000010EBEF1150FF2D1C2E725F00105C8F8E7
:1040B000BC5096F8B8E096F8B9304FF00009BDE76B
:1040C00015F0040979D115F0080A40F0978015F031
:1040D000200964D115F0400140F09F8015F0800F59
:1040E00040F0BE8015F4807940F02381A90500F1ED
:1040F000FC80680500F1118115F4006971D115F497
:10410000805140F09D8015F4005940F0DF80690433
:1041100000F1F48015F4004100F03F81002003F02D
:1041200040010143634D07D005EB070EDEE90001B6
:1041300020F01000CEE900013D44D5E90089344467
:1041400029EA0309374428EA020800200021002355
:10415000C5E90089C7E90001C4F8BC3068E74FEA47
:10416000400806EB080504EB4E11840006EB040C36
:10417000B5F8C450D1F80CE0CCF8C8106906CCF8FA
:10418000BCE003D52EF06C0ECCF8BCE0B044F119C5
:1041900045EA0E05C1E90023A8F8C450F6E600F090
:1041A000B5F9D8F8BC2096F8B8E096F8B93022F006
:1041B0002002D146C8F8BC2040E7424C96F8B8E04F
:1041C00096F8B930942202FB004025F0040542889D
:1041D000C8F8BC5022F06F0242F00F0289464280BC
:1041E0002CE7384B5B8803F06F03082B42D096F81E
:1041F000B8E096F8B9304FF000091FE7314B94242E
:1042000004FB00340121626E00F04AFA012840D01C
:1042100096F8B8E096F8B93010E72A4996F8B8E071
:1042200096F8B930942202FB001025F04005428830
:10423000C8F8BC5022F06F0242F008024280FDE64E
:10424000204B5B8803F06F03082BD0D1344425F456
:104250008055C4F8BC5096F8B8E096F8B930EDE651
:1042600025F08005C8F8BC50894696F8B8E096F865
:10427000B930E3E63444144A96F8B8E096F8B93019
:1042800025F400654FF00009C4F8BC5082F8009096
:10429000D4E66188D8F8BC2096F8B8E096F8B93032
:1042A00041F4806122F008026180C8F8BC20C5E6B4
:1042B0004836FF1F3086FF1F4086FF1F5836FF1FFE
:1042C0006815FF1F4000FF1F2886FF1F414B5B88BA
:1042D00003F06F03082B8AD10120894602F018FEF3
:1042E00096F8B8E096F8B930A8E625F40075C8F855
:1042F000BC5096F8B8E096F8B9309FE6364BD3E953
:104300000023002302F0007213433FF470AF3444E3
:1043100025F48045C4F8BC507AE7344425F4806520
:10432000C4F8BC5096F8B8E096F8B9304FF00009E0
:1043300084E696F8B93096F8B8E05F1C774524D04B
:10434000B6F8B820B2F5A05F1FD03119DA00D1F865
:10435000C8C0B118BCF80880A1F8108001289CF8EA
:104360000AC081F812C0324408BFFF20142BC87461
:1043700018BFFBB24FF0000111755175917506BF62
:1043800086F8B9100B4686F8B930344425F48075A8
:10439000C4F8BC504FF0000950E6E8037FF527AFA2
:1043A0000D4D96F8B8E03D44D5E90089344443EA20
:1043B000090342EA0802C5E900233744002300222A
:1043C000C7E90023C4F8BC1096F8B9304FF00109D2
:1043D00034E600BF4000FF1F4086FF1FF0B40F4BC4
:1043E0000F4E1049104FC2000024002516441144FE
:1043F0001A44C2E90045C1E900450022C6E900456A
:1044000003EB400403EB800308493A70A4F8C4208E
:10441000C3F8BC20C3F8C810F0BC70474836FF1F73
:104420003086FF1F4086FF1F2886FF1F6815FF1F6D
:104430002DE97003124E1349134AC3001E44D6E9F6
:1044400000451944D1E9008904F0804405F03C0599
:1044500044F00104C6E9004513440024002502EBA2
:10446000400008F0804809F03C09C3E900450023FA
:10447000C1E90089A0F8C430BDE87003704700BFEF
:104480003086FF1F4086FF1F4836FF1F10B50023F0
:1044900014460A4601460620F9F736FB2060F8F775
:1044A000A5FC642814BF4FF48370002010BD00BF2A
:1044B00008B513680A4601460520F9F725FBF8F709
:1044C00095FC642814BF4FF48370002008BD00BF22
:1044D00038B5024604460D46002303210620F9F7AD
:1044E00013FB084B942202FB0434E16A6B1A9842D6
:1044F00005DB29448842CCBF0020012038BD0020C4
:1045000038BD00BF4000FF1F00F0D0BF10B504460B
:1045100002F0EEFC064800EB0410FFF7C1FA054A72
:1045200032F8143023F0010322F81430012010BDBA
:104530005486FF1F5086FF1F70B50D4E345C054634
:104540004CB10C4A32F8100010F0010002D00022E9
:104550007255012070BD02F0C9FC064A012132F8F3
:10456000153071550B43204622F8153070BD00BF41
:104570001837FF1F5086FF1F012803D0024B00226F
:1045800023F81020704700BF5086FF1F2DE9F0412F
:10459000164E174D56F82060044617469846B04709
:1045A00055F82430394606462046984755F82420C9
:1045B00007464146204690473B46054622460B218A
:1045C0000520F9F7A1FA2B4622460B210520F9F721
:1045D0009BFA15B1074B43F824503346224600217D
:1045E0000120F9F791FA0020BDE8F0816486FF1FF1
:1045F0007086FF1F8486FF1F002302461946032092
:10460000F9F782BA2DE9F8431A4E1B4D56F820806F
:104610009DF82060044617469946C04755F8243057
:10462000394680462046984755F824200746494693
:104630002046904743460546224604210520F9F7C7
:1046400063FA3B4622460B210520F9F75DFA2B461B
:1046500022460B210520F9F757FA15B1074B43F80D
:10466000245022463146099B0420F9F74DFA0020D8
:10467000BDE8F8836486FF1F7086FF1F8486FF1FD6
:1046800038B502460C4605460B4605200B21F9F7C6
:104690003BFA14B1014B43F8254038BD8486FF1F17
:1046A000F8B51A4D2B1804461B798B4215D0184BC0
:1046B0000E4653F8203011469847224607460346D7
:1046C0000B210520F9F720FACFB90023194622461D
:1046D0000320F9F719FA2B191E7100232246032132
:1046E0000620F9F711FA0B4B014653F82430204607
:1046F0009847034638B92C4401202371F8BD064B76
:1047000043F82470E1E70020F8BD00BF1837FF1F11
:104710007086FF1F6C86FF1F8486FF1F00F068BB3A
:10472000064B10B441F2F2720124042000219C6077
:10473000D86019615A609A6110BC70478801FF1FE8
:10474000014B024A1A6070472023FF1F010004003A
:104750002DE9F04784B004AB002502AC43F8045DBA
:104760002246032141F218000295FBF77BFE002848
:1047700038D1029AADF80620120CADF804204FF0A3
:104780000009DFF86CE0194F4E460DF1040C4FF0B4
:104790002E08052542F21070B2FBF0F3A7FB00A132
:1047A00000FB13229BB292B2C80813B9B9F1000FF3
:1047B00006D03033711C0EF806304FF00109CEB22E
:1047C000013DE9D12CF8022BA4450EF8068004D057
:1047D0000136F6B2BCF80020DBE70EF8065004B054
:1047E000BDE8F087BDF80420C9E700BFCDCCCCCC34
:1047F000A001FF1F0149002000F0FAB80818FF1FB0
:10480000A0F50053B3F5E06F10B40AD3A0F5C04390
:10481000B3F5006F14D24FF4006422464FF4C04346
:1048200004E04FF4007422464FF40053C31A93FB84
:10483000F4F3DBB203FB1200088010BC184670478B
:104840000123088010BC1846704700BF0B4610B506
:1048500011460446184600F071FA28B10146204678
:104860004B69BDE81040184710BD00BF10B50446A5
:1048700000F016FE044A942303FB042398612046AB
:1048800000F0D2FB002010BD4000FF1F38B50446E9
:104890000D4600F0DDFD2946204600F01BFD2046B8
:1048A00000F00AFD002038BD10B502460446497AE2
:1048B00000230620F9F728F9034BB42202FB043445
:1048C0006060002010BD00BFD400FF1F00207047B3
:1048D000F0B50A88B1F9044083B004FB002402ABB0
:1048E0000026A4B20D460746897843F8046D204699
:1048F0006A460096FBF7B6FD08B103B0F0BD03466B
:104900003A46697A0620F9F7FFF8AB79012B0AD00D
:10491000022B10D000906A46A978019B2046FBF735
:10492000C7FD03B0F0BD054B53F8273001463846AC
:1049300098470090EFE7024BF6E700BF6C86FF1F39
:104940006886FF1F4FF48870704700BF034A9423A6
:1049500003FB00230020DA6D1A6670474000FF1F3A
:1049600010B502460446002303210620F9F7CCF8CF
:10497000154B014653F8243020469847002818D09C
:104980000BDD124A942303FB042400206388C3F345
:104990000E0343F48043638010BD0C4B942202FB52
:1049A0000434002063886FEA83436FEA9343638093
:1049B00010BD064A942303FB042400206388C3F33C
:1049C0000D03638010BD00BF6C86FF1F4000FF1FFA
:1049D0000B4610B511460446184600F0AFF928B151
:1049E000014620460B69BDE81040184710BD00BFC6
:1049F000064A942303FB002340F215105B8803F062
:104A00006F03402B08BF0020704700BF4000FF1F0E
:104A100000F052BF002070471E4A942303FB00237E
:104A200093F90E1093F90F308B422BD010B5B1B122
:104A300006290CD001290AD0082908D009290ED04E
:104A40000A2904D003290AD04FF4897010BD124CF2
:104A5000B42303FB004393F87430082B0AD094234B
:104A600003FB00235A8802F06F02272A05D0D9736E
:104A7000002010BD40F2151010BD044600F00EFFDE
:104A800010B110BD002070472046BDE8104000F076
:104A9000BBBE00BF4000FF1FD400FF1F4FF4887053
:104AA000704700BF4FF48870704700BF054A9423D9
:104AB00003FB0020B0F90430042B0CBF4FF48470CA
:104AC000002070474000FF1F0A4A0B4B12689A42B1
:104AD00002D04FF48470704710B500240023E1B277
:104AE0001A4607200134F9F70FF8B4F5807FF5D1A5
:104AF000002010BD2423FF1F73617665024B012245
:104B00001A600020704700BF2423FF1FF0B5B1F9E1
:104B100004500F8883B002AB4FF0000E064605FB31
:104B200000700C4643F804ED8978CDF800E0174694
:104B300080B26A46FBF7ACF9054670B9E379023BEF
:104B4000052B2BD8DFE803F022260C1C1F0C144B7E
:104B5000304653F8263098473860284603B0F0BDF9
:104B6000009B1968A379012BF1D0022B18BF396083
:104B7000F3D10C4B304653F8263098473860ECE7B9
:104B8000009B1978EEE7009B1988EBE7009B93F9EF
:104B90000010E7E7009BB3F90010E3E70021E1E72D
:104BA0006486FF1F7086FF1F70B5114C942303FBB2
:104BB000004382B05B8803F06F03402B18BF40F2C4
:104BC000151502D0284602B070BD02AA002342F893
:104BD000043D0E460446FFF799FF05460028F1D133
:104BE0002246717A019B0520F8F78EFFEAE700BFA5
:104BF0004000FF1F70B582B002AA002342F8043DB6
:104C000006460D46FFF782FF044628B93246697A08
:104C1000019B0520F8F778FF204602B070BD00BF69
:104C200070B582B002AA002342F8043D05460E4644
:104C3000FFF76CFF044640B90F4A942303FB05239A
:104C40005A8802F06F02272A02D0204602B070BDB7
:104C500093F90F3023F00203012BF6D1717A019BF7
:104C60002A460520F8F750FF28460199FFF708FD6E
:104C7000204602B070BD00BF4000FF1F30B583B0BA
:104C800002AA002342F8043D0546FFF73FFF044611
:104C900060B9084A942303FB05235B8803F067038C
:104CA000072B03D128460199FFF7EAFC204603B001
:104CB00030BD00BF4000FF1F10B5044600F0F0FB00
:104CC000034B942202FB0434A061002010BD00BFFE
:104CD0004000FF1F70B5184E338853B30546344665
:104CE00005E00BB1E368984734F8183F53B1012D44
:104CF000A38821462846F4D1002BF3D034F8183F7E
:104D0000002BF4D13388012D14BF0426072683B16C
:104D1000094C02E034F8183F63B1237AB342F9D169
:104D200021462846FFF766FF238B18340BB1002875
:104D3000F3D070BD70BD00BF0818FF1F094B10B441
:104D40001A88044602E033F8182F3AB19442184604
:104D5000F9D19A788A42F6D110BC7047104610BC3F
:104D6000704700BF0818FF1F2DE9F04182B002AB69
:104D7000002423F8024D1D4E884619461746FFF7BA
:104D80003FFD96F89920BDF806E06AB3012102E0E4
:104D90008A4216D9E1B24B1EDBB24C1C16F83350D6
:104DA0008542F5D106EBC3035D887545F0D11D79C9
:104DB0004545EDD13B44012200205A7102B0BDE8C7
:104DC000F081541CE4B206EBC201CB1906F83200A4
:104DD00001220020A1F802E081F8048086F89940C1
:104DE0005A7102B0BDE8F0810124ECE72037FF1FC3
:104DF00038B5124C94F8983014F8335004EBC303D0
:104E000028461A795988FFF721FD94F8983004EB69
:104E1000C30146F264024988914208D094F899206F
:104E20000133934208BF002384F8983038BD044A08
:104E3000942101FB0525AA696A61EFE72037FF1F6E
:104E40004000FF1F2A4900222DE9F0470B4681F858
:104E5000982001F198044A800831A1424FF00000E7
:104E6000F9D1012146F2FD0A46F2620946F26408D0
:104E700046F26B0C46F26C0E46F2740746F2770669
:104E800042F20D05082418701A711A721A731A74F6
:104E90001A751A761A7783F8202083F8242083F86D
:104EA000282083F82C2083F8302083F8342083F8DE
:104EB000382083F83C20A3F802A099719973997562
:104EC000997783F8261083F82E1083F8361083F82C
:104ED0003E10A3F80A90A3F81280A3F81AC0A3F812
:104EE00022E05F855E865D8783F89940BDE8F087A4
:104EF0002037FF1F2DE9F04383B002AB002423F8D5
:104F0000024D0F4619461646FFF77AFC344BBDF8A2
:104F1000069093F899809C466246234608F1010565
:104F200003E0AB4202F108020CD011788142DCB2FE
:104F30009E4603F10103F4D151884945F1D111791D
:104F4000B942EED1444543D04FEACE000CEB00030A
:104F50001E44002272715A79B2BB9B79A3BB9CF8A4
:104F60009870BC4208F1FF3605D2B64503DA013F1E
:104F7000FFB28CF89870631CDAB242451AD25FFA1D
:104F800086F800E00133DBB2D8000CEB00010CEB3B
:104F9000C4024D7955711CF83350B1F802E00CF899
:104FA000345098450D798979A2F802E01C461571B4
:104FB0009171E7D10CEB0003F6B20020BE428CF8F1
:104FC00099605880187108D0002003B0BDE8F083C4
:104FD00040F20B1003B0BDE8F0838CF89800F9E7BD
:104FE0002037FF1F084670470846704770B40849CD
:104FF000084E094D094C0A4A0A4B46F8202045F84C
:10500000202044F8203041F8203070BC704700BFA9
:105010006886FF1F6486FF1F6C86FF1F7086FF1F58
:10502000E54F0100E94F01002DE9F047DFF858E1B5
:10503000942101FB00E191F90F90B9F1060F7ED0A8
:105040004300DFF83CC189691A180CEB8202D2F8E0
:1050500008A051453CDD494EC2001644D6E9004542
:1050600045F00405C6E9004503440CEB830CDCF86D
:1050700004308B4258DCDFF8148108EB0203D3E9DB
:105080000045002605F0080756EA07031DD03C49F5
:105090003C4E00EB400301EB8301942303FB00EE45
:1050A0004B6856F82000DEF81810034499420CDBD8
:1050B000324B1344D3E90001424425F0080521F0A6
:1050C0000801C2E90045C3E900010020BDE8F087FE
:1050D000DFF8B880C20008EB0204D4E900450026DE
:1050E00005F004073E43BFD0264E56F82060AAEBD9
:1050F000060A5145B8DC214B1344D3E9006725F07B
:10510000040508EB020A27F00407B9F1060FCAE903
:105110000045C3E900672CD0430003440CEB830C2B
:10512000DCF804308B42A6DD144B1A44D2E90001AE
:1051300041F00801C2E900010020BDE8F087DFF876
:105140004C80C20008EB0203D3E90045002605F0BD
:10515000040756EA070394D00A4BDFF824C053F83B
:10516000206089690C2303FB00C39B689B1B994249
:10517000C1DD08EB0203D3E9004582E73086FF1F5B
:105180007886FF1F8C86FF1F4000FF1F4086FF1F91
:10519000012930B41FD0022902D0002030BC704752
:1051A000234C24499422B42302FB004203FB001346
:1051B000D26CD3F8B0306FF000418D1A5C42A5423A
:1051C0002DDB1D4900EB400001EB8000D21A82600C
:1051D00030BC00207047164D164C9422B42302FBBD
:1051E000005203FB0043926CD3F8B03001F1004150
:1051F0008D1A5C42A54208DD0F4B00EB400003EB2B
:10520000800030BC4160002070470B4900EB40003B
:1052100001EB8000D21A426030BC00207047064B80
:1052200000EB400003EB800030BC81600020704741
:105230004000FF1FD400FF1F7886FF1F08B5897844
:10524000FFF7A6FF002008BD0B4A08B5942303FB17
:10525000002389789A6CDB6C9A4203DB012905D024
:10526000022906D0FFF794FF002008BD4FF4877095
:1052700008BD40F20D1008BD4000FF1F10B58C782E
:10528000013CE1B2002301220F20F8F73DFC024B64
:1052900043F82400002010BD0823FF1F08B5002399
:1052A0001A46FF210F20F8F72FFC024B1860002050
:1052B00008BD00BF2823FF1F054A942303FB0023DA
:1052C0000020D3F8842022F00402C3F88420704721
:1052D0004000FF1F2DE9F047024604460023142139
:1052E0000620F8F711FC224600231521054606206A
:1052F000F8F70AFC524A534E4FF0940EB4230EFBBB
:10530000042E03FB04F3DEF88410F35821F0030CA1
:105310009907CEF884C040D4690001F0020141EA47
:105320000C0113F00103CEF8841005D100F0010C3C
:105330004CEA0101CEF88410002D66D0942101FBC7
:1053400004214D8805F02F0565B191F90F1006294C
:105350005BD03D4901EBC401D1E9006747F010077C
:10536000C1E90067002B37D1002835D0942303FB17
:105370000422538803F02F0363B192F90F30062BF8
:105380002AD0314B03EBC404D4E9002343F02003BB
:10539000C4E900230020BDE8F0872C49E5004E1940
:1053A00013F00103D6E900673CD04FF0000807F086
:1053B000100958EA090E11D0DFF88CE0AE44DEE99E
:1053C0000089294427F0100729F01009C1E9006776
:1053D000CEE90089002BC7D01C49E5004C19D4E95F
:1053E0000023002003F020010143D3D016480544D8
:1053F000D5E9000123F0200321F02001C5E90001D7
:10540000C4E900230020BDE8F0871049E5004E19EB
:10541000D6E900674FF0000807F0100958EA090EB6
:10542000CAD19FE700F0010A4FF0000807F0100909
:105430004AEA0C0CCEF884C058EA090EBCD193E7B6
:105440004000FF1FD400FF1F3086FF1F4086FF1F54
:10545000054A942303FB00230020D3F8842022F084
:105460000802C3F8842070474000FF1F38B5054686
:10547000FFF7BEFA044678B9B423084A03FB05F3E4
:105480000520D358590801F00201C3F3C0030B43B0
:105490002A46A621F8F738FB204638BDD400FF1F66
:1054A0000246002301210620F8F72EBB002070479A
:1054B000002070470C4A942303FB002393F90F103C
:1054C0004B1E092B0CD8DFE803F0090B070B0B056B
:1054D0000B09070C01F026BB00F096BD00F0E4BC00
:1054E000704700F063BE00BF4000FF1F2DE9F04190
:1054F000B54D35F81030D907044639D49A0700F174
:1055000084805F073FD41E0700F1918013F02006CE
:1055100040F0A58059064BD4DA0500F1D6809F05EE
:1055200000F1B7805E0500F1A480180500F1078145
:10553000D90400F114819A0400F121815B0400F187
:105540002E81A24A942303FB04235A8802F06F029F
:10555000272A23D193F90F30012B00F03081062B3D
:1055600000F02881D3B92046BDE8F04100F02CBB03
:105570000121FEF7C9FF98B101280FD0002325F8BB
:105580001430BDE8F081914B942606FB00360321D0
:10559000726EFFF785F8012800F08B80BDE8F0817E
:1055A00035F8143023F0010325F81430BDE8F081FC
:1055B000FEF7C2FF01280746F0D12046FFF71CF88E
:1055C000824B4FF0940808FB043898F90E300A2BF0
:1055D00013D0324646F264012046FFF737F93146D0
:1055E000D8F8183022460520F8F78EFAD8F8183087
:1055F000394622460520F8F787FA35F8143023F0AB
:10560000400325F81430BDE8F08101F079FC6F4AC1
:1056100035F81410942303FB042321F002015A8867
:1056200025F8141042F480625A80BDE8F081684B7E
:10563000032153F82020FFF733F80128AED1634A45
:1056400035F81410942303FB042321F008015A8831
:1056500025F8141042F480625A80BDE8F081FEF70C
:1056600055FF35F8143023F0200325F81430BDE839
:10567000F0815649942202FB001223F48061538882
:1056800025F8101023F06F0343F021035380BDE889
:10569000F0814E49942202FB001223F400715388DA
:1056A00025F8101023F06F0343F040035380BDE84A
:1056B000F081728835F8143042F4806223F00403DC
:1056C000728025F81430BDE8F0814049942202FB35
:1056D000001292F90E100A290ED8DFE801F02B23F0
:1056E0000D1B0D0D130D231B060000F065FD20465C
:1056F00000F046FD35F8143023F4807325F814309B
:10570000BDE8F08101F042FA204600F0ADFE35F828
:105710001430F1E700F08AFC204600F05FFC35F819
:105720001430E9E700F0F8FB204600F01FFB35F8E5
:105730001430E1E700F062FA35F81430DCE7234971
:10574000942202FB041223F40061538825F81410FC
:1057500023F06F0343F023035380BDE8F0811B491E
:10576000942202FB041223F48051538825F814106C
:1057700023F06F0343F027035380BDE8F081134902
:10578000942202FB041223F40051538825F81410CC
:1057900023F06F0343F007035380BDE8F0812046F8
:1057A000FFF788FE35F8143023F4804325F81430D1
:1057B000BDE8F0812046BDE8F04100F0D7BF2046AB
:1057C000BDE8F04100F050BBBC37FF1F4000FF1F99
:1057D0008486FF1F38B50A4B03EB40024FF6FF717A
:1057E0000025044623F81050918001F09BF9054BE9
:1057F000942202FB04344FF40473638038BD00BF6D
:10580000BC37FF1F4000FF1F38B5234D0446FFF78C
:1058100051FE942303FB045393F90E100A2937D841
:10582000DFE801F01330361C36362536301C060012
:10583000204600F0C1FC204600F0A2FCB0B9942341
:1058400003FB0454A37BE37338BD204600F0D6F974
:10585000942303FB04540020E07338BD204600F07D
:10586000E5FB204600F0BAFB0028E8D038BD204612
:1058700001F070F90028F9D1942303FB04540623A6
:10588000E37338BD204600F027FB0028EED1D6E7B1
:105890004FF48470EAE700BF4000FF1F0929034668
:1058A00005D00A2906D0032901D0002070471846E8
:1058B00000F0DCBB00F094BC2DE9F84FB84DB94FB7
:1058C000942303FB00F3EE1835F803E0738827F800
:1058D00010E013F06F01024607D1B34B4FF40C7484
:1058E000084623F81240BDE8F88FDFF8BC924FEA73
:1058F000400809EB080A4029BAF804C004460EF033
:105900008F020CF08F0B0CD10EF0870EBEF1060F3C
:1059100000F089805A4514BF4FF489700020BDE81B
:10592000F88F212919D023293AD0272947D00729D0
:1059300059D0082974D11EF0800FEBD0FEF778FD06
:10594000738837F81420AAF8042023F06F0343F07B
:10595000400373800020BDE8F88F072A16D00F2A75
:105960004FD00EF08601022902D01EF0820FD1D155
:105970009422C84402FB045423F06F0343F0400315
:10598000A8F804E063800020BDE8F88F23F06F03DF
:1059900043F023037380AAF804E00020BDE8F88FE9
:1059A0000F2A2ED00EF087010629DAD14FF4846336
:1059B00029F81030AAF804E00020BDE8F88F072A83
:1059C00051D00EF08703062B56D01EF0820042D035
:1059D0000EF08603022B58D05A4500F0A9804FF4F0
:1059E0008970BDE8F88F1EF082002CD00F2A91D16B
:1059F0004FF48853AAF804E029F814300020BDE8D9
:105A0000F88F96F90F10FFF749FF50B937F81430A7
:105A1000AAF804304FF48E5329F81430BDE8F88FFB
:105A20000020BDE8F88F0021FEF76EFD0128F8D8B0
:105A300037F81430AAF8043040F2014329F8143042
:105A40000020BDE8F88F4FF40C73AAF804E029F8A1
:105A50001430BDE8F88F44F23823AAF804E029F89E
:105A60001430BDE8F88F44F6380329F81030AAF84E
:105A700004E00020BDE8F88F44F2384329F81030E4
:105A8000AAF804E00020BDE8F88FB6F90430013B25
:105A9000062BA4D801A252F823F000BF1D5B010021
:105AA000095B0100F55A0100DF590100E15A0100CC
:105AB000CD5A0100B95A0100C84446F20203A8F8C1
:105AC00004E029F814300020BDE8F88FC84446F2FD
:105AD0000403A8F804E029F814300020BDE8F88F8A
:105AE000C84446F20803A8F804E029F8143000205E
:105AF000BDE8F88FC84444F23223A8F804E029F83E
:105B000014300020BDE8F88FC84444F23423A8F8CC
:105B100004E029F814300020BDE8F88FC84444F2AE
:105B20003823A8F804E029F814300020BDE8F88FE5
:105B30000EF45C7E0CF45C7CE6453FF471AF94237C
:105B400003FB045595F90F300A2B24D8DFE803F046
:105B50001F1B2317232313231B170600204600F0C7
:105B60000FFB00287FF45DAFC84437F81430A8F865
:105B70000430BDE8F88F204600F076FCF1E72046BF
:105B800000F02CFAEDE7204600F0F0F8E9E72046B7
:105B900000F018F8E5E74FF48470BDE8F88F00BF17
:105BA0004000FF1F8886FF1FBC37FF1F044B33F8E0
:105BB000100000F00E00003018BF0120704700BF39
:105BC000BC37FF1F002070470A4A10B5942404FB1D
:105BD00000246288530500D510BD074A072152F8FA
:105BE0002020FEF75DFD0128F6D1638843F4806331
:105BF000638010BD4000FF1F8486FF1F044A94236A
:105C000003FB0020438823F450534380704700BFB8
:105C10004000FF1FF0B4234D942303FB005393F97E
:105C20000F40012C35D0082C05BF1A6C996F00214C
:105C300089181D4B00EB400203EB82039A689142E6
:105C400003DB40F21510F0BC70475B689942F8DD49
:105C5000164B03EBC003D3E90023002603F0100723
:105C600056EA070405D0942404FB0054A469A14219
:105C7000E7DA002203F02003134310D0942303FB40
:105C8000005040F2151380698142D4BF18460020AD
:105C9000D9E7402ACDD19A69196C1144C9E700208F
:105CA000D1E700BF4000FF1F7886FF1F3086FF1F2F
:105CB00010B50446FEF70CFE0449054A942303FB85
:105CC00004131B6A42F8243010BD00BF4000FF1FC0
:105CD0008C86FF1F0E4A942303FB002310B51A6A1B
:105CE000531C0FD0002A0ADB0A4C44F8202013462C
:105CF0000246497A0520F7F707FF002010BD4FF450
:105D0000877010BD034A002342F82030F0E700BF3F
:105D10004000FF1F8C86FF1F70B582B002AA0023CF
:105D200042F8043D05460E46FEF7F0FE044640B933
:105D30000D4A942303FB05235A8802F06F02272A99
:105D400002D0204602B070BD93F90F30012B01D074
:105D5000082BF6D12A46717A019B0520F7F7D4FE6D
:105D6000204602B070BD00BF4000FF1F2DE9F04388
:105D70002A4B2B4E33F81020942712F0400283B0A8
:105D8000044607FB00670BD1D7F840804146FFF778
:105D900041FF0546002836D0284603B0BDE8F08311
:105DA000D7F8408040224146FFF734FF0546814640
:105DB0000028F1D1FB6D796DCDF8048001201A46E1
:105DC00000902046FEF71EFC4B46054622464946FB
:105DD0000620F7F799FE002DDED11248942101FB31
:105DE000046130F814204B8822F0020242F00102D4
:105DF00023F4806343F4805320F8142028464B801A
:105E000003B0BDE8F083FB6D796D1A468DE8200183
:105E10002046FEF7F7FB0546DDE700BF8886FF1F3B
:105E20004000FF1F9086FF1F0E4A942303FB0023B0
:105E30005A8802F06F02272A01D00020704793F998
:105E40000F30012B01D0082BF7D110B50446FFF716
:105E5000ADFE08B1002010BD2046BDE81040FFF7A0
:105E600085BF00BF4000FF1F0D4B33F8103013F00B
:105E7000020300D07047024610B59C21044606205C
:105E8000F7F742FE074B942202FB043400096388B3
:105E900000F4806023F480631843608010BD00BF6D
:105EA0009086FF1F4000FF1F38B50A4B942404FB67
:105EB00000340D46E36D00211A46FEF767FB012D05
:105EC00002D0082D00D038BD638823F4405363808E
:105ED00038BD00BF4000FF1F0C4A0D4B32F81020A8
:105EE000D20648BF03224FF0020123F8101048BF2A
:105EF00023F81020074B942202FB003300205A881D
:105F000022F4405242F480625A8070478886FF1F14
:105F10009086FF1F4000FF1F012910B5044611D0D5
:105F2000082900D010BD0246002392210520F7F772
:105F3000EBFD0F4B942202FB0434638843F480533F
:105F4000638010BD0B46024692210520F7F7DCFD69
:105F5000074B0849942202FB04320220538821F89F
:105F6000140023F4405343F48063538010BD00BFFA
:105F70004000FF1F9086FF1F38B502460446497A4D
:105F800000230620F7F7C0FD124B014653F82430DA
:105F9000204698471049942303FB04135A88D8627B
:105FA00002F06F05272D01D0002038BD93F90F3086
:105FB000032B01D0092BF7D1942303FB0414D4F84D
:105FC000883098420CBF42F4806222F48062628082
:105FD000002038BD6C86FF1F4000FF1F10B504462F
:105FE000FFF7E4FD08B1002010BD064B942202FB30
:105FF00004322046D36DD2F88810BDE810401A460E
:10600000FEF7C4BA4000FF1F074B10B5942404FBF1
:1060100000340021E36D1A46FEF7B8FA638823F4D2
:106020004053638010BD00BF4000FF1F032910B51F
:10603000044611D0092908D00B48942303FB04001F
:10604000438823F45053438010BD0246002392211D
:106050000520F7F759FDEFE70246012392210520BD
:10606000F7F752FDE8E700BF4000FF1F2A4B03EBA4
:10607000C003D3E9002330B4002403F0040554EA3C
:10608000050123D0254C942101FB0041D1F8881053
:1060900000291BDD002403F0100554EA050140F23D
:1060A000151129D1002203F02003134324D01B4AE9
:1060B000942303FB002040F21513D0F8882031EA26
:1060C000220128BF1946084630BC7047002403F05F
:1060D000080554EA050112D10021002403F010053F
:1060E0002C43DFD00D4D942404FB0054D4F8884099
:1060F000002CD7DD40F21511084630BC7047074927
:10610000942404FB001440F21511D4F88840002CAC
:10611000A8BF0021E1E700BF3086FF1F4000FF1F3E
:1061200030B583B002AA002342F8043D0546FEF7CD
:10613000EDFC044668B92846FFF798FF044640B9CD
:106140000E4A942303FB05235A8802F06F02272A84
:1061500002D0204603B030BD93F90F30032B01D09D
:10616000092BF6D12846FFF721FD0028F1D12A4658
:10617000019B02210520F7F7C7FCEAE74000FF1F5B
:1061800010B50446FFF712FD58B9074B942101FBE7
:1061900004312246086BCB6F9B2103440520F7F79F
:1061A000B3FC002010BD00BF4000FF1F02460023CB
:1061B0009B210520F7F7A8BC024610B50023044632
:1061C00092210520F7F7A0FC044B942202FB043433
:1061D000638843F48053638010BD00BF4000FF1FFD
:1061E000284B03EBC003D3E9002330B4002403F0B1
:1061F000040554EA050121D0234C942101FB004100
:10620000096B00291ADD002403F0100554EA05018A
:1062100040F2151127D1002203F02003134322D0AE
:10622000194A942303FB002040F21513026B31EA54
:10623000220128BF1946084630BC7047002403F0ED
:10624000080554EA050111D10021002403F01005CE
:106250002C43E0D00C4D942404FB0054246B002C00
:10626000D9DD40F21511084630BC70470649942428
:1062700004FB001440F21511246B002CA8BF002170
:10628000E3E700BF3086FF1F4000FF1F70B582B0FC
:1062900002AA002342F8043D0646FEF737FC134AE3
:1062A000019B942404FB06240546E26F13440193EA
:1062B00048B93046FFF794FF054620B9638803F0DC
:1062C0006F03272B02D0284602B070BD94F90F301F
:1062D0000A2BF8D13046FFF769FC0028F3D132468B
:1062E000019B9B210520F7F70FFCECE74000FF1F07
:1062F00070B582B002AA002342F8043D0646FEF7BC
:1063000005FC134A019B942404FB06240546226BDA
:106310001344019348B93046FFF762FF054620B9A0
:10632000638803F06F03272B02D0284602B070BDAC
:1063300094F90F300A2BF8D13046FFF737FC0028CC
:10634000F3D13246019B9B210520F7F7DDFBECE7FB
:106350004000FF1F70B582B002AA002342F8043D3E
:1063600005460E46FEF7D2FB044640B90B4A94237D
:1063700003FB05235A8802F06F02272A02D0204629
:1063800002B070BD93F90F30062BF8D12A46717A0E
:10639000019B0520F7F7B8FBF1E700BF4000FF1FA6
:1063A0001C4A942303FB002393F96830232B2DD838
:1063B000DFE803F0122C2C2C2C2C2C2C2C2C2C2C2D
:1063C0002C2C2C2C2C20142C2C2C2C2C2C2C2C2C31
:1063D0002C2C2C2C2C2C2C1200207047B42303FBCB
:1063E00000F00D4B1B5813F0020F40F2151008BFC0
:1063F00000207047B42303FB00F0074B1B5813F039
:10640000010F40F2151008BF002070474FF4847050
:10641000704700BF4000FF1FD400FF1F70B582B05F
:1064200002AA002342F8043D05460E46FEF76EFB25
:10643000044618B90B4B5A5D012A02D0204602B01F
:1064400070BD5A19B17812799142F7D103EB8503E7
:1064500001989B68717A00FB03F32A460520F7F741
:1064600053FBEBE7C437FF1F9E4B33F8103013F09C
:106470001003F0B504D09C4B1A5CC2B10020F0BDF3
:10648000994A115C0029F9D0984C1354942101FBCE
:10649000004115184C882B7102EB800024F4405207
:1064A0004FF40004836004614A800020F0BD8F4DEA
:1064B000942404FB00548100D4F884E094F96860CB
:1064C0005F181C18C7F80CE0BA602271232E3AD866
:1064D000DFE816F0D500AA00B70085003900C60035
:1064E00039003900390039003900390039003900E4
:1064F00039003900390099002400700039005C002F
:1065000039003900390039003900390039003900C3
:106510003900390039005200490044005A18744CBF
:1065200014611EF0020F4FF00204546100F0CF809E
:10653000704C14614FF0FF34946119444FF0FF34F4
:106540000122CC610A62942202FB0052012451888C
:106550001C5421F4505353800020F0BD19444FF4D3
:1065600040020A61EFE719444FF4E00600240122DB
:106570000E614C610A62E6E719444FF4E00600241C
:106580004FF0FF320E614C610A62DCE75A18584C3A
:1065900014611EF0020F4FF00404546174D04FF0E8
:1065A000FF36554C96611461194401240022CC61D8
:1065B0000A62C8E75A184E4C14611EF0020F4FF0E1
:1065C000040454617BD04FF0FF364B4C966114614C
:1065D00019444FF0FF340022CC610A62B3E75A1825
:1065E000464C14611EF0020F4FF00404546159D060
:1065F0004FF0FF36424C9661146119444FF0FF3260
:10660000CA610A629FE75A18394C14611EF0010FE3
:106610004FF0010454615FD0364E94611661194405
:106620000122CA610A628EE75A18344C14611EF0C6
:10663000010F4FF0010454612ED0324E9461166167
:10664000EDE75A182D4C14611EF0020F4FF00204B2
:1066500054612FD02B4C14614FF0FF349461CCE780
:106660005A18264C14611EF0020F4FF004045461B6
:1066700052D04FF0FF36224C96611461CFE7194497
:106680004FF400020A615EE71EF0010F5CD00126A4
:10669000194C9661146187E74FF0FF361A4C9661EA
:1066A0001461BCE71EF0010F56D00126144C966110
:1066B0001461A2E70126154C966114619DE71EF056
:1066C000010F31D001260C4C9661146180E7012640
:1066D0000F4C9661146130E74FF0FF360D4C966118
:1066E00014619CE78886FF1FC437FF1F4000FF1F0F
:1066F000F303400000034000EF034000F303700089
:10670000EF03700000037000E7037000EB037000FC
:10671000EB034000E70340001EF0010F0CD0012600
:10672000114C966114617AE71EF0040F0CBF01242E
:106730004FF0FF3494614BE71EF0040F0CBF4FF095
:10674000FF34012494616AE71EF0040F0CBF4FF080
:10675000FF340124946127E71EF0040F0CBF0124CD
:106760004FF0FF34946148E7EF0370002DE9F043E8
:10677000B84E8700F41983B0226912F0F30F054672
:106780000FD112F4407178D112F4401F58D112F495
:10679000000340F0A880520200F1DB8003B0BDE8A6
:1067A000F083D30700F10081910740F1B080DFF85A
:1067B000ACE2E1686369942000FB05E0D0F8840056
:1067C00080EA010E1EEA030F1CBF22F01E022261A6
:1067D000820740F1FF800B4313F0020313D1F41939
:1067E000226912F0040F00F089819B4A236102EBB9
:1067F000C504D4E9002343F01003C4E90023F319CE
:1068000041F00201D960C20740F10581CB07C5D430
:10681000F219536913F00103C0D11069040740F164
:1068200073818D48136100EBC505D5E9002343F062
:106830002003C5E900233E4441F00101F160ADE7CA
:1068400012F4801340F00E819002A7D59C212A46B5
:106850000620F7F759F9C106A0D52846FDF7CCFE6A
:106860007E492269942303FB051522F400126B88EC
:10687000226143F480536B8090E7D10500F1D3800F
:1068800092058BD5754A63694FF0940909FB00297D
:10689000D9F8841011EA030800F00E818B070ED599
:1068A000F219536913F0020309D16B48136100EB2D
:1068B000C500D0E9002343F01003C0E90023CC0752
:1068C0007FF56CAF3E44736913F001037FF466AF4C
:1068D000614A336102EBC505D5E9002343F020038B
:1068E000C5E900235AE75D4A942303FB00250621EE
:1068F0006A6FFDF7D5FE01287FF450AF6A882369DF
:1069000042F4806223F400036A80236146E7D306E1
:1069100000F1BD80910665D412F0400940F0D880A6
:1069200013067FF53BAF4D4A63694FF0940808FBAF
:106930000028D8F884101942B0D000F0E1FA22699A
:10694000D8F88410731922F08002226183F8049031
:10695000A4E7024603210620F7F7D6F800287FF4C3
:106960001DAF3E4B3E4A942606FB0536B42303FB7F
:106970000523726CC3F8B02001212846FEF708FCFD
:1069800002212846FEF704FC736C2A465B42012173
:106990000520F7F7B9F87288236942F4A05223F46E
:1069A000800372802361F9E62C4BA169942202FBDB
:1069B00000323544536FD26E01FB02F11A46FDF7E7
:1069C000E5FD2369A269A26023F0010301222A7177
:1069D0002361E3E68C077FF516AFF31921F002017E
:1069E000D96010E71D4A942303FB002505216A6F37
:1069F000FDF756FE01287FF4D1AED5F884206369F7
:106A00001A4200F08780236923F0C0033E4423F03C
:106A100020033361C2E6CA077FF5C0AE3E4421F0D1
:106A20000101F160BAE60D4BE169942202FB0032EC
:106A30003544536F126F01FB02F11A46FDF7A6FDB4
:106A40002369E269A26023F4807302222A71236120
:106A5000A4E600BFC437FF1F3086FF1F4000FF1FA2
:106A6000D400FF1F2E4B0191942202FB00320091B3
:106A7000536F116F1A46FDF7C5FD2369226AA260A4
:106A80003544022223F480132A71236186E6244AC6
:106A9000942303FB002504216A6FFDF701FE012802
:106AA0007FF47CAE2369A26923F0100343F0030353
:106AB00052422361A26171E600F022FA2269D9F8FC
:106AC0008410731922F40072226183F80480E5E6D1
:106AD000134BA169942202FB00323544536F126FAD
:106AE00001FB02F11A46FDF751FD2369A269A2607C
:106AF00023F0400302222A7123614FE622F00203B1
:106B000043F00C0323617AE620F0020343F00C0308
:106B1000136190E6A26923695242A26176E700BF41
:106B20004000FF1F094B942270B402FB0032084C56
:106B300051882618002304EB800521F4405133715D
:106B40002354AB602B61518070BC70474000FF1F25
:106B5000C437FF1F0A4B0B4A33F810300A4913F0B1
:106B6000100318BF01231354942303FB001302EBFB
:106B700080025988002021F45051106159807047DB
:106B80008886FF1FC437FF1F4000FF1F084A942359
:106B900030B403FB0023074C5A8804EB8005002126
:106BA00022F45052215429615A8030BC704700BFF2
:106BB0004000FF1FC437FF1F014B01221A707047AE
:106BC000E837FF1F30B583B002AB002023F8020D79
:106BD000084619461446FDF713FEBDF80610B1F538
:106BE000005F0CD2B1F5B05F06D041F61243994276
:106BF00002D0002003B030BD00F016F9F9E72246BC
:106C00000546FDF7E5FE0028F4D1BDF8062046F262
:106C100040039A42EDD1054B0549942202FB05F24F
:106C200003EB45058B5AAB80E4E700BFE837FF1F55
:106C30004000FF1F30B583B002AB002423F8024DA3
:106C4000084619461546FDF7DBFDBDF80610B1F5FF
:106C5000005F02D2204603B030BD2A46FDF7F6FDA4
:106C600003B030BD431E032B14D8DFE803F002024B
:106C70000202094B9A79082A01D098717047074A95
:106C800030B4D2E90245987144F00064C2E902458B
:106C900030BC7047004BF0E7E837FF1F3086FF1F1E
:106CA000024B0122DA710020704700BFE837FF1F56
:106CB000704700BF00207047704700BF704700BF9B
:106CC00030B583B002AC0C4B44F8043D15460423A8
:106CD0002246052141F63240F9F7EAFB2246042319
:106CE000052141F63340F9F7E3FB0448854294BFA0
:106CF0000220002003B030BD40420F003F420F0091
:106D00002DE9F0413D4E337882B013B902B0BDE8B1
:106D1000F0813B4C00253570F9F70EF8208801957D
:106D2000002840D0374FDFF8E88046F2400518E0F1
:106D300046F26003994228D0019B04EB83039A78C2
:106D4000FDF746FE28B1D7E9022342F00402C7E965
:106D50000223019B0133072B019324D834F823002D
:106D600008B36946FDF74CFDBDF80010A942DFD11C
:106D7000942303FB00F306EB400238F80330B2F82B
:106D800004E09E45E5D09380D6E7942303FB00837F
:106D900093F90E2093F90F309A42CDD1019B013324
:106DA000072B0193DAD9184C2378002BAED002AD13
:106DB000164B45F8043D03212A46042341F6324090
:106DC000F9F776FB2A460423062141F63240F9F70B
:106DD0006FFB2A460423092141F63240F9F768FB8C
:106DE00002AA002522F8065D0223082141F632405E
:106DF000F9F75EFB257002B0BDE8F081E837FF1FB0
:106E00009486FF1F3086FF1F9386FF1FA086010018
:106E10004000FF1F034BD87910B10022DA71012026
:106E2000704700BFE837FF1F2DE9F043DFF8B88057
:106E300085B00024434608F120021C809C70043376
:106E40009342FAD104AF01AA47F8044D00213B4612
:106E500041F612400194F9F705FBC0B9019BB3B1AB
:106E60000546012400E0144602AA3B46E1B241F681
:106E7000124002950395F9F7F5FA621C064618B917
:106E80000298B0F5B05F05D0019BA342EBD805B0E6
:106E9000BDE8F08331463B4602AA02960396F9F715
:106EA000E1FA0028F3D1029E002EF0D0054681467B
:106EB000012401E0A642EAD302AA3B4621464FF450
:106EC000B050CDF80890F9F7CDFA08EB850230B94B
:106ED000029B190C1B0A28F8251093700135013408
:106EE000072DE4B2E6D9D2E79486FF1FF1F768BF19
:106EF00008B5F7F76FFFBDE80840F1F779BF00BFAD
:106F000008B5F7F767FFBDE80840F1F771BF00BFAC
:106F1000F6F7FEBAF3F74CB8F3F770B8F6F7A0BD82
:106F2000034613F8012B002AFBD1181A01387047C9
:106F300081F0004102E000BF83F0004330B54FEA2A
:106F400041044FEA430594EA050F08BF90EA020F97
:106F50001FBF54EA000C55EA020C7FEA645C7FEA2A
:106F6000655C00F0E2804FEA5454D4EB5555B8BF4D
:106F70006D420CDD2C4480EA020281EA030382EABE
:106F8000000083EA010180EA020281EA0303362D50
:106F900088BF30BD11F0004F4FEA01314FF4801C23
:106FA0004CEA113102D0404261EB410113F0004F35
:106FB0004FEA03334CEA133302D0524263EB4303EC
:106FC00094EA050F00F0A780A4F10104D5F1200E8A
:106FD0000DDB02FA0EFC22FA05F2801841F10001E5
:106FE00003FA0EF2801843FA05F359410EE0A5F1B9
:106FF00020050EF1200E012A03FA0EFC28BF4CF0EA
:10700000020C43FA05F3C01851EBE37101F000459F
:1070100007D54FF0000EDCF1000C7EEB00006EEBAC
:107020000101B1F5801F1BD3B1F5001F0CD3490836
:107030005FEA30004FEA3C0C04F101044FEA44528D
:1070400012F5800F80F09A80BCF1004F08BF5FEA14
:10705000500C50F1000041EB045141EA050130BDF4
:107060005FEA4C0C404141EB010111F4801FA4F197
:107070000104E9D191F0000F04BF01460020B1FAEC
:1070800081F308BF2033A3F10B03B3F120020CDA24
:107090000C3208DD02F1140CC2F10C0201FA0CF002
:1070A00021FA02F10CE002F11402D8BFC2F1200C67
:1070B00001FA02F120FA0CFCDCBF41EA0C0190401D
:1070C000E41AA2BF01EB0451294330BD6FEA040466
:1070D0001F3C1CDA0C340EDC04F11404C4F1200251
:1070E00020FA04F001FA02F340EA030021FA04F363
:1070F00045EA030130BDC4F10C04C4F1200220FABA
:1071000002F001FA04F340EA0300294630BD21FAF7
:1071100004F0294630BD94F0000F83F4801306BFBD
:1071200081F480110134013D4EE77FEA645C18BFB1
:107130007FEA655C29D094EA050F08BF90EA020F48
:1071400005D054EA000C04BF1946104630BD91EA40
:10715000030F1EBF0021002030BD5FEA545C05D143
:107160004000494128BF41F0004130BD14F5800482
:107170003CBF01F5801130BD01F0004545F0FE41F6
:1071800041F470014FF0000030BD7FEA645C1ABF2B
:10719000194610467FEA655C1CBF0B46024650EA62
:1071A000013406BF52EA033591EA030F41F400218E
:1071B00030BD00BF90F0000F04BF0021704730B514
:1071C0004FF4806404F132044FF000054FF00001E9
:1071D00050E700BF90F0000F04BF0021704730B5AA
:1071E0004FF4806404F1320410F0004548BF40427F
:1071F0004FF000013EE700BF42004FEAE2014FEAD4
:1072000031014FEA02701FBF12F07F4393F07F4FAE
:1072100081F06051704792F0000F14BF93F07F4FE0
:10722000704730B54FF4607401F0004521F0004123
:1072300020E700BF50EA010208BF704730B54FF0A9
:1072400000050AE050EA010208BF704730B511F0AE
:10725000004502D5404261EB41014FF4806404F1E6
:1072600032045FEA915C3FF4DCAE4FF003025FEA68
:10727000DC0C18BF03325FEADC0C18BF033202EBF0
:10728000DC02C2F1200300FA03FC20FA02F001FA4A
:1072900003FE40EA0E0021FA02F11444C1E600BFE9
:1072A00070B54FF0FF0C4CF4E06C1CEA11541DBF9C
:1072B0001CEA135594EA0C0F95EA0C0F00F0DEF867
:1072C0002C4481EA030621EA4C5123EA4C5350EA4C
:1072D000013518BF52EA033541F4801143F480139D
:1072E00038D0A0FB02CE4FF00005E1FB02E506F02E
:1072F0000042E0FB03E54FF00006E1FB03569CF083
:10730000000F18BF4EF0010EA4F1FF04B6F5007F88
:1073100064F5407404D25FEA4E0E6D4146EB0606FA
:1073200042EAC62141EA55514FEAC52040EA5E5083
:107330004FEACE2EB4F1FD0C88BFBCF5E06F1ED82D
:10734000BEF1004F08BF5FEA500E50F1000041EB64
:10735000045170BD06F0004646EA010140EA020011
:1073600081EA0301B4EB5C04C2BFD4EB0C0541EA33
:10737000045170BD41F480114FF0000E013C00F348
:10738000AB8014F1360FDEBF002001F0004170BD6C
:10739000C4F10004203C35DA0C341BDC04F1140485
:1073A000C4F1200500FA05F320FA04F001FA05F211
:1073B00040EA020001F0004221F0004110EBD370DE
:1073C00021FA04F642EB06015EEA430E08BF20EA0A
:1073D000D37070BDC4F10C04C4F1200500FA04F3AD
:1073E00020FA05F001FA04F240EA020001F000413F
:1073F00010EBD37041F100015EEA430E08BF20EAB2
:10740000D37070BDC4F1200500FA05F24EEA020EF9
:1074100020FA04F301FA05F243EA020321FA04F028
:1074200001F0004121FA04F220EA020000EBD370DF
:107430005EEA430E08BF20EAD37070BD94F0000FDF
:107440000FD101F00046400041EB010111F4801F13
:1074500008BF013CF7D041EA060195F0000F18BFC4
:10746000704703F00046520043EB030313F4801F00
:1074700008BF013DF7D043EA0603704794EA0C0FBA
:107480000CEA135518BF95EA0C0F0CD050EA4106D0
:1074900018BF52EA4306D1D181EA030101F000414D
:1074A0004FF0000070BD50EA410606BF1046194675
:1074B00052EA430619D094EA0C0F02D150EA013681
:1074C00013D195EA0C0F05D152EA03361CBF1046C2
:1074D00019460AD181EA030101F0004141F0FE4161
:1074E00041F470014FF0000070BD41F0FE4141F4E5
:1074F000780170BD70B54FF0FF0C4CF4E06C1CEAE5
:1075000011541DBF1CEA135594EA0C0F95EA0C0F99
:1075100000F0A7F8A4EB050481EA030E52EA033554
:107520004FEA013100F088804FEA03334FF0805575
:1075300045EA131343EA12634FEA022245EA1115A2
:1075400045EA10654FEA00260EF000419D4208BF53
:10755000964244F1FD0404F5407402D25B084FEA00
:107560003202B61A65EB03055B084FEA32024FF4AC
:1075700080104FF4002CB6EB020E75EB030E22BF09
:10758000B61A754640EA0C005B084FEA3202B6EBC9
:10759000020E75EB030E22BFB61A754640EA5C0078
:1075A0005B084FEA3202B6EB020E75EB030E22BF08
:1075B000B61A754640EA9C005B084FEA3202B6EB09
:1075C000020E75EB030E22BFB61A754640EADC00C8
:1075D00055EA060E18D04FEA051545EA16754FEA2A
:1075E00006164FEAC30343EA52734FEAC2025FEA48
:1075F0001C1CC0D111F4801F0BD141EA00014FF0D7
:1076000000004FF0004CB6E711F4801F04BF0143A7
:107610000020B4F1FD0C88BFBCF5E06F3FF6AFAEC3
:10762000B5EB030C04BFB6EB020C5FEA500C50F153
:10763000000041EB045170BD0EF0004E4EEA1131D6
:1076400014EB5C04C2BFD4EB0C0541EA045170BDDD
:1076500041F480114FF0000E013C90E645EA060E21
:107660008DE60CEA135594EA0C0F08BF95EA0C0F4F
:107670003FF43BAF94EA0C0F0AD150EA01347FF497
:1076800034AF95EA0C0F7FF425AF104619462CE76E
:1076900095EA0C0F06D152EA03353FF4FDAE1046D1
:1076A000194622E750EA410618BF52EA43067FF422
:1076B000C5AE50EA41047FF40DAF52EA43057FF4B2
:1076C000EBAE12E74FF0FF3C06E000BF4FF0010CBD
:1076D00002E000BF4FF0010C4DF804CD4FEA410C21
:1076E0007FEA6C5C4FEA430C18BF7FEA6C5C1BD0EE
:1076F00001B050EA410C0CBF52EA430C91EA030F6F
:1077000002BF90EA020F0020704710F1000F91EACB
:10771000030F58BF994208BF90422CBFD8176FEA99
:10772000E37040F0010070474FEA410C7FEA6C5C67
:1077300002D150EA013C07D14FEA430C7FEA6C5C6E
:10774000D6D152EA033CD3D05DF8040B704700BF9A
:107750008446104662468C461946634600E000BFE8
:1077600001B5FFF7B7FF002848BF10F1000F01BDBA
:107770004DF808EDFFF7F4FF0CBF012000205DF885
:1077800008FB00BF4DF808EDFFF7EAFF34BF01200A
:1077900000205DF808FB00BF4DF808EDFFF7E0FFA3
:1077A00094BF012000205DF808FB00BF4DF808EDF4
:1077B000FFF7CEFF94BF012000205DF808FB00BF5B
:1077C0004DF808EDFFF7C4FF34BF012000205DF83D
:1077D00008FB00BF4FEA410C7FEA6C5C02D150EA23
:1077E000013C0AD14FEA430C7FEA6C5C02D152EAB9
:1077F000033C02D14FF0000070474FF0010070478A
:107800004FEA4102B2F1E04324BFB3F5001CDCF1C2
:10781000FE5C0DD901F0004C4FEAC0024CEA5070FA
:10782000B2F1004F40EB830008BF20F00100704729
:1078300011F0804F21D113F13872BCBF01F000402C
:10784000704741F480114FEA5252C2F11802C2F15E
:10785000200C10FA0CF320FA02F018BF40F00100DF
:107860004FEAC1234FEAD32303FA0CFC40EA0C0091
:1078700023FA02F34FEA4303CCE77FEA625307D1CE
:1078800050EA01331EBF4FF0FE4040F44000704705
:1078900001F0004040F0FE4040F40000704700BF9F
:1078A00080F0004002E000BF81F0004142001FBFB5
:1078B0005FEA410392EA030F7FEA226C7FEA236CBE
:1078C0006AD04FEA1262D2EB1363C1BFD2184140B3
:1078D00048404140B8BF5B42192B88BF704710F049
:1078E000004F40F4000020F07F4018BF404211F0EC
:1078F000004F41F4000121F07F4118BF494292EA54
:10790000030F3FD0A2F1010241FA03FC10EB0C007F
:10791000C3F1200301FA03F100F0004302D549420C
:1079200060EB4000B0F5000F13D3B0F1807F06D3B9
:1079300040084FEA310102F10102FE2A51D2B1F1B1
:10794000004F40EBC25008BF20F0010040EA0300A6
:107950007047490040EB000010F4000FA2F1010253
:10796000EDD1B0FA80FCACF1080CB2EB0C0200FADD
:107970000CF0AABF00EBC25052421843BCBFD0402B
:107980001843704792F0000F81F4000106BF80F4A5
:1079900000000132013BB5E74FEA41037FEA226C68
:1079A00018BF7FEA236C21D092EA030F04D092F033
:1079B000000F08BF0846704790EA010F1CBF002067
:1079C000704712F07F4F04D1400028BF40F00040C4
:1079D000704712F100723CBF00F50000704700F0E4
:1079E000004343F0FE4040F4000070477FEA22620B
:1079F00016BF08467FEA23630146420206BF5FEADC
:107A0000412390EA010F40F4800070474FF00003DB
:107A100004E000BF10F0004348BF40425FEA000CA2
:107A200008BF704743F0964301464FF000001CE04A
:107A300050EA010208BF70474FF000030AE000BFA0
:107A400050EA010208BF704711F0004302D54042DE
:107A500061EB41015FEA010C02BF84460146002050
:107A600043F0B64308BFA3F18053A3F50003BCFA6B
:107A70008CF2083AA3EBC25310DB01FA02FC634418
:107A800000FA02FCC2F12002BCF1004F20FA02F21F
:107A900043EB020008BF20F00100704702F1200212
:107AA00001FA02FCC2F1200250EA4C0021FA02F273
:107AB00043EB020008BF20EADC7070474FF0FF0C78
:107AC0001CEAD0521EBF1CEAD15392EA0C0F93EA73
:107AD0000C0F6FD01A4480EA010C400218BF5FEA15
:107AE00041211ED04FF0006343EA501043EA511188
:107AF000A0FB01310CF00040B1F5000F3EBF490082
:107B000041EAD3715B0040EA010062F17F02FD2A85
:107B10001DD8B3F1004F40EBC25008BF20F0010068
:107B2000704790F0000F0CF0004C08BF49024CEA7F
:107B3000502040EA51207F3AC2BFD2F1FF0340EA11
:107B4000C250704740F400004FF00003013A5DDC82
:107B500012F1190FDCBF00F000407047C2F10002C3
:107B6000410021FA02F1C2F1200200FA02FC5FEAB0
:107B7000310040F1000053EA4C0308BF20EADC70FA
:107B8000704792F0000F00F0004C02BF400010F46C
:107B9000000F013AF9D040EA0C0093F0000F01F019
:107BA000004C02BF490011F4000F013BF9D041EA3B
:107BB0000C018FE70CEAD15392EA0C0F18BF93EA3D
:107BC0000C0F0AD030F0004C18BF31F0004CD8D167
:107BD00080EA010000F00040704790F0000F17BFEE
:107BE00090F0004F084691F0000F91F0004F14D034
:107BF00092EA0C0F01D142020FD193EA0C0F03D18C
:107C00004B0218BF084608D180EA010000F000408E
:107C100040F0FE4040F40000704740F0FE4040F469
:107C2000400070474FF0FF0C1CEAD0521EBF1CEA08
:107C3000D15392EA0C0F93EA0C0F69D0A2EB030226
:107C400080EA010C49024FEA402037D04FF08053C0
:107C500043EA111143EA10130CF000408B4238BF85
:107C60005B0042F17D024FF4000C8B4224BF5B1A93
:107C700040EA0C00B3EB510F24BFA3EB510340EAE1
:107C80005C00B3EB910F24BFA3EB910340EA9C008F
:107C9000B3EBD10F24BFA3EBD10340EADC001B01FF
:107CA00018BF5FEA1C1CE0D1FD2A3FF650AF8B42A3
:107CB00040EBC25008BF20F0010070470CF0004CB0
:107CC0004CEA50207F32C2BFD2F1FF0340EAC250DB
:107CD000704740F400004FF00003013A37E792F09C
:107CE000000F00F0004C02BF400010F4000F013AFA
:107CF000F9D040EA0C0093F0000F01F0004C02BFF5
:107D0000490011F4000F013BF9D041EA0C0195E75D
:107D10000CEAD15392EA0C0F08D142027FF47DAFF6
:107D200093EA0C0F7FF470AF084676E793EA0C0FE6
:107D300004D14B023FF44CAF08466EE730F0004CE4
:107D400018BF31F0004CCAD130F000427FF45CAF74
:107D500031F000437FF43CAF5FE700BF4FF0FF3CE2
:107D600006E000BF4FF0010C02E000BF4FF0010C35
:107D70004DF804CD4FEA40024FEA41037FEA226CFE
:107D800018BF7FEA236C11D001B052EA530C18BF20
:107D900090EA010F58BFB2EB030088BFC81738BF85
:107DA0006FEAE17018BF40F0010070477FEA226C73
:107DB00002D15FEA402C05D17FEA236CE4D15FEA6F
:107DC000412CE1D05DF8040B704700BF84460846A3
:107DD0006146FFE70FB5FFF7C9FF002848BF10F164
:107DE000000F0FBD4DF808EDFFF7F4FF0CBF0120A9
:107DF00000205DF808FB00BF4DF808EDFFF7EAFF33
:107E000034BF012000205DF808FB00BF4DF808EDED
:107E1000FFF7E0FF94BF012000205DF808FB00BFE2
:107E20004DF808EDFFF7D2FF94BF012000205DF868
:107E300008FB00BF4DF808EDFFF7C8FF34BF012075
:107E400000205DF808FB00BF4FEA4002B2F1FE4F90
:107E50000FD34FF09E03B3EB12620DD94FEA00230C
:107E600043F0004310F0004F23FA02F018BF4042E5
:107E700070474FF00000704712F1610F01D14202CC
:107E800005D110F0004008BF6FF0004070474FF080
:107E9000000070477BB972B90029BEBF00204FF0C7
:107EA000004106E008BF00281CBF6FF000414FF002
:107EB000FF3000F0FFB9ADF1080C6DE904CE0029E8
:107EC00009DB002B1ADB00F087F8DDF804E0DDE9C0
:107ED000022304B07047404261EB4101002B1BDBE1
:107EE00000F07AF8DDF804E0DDE9022304B0404256
:107EF00061EB4101524263EB43037047524263EB33
:107F0000430300F069F8DDF804E0DDE9022304B082
:107F1000404261EB41017047524263EB430300F082
:107F20005BF8DDF804E0DDE9022304B0524263EBC4
:107F30004303704753B94AB9002908BF00281CBF42
:107F40004FF0FF314FF0FF3000F0B4B9ADF1080C45
:107F50006DE904CE00F040F8DDF804E0DDE902232D
:107F600004B0704710B500210446FFF745FF20B963
:107F70002046BDE8104000F009B804F1004000F0D0
:107F800005F8404261EB410110BD00BFD0B5FFF7DD
:107F900033F900220E4B06460F46FFF781F900F039
:107FA0008BF90446FFF706F900220A4BFFF778F930
:107FB00002460B4630463946FEF7BEFF00F07CF91C
:107FC0002346002242EA000210461946D0BD00BFF7
:107FD0000000F03D0000F0412DE9F0478C460D46D1
:107FE0000446089E002B51D18A4217466DD9B2FA39
:107FF00082FEBEF1000F0BD0CEF1200C01FA0EF57F
:1080000020FA0CFC02FA0EF74CEA050C00FA0EF40A
:108010004FEA174A250CBCFBFAF81FFA87F90AFB4E
:1080200018CC45EA0C4508FB09F3AB420AD9ED1917
:1080300008F1FF3280F02381AB4240F22081A8F1A9
:1080400002083D44ED1AA4B2B5FBFAF00AFB105544
:1080500044EA054400FB09F9A14509D9E41900F1F6
:10806000FF3380F00A81A14540F2078102383C4489
:10807000A4EB090440EA08400021002E61D024FA54
:108080000EF4002334607360BDE8F0878B4207D99B
:10809000002E54D0002186E821000846BDE8F08774
:1080A000B3FA83F1002940F08E80AB4202D38242C2
:1080B00000F2FA80841A65EB03050120AC46002E1D
:1080C0003FD086E81010BDE8F08712B90127B7FB52
:1080D000F2F7B7FA87FEBEF1000F34D1EB1B3A0C72
:1080E0001FFA87FC0121B3FBF2F8250C02FB1833C1
:1080F00045EA03450CFB08F3AB4207D9ED1908F13B
:10810000FF3002D2AB4200F2D1808046ED1AA3B21A
:10811000B5FBF2F002FB105543EA05440CFB00FCF2
:10812000A44507D9E41900F1FF3302D2A44500F2B7
:10813000B8801846A4EB0C0440EA08409DE731469D
:108140003046BDE8F087CEF1200405FA0EF307FAB9
:108150000EF720FA04F83A0C25FA04F448EA03086A
:10816000B4FBF2F14FEA184502FB11441FFA87FCF9
:1081700045EA044501FB0CF3AB4200FA0EF409D9C1
:10818000ED1901F1FF3080F08A80AB4240F2878028
:1081900002393D44EB1A1FFA88F5B3FBF2F002FBFB
:1081A000103345EA034500FB0CF3AB4207D9ED1948
:1081B00000F1FF386FD2AB426DD902383D44EB1A63
:1081C00040EA01418FE7C1F1200722FA07F88B400E
:1081D00005FA01F448EA030320FA07FE4FEA134CBC
:1081E000FD404EEA040EB5FBFCF94FEA1E440CFBC1
:1081F00019551FFA83F844EA054509FB08F4AC4217
:1082000002FA01F200FA01FA08D9ED1809F1FF307B
:1082100043D2AC4241D9A9F102091D442D1B1FFADA
:108220008EFEB5FBFCF00CFB10554EEA054400FB3E
:1082300008F8A04507D9E41800F1FF3529D2A04578
:1082400027D902381C4440EA0940A4EB0804A0FBEB
:1082500002894C45C6464D4615D312D056B1BAEBED
:108260000E0364EB050404FA07F7CB401F43CC4030
:10827000376074600021BDE8F0871846F8E6904644
:10828000E0E6C245EAD2B8EB020E69EB030501381D
:10829000E4E72846D7E7404691E78146BEE7014636
:1082A00078E702383C4445E7084608E7A8F10208A9
:1082B0003D442BE7704700BF4A0011D212F500126F
:1082C00011D20DD56FF47873B3EB62520ED44FEA2E
:1082D000C12343F0004343EA505323FA02F07047AE
:1082E0004FF00000704750EA013002D14FF0FF30EC
:1082F00070474FF00000704738B5F1F71FFB62B6CA
:10830000F0F7A8FAF0F7C4FAF0F728FB204C05467E
:10831000F1F716FBF0F7BEFE2A461E492046F1F79C
:10832000F9FFF0F70BFF2078F1F79CF82079F1F7CF
:10833000E3F8F0F7E1FBF0F743FE174B01241C7064
:10834000F4F728FDF5F7CAFD40F21670F2F74EFE7D
:10835000FBF7C8FCFBF706FD0AE0FBF709FDC0B21E
:1083600005280FD0F7F7E0FCF1F7FEFAF7F7B4FCB9
:108370000120F5F729FAF6F765F8002CEDD1FBF7A7
:10838000A7FDEFE7F9F784F90024FBF761FDE9E7C2
:108390007438FF1FF037FF1F7038FF1F10B5431EE2
:1083A0000A44914200D110BD11F8014B03F8014F6E
:1083B000F7E702440346934200D1704703F8011BDC
:1083C000F9E700002DE970438AB004460D4600F03D
:1083D00077F8354B93F90060731C804689460DD0C1
:1083E00022462B4620462946FFF7F4F930B90022F1
:1083F000002320462946FFF7E3F920B140464946CD
:108400000AB0BDE87083294B0890CDE90245CDE95B
:108410000445019320462946CEB9254D4FF06044CE
:1084200000220023CDE90645FFF7A2F9002833D04A
:1084300002230093684600F037FAA8B1089BC3B93D
:10844000DDE90689404649460AB0BDE87083194D0A
:10845000002400220023CDE90645FFF789F968B121
:1084600002239E420093E5D100F026FA2223036006
:10847000E4E700F021FA089B0360E1E70123022E04
:1084800000930BD100F018FA212303600A4800F092
:108490000DFACDE90601D1E701230093684600F00B
:1084A00003FA0028F2D1EDE72421FF1F40A80100C4
:1084B000FFFFEFC70000F0FF109D0100000000006B
:1084C0002DE9F04FB1F5801F85B006460F460B46EB
:1084D0005ADA024621F00044224300F0F8800029D5
:1084E000C0F27A810022D64BFEF7DAFED54A0B465F
:1084F000934206460F466FF0350C4ADCC3F3130572
:1085000005F5152E0EF6647E0EF4801E8EF07F5259
:1085100082F440121C1542EA0507A4F2FF346444B9
:108520000022C94B3046394604EB1E54FEF704FDC9
:10853000AB1CC3F31303022B82468B464FF00002A1
:1085400030DC0023FFF714F9002800F0C980002C6C
:1085500000F04B812046FEF73DFEA5A3D3E90023A2
:1085600006460F46FEF79CFEA3A3D3E9002304466C
:108570000D4630463946FEF793FE02460B4620462E
:108580002946FEF7DBFC0AE0AE4A93424FF0000CAE
:10859000B4DD32463B4630463946FEF7CFFC05B0E7
:1085A000BDE8F08F4FF08043FEF7C8FC02460B4653
:1085B00050465946FEF79EFF064620460F46FEF7F8
:1085C00009FE3246CDE900013B4630463946CDE949
:1085D0000267FEF765FE02460B4680468946FEF7B7
:1085E0005FFE87A3D3E9002306460F46FEF758FE39
:1085F00085A3D3E90023FEF7A1FC32463B46FEF7F4
:108600004FFE83A3D3E90023FEF798FC32463B4696
:10861000FEF746FE80A3D3E90023FEF78FFC424617
:108620004B46FEF73DFE7EA3D3E9002380468946F4
:1086300030463946FEF734FE7BA3D3E90023FEF72C
:108640007DFC32463B46FEF72BFE79A3D3E900239F
:10865000FEF774FC32463B46FEF722FE0B4602460E
:1086600049464046FEF76AFCA5F5C223C5F5D72565
:10867000A3F27A4351351D43002D8046894656DDCD
:108680000022724B50465946FEF70AFE52465B46A0
:10869000FEF706FE06460F46002C68D132463B46E2
:1086A00040464946FEF74AFCDDE90223FEF7F8FDA5
:1086B00002460B4630463946FEF73EFC02460B4664
:1086C00050465946FEF738FC05B0BDE8F08F002251
:1086D000002300205E49FEF70DFF05B0BDE8F08FD6
:1086E00055A3D3E9002350465946FEF7D9FD02466B
:1086F0000B4600205549FEF71FFC524606460F4622
:108700005B4650465946FEF7CBFD02460B463046C7
:108710003946FEF7C5FD06460F46002C40F09A800C
:1087200002460B4650465946FEF706FC37E7002C3A
:1087300000F0A4802EA3D3E90023DDE90001FEF7B9
:10874000AFFD42464B4604460D4650465946FEF79D
:10875000F3FBDDE90223FEF7A3FD27A3D3E9002302
:1087600006460F46DDE90001FEF79AFD21E020A351
:10877000D3E90023DDE90001FEF792FD32463B46D6
:1087800004460D4640464946FEF7D8FBDDE9022384
:10879000FEF786FD18A3D3E9002380468946DDE96C
:1087A0000001FEF77DFD02460B4640464946FEF7B6
:1087B000C5FB02460B4630463946FEF7BDFB524626
:1087C0005B46FEF7B9FB02460B4620462946FEF7FC
:1087D000B3FB05B0BDE8F08F02460B46FEF7ACFBDD
:1087E00000220023FEF786FED9E600200021D6E60F
:1087F0000000E0FE422EE63F763C7935EF39EA3D57
:1088000044523EDF12F1C23FDE03CB966446C73FBF
:10881000599322942449D23F935555555555E53FD8
:108820009FC678D0099AC33FAF788E1DC571CC3FE3
:1088300004FA97999999D93F555555555555D53FAE
:1088400000005043FFFFEF7F0000F03F0000E03FDB
:10885000000050C32046FEF7BDFC0FA3D3E9002360
:1088600080468946FEF71CFD0DA3D3E9002304468C
:108870000D4640464946FEF713FD9AE702460B4671
:1088800050465946FEF758FBDDE90223FEF708FD86
:1088900014E700BFAFF300800000E0FE422EE63F89
:1088A000763C7935EF39EA3D0020704700200149D8
:1088B000704700BF0000F87F014B1868704700BF89
:1088C000C020FF1F8025000040380000004B000042
:1088D000807000000096000000E10000002C010004
:1088E00000C201005515AC6A004001C0ABEA5795C3
:1088F0000010161B2023272A2D30323537393B3DF7
:108900004041434547494B4C4E505153545657599B
:108910005A5B5D5E60616263656667686A6B6C6D19
:108920006E707172737475767778797A7B7C7D7EE0
:1089300080808182838485868788898A8B8C8D8ECE
:108940008F9090919293949596969798999A9B9BD5
:108950009C9D9E9FA0A0A1A2A3A3A4A5A6A7A7A8F3
:10896000A9AAAAABACADADAEAFB0B0B1B2B2B3B420
:10897000B5B5B6B7B7B8B9B9BABBBBBCBDBDBEBF5C
:10898000C0C0C1C1C2C3C3C4C5C5C6C7C7C8C9C9A1
:10899000CACBCBCCCCCDCECECFD0D0D1D1D2D3D3ED
:1089A000D4D4D5D6D6D7D7D8D9D9DADADBDBDCDD43
:1089B000DDDEDEDFE0E0E1E1E2E2E3E3E4E5E5E69F
:1089C000E6E7E7E8E8E9EAEAEBEBECECEDEDEEEE02
:1089D000EFF0F0F1F1F2F2F3F3F4F4F5F5F6F6F767
:1089E000F7F8F8F9F9FAFAFBFBFCFCFDFDFEFEFFD7
:1089F000000203050608090B0D0E101113141617BB
:108A0000191B1C1E1F2122242527292A2C2D2F301B
:108A10003233353638393B3C3E3F41434446474983
:108A20004A4C4D4F505153545657595A5C5D5F60F4
:108A30006263646667696A6C6D6E70717374757772
:108A4000787A7B7C7E7F808283848687888A8B8C01
:108A50008E8F90929394959798999A9C9D9E9FA1A2
:108A6000A2A3A4A5A7A8A9AAABACAEAFB0B1B2B35C
:108A7000B4B5B7B8B9BABBBCBDBEBFC0C1C2C3C430
:108A8000C5C6C7C8C9CACBCCCDCECFD0D0D1D2D322
:108A9000D4D5D6D7D7D8D9DADBDCDCDDDEDFDFE032
:108AA000E1E2E2E3E4E4E5E6E7E7E8E8E9EAEAEB65
:108AB000ECECEDEDEEEEEFF0F0F1F1F2F2F3F3F4B9
:108AC000F4F4F5F5F6F6F7F7F7F8F8F8F9F9F9FA36
:108AD000FAFAFBFBFBFCFCFCFCFCFDFDFDFDFDFED6
:108AE000FEFEFEFEFEFEFFFFFFFFFFFFFFFFFFFF9C
:108AF0006B7FD87EB87DA07C8F7B857A82798578E4
:108B00000878147726763D7559747B73A172367296
:108B100064719670CC6F076F456EE66D2A6D726C4E
:108B2000BE6B0D6B5F6AB5696169BB68196879676F
:108B3000DC664266AB656065CC643B64AD63206314
:108B400096620F62CB614761C4604460C65F495F53
:108B5000CE5E925E1A5EA45D2F5DBD5C4B5CDC5BFD
:108B6000A55B385BCC5A625AF95992592C59F9587D
:108B700095583358D15771571257B4560000C90051
:108B800092015B022403ED03B6047F05480611073A
:108B9000D907A2086A09330AFB0AC40B8C0C540DCE
:108BA0001C0EE30EAB0F72103A110112C8128F1394
:108BB00055141C15E215A8166E173318F918BE19AE
:108BC000821A471B0B1CCF1C931D571E1A1FDD1F3B
:108BD0009F2061212322E522A62367242825E8255A
:108BE000A82667272628E528A329612A1F2BDC2B26
:108BF000992C552D112ECC2E872F4130FB30B531BD
:108C00006E322633DF3396344D350436BA366F373D
:108C10002438D9388C39403AF23AA53B563C073DC6
:108C2000B83D683E173FC53F73402141CE417A426F
:108C30002543D0437A442445CD4575461C47C34758
:108C400069480F49B449584AFB4A9D4B3F4CE04C98
:108C5000814D204EBF4E5D4FFB4F97503351CE514B
:108C6000685202539B533254C9546055F5558A5685
:108C70001D57B0574258D3586459F359825A0F5B65
:108C80009C5B285CB35C3E5DC75D4F5ED75E5D5FFD
:108C9000E35F6860EB606E61F0617162F162706366
:108CA000EE636C64E8646365DD655666CF664667AF
:108CB000BC673268A66819698B69FD696D6ADC6AF0
:108CC0004A6BB76B236C8E6CF86C616DC96D306E3E
:108CD000966EFB6E5E6FC16F22708370E2704071A2
:108CE0009D71F9715472AE7207735E73B5730A7435
:108CF0005F74B27404755575A575F37541768D76FC
:108D0000D87622776B77B377FA773F788478C7780D
:108D100009794A798979C879057A417A7C7AB67A6B
:108D2000EE7A267B5C7B917BC57BF87B297C597C2A
:108D3000887CB67CE37C0E7D397D627D897DB07D4B
:108D4000D57DFA7D1D7E3E7E5F7E7E7E9C7EB97ED9
:108D5000D57EEF7E097F217F377F4D7F617F747FD6
:108D6000867F977FA67FB47FC17FCD7FD87FE17F4D
:108D7000E97FF07FF57FF97FFD7FFE7F109D010089
:108D80003C9501004895010058950100749501003B
:108D900094950100B4950100C8950100D495010097
:108DA000E4950100F4950100049601001896010075
:108DB0002896010038960100489601005896010057
:108DC00004960100189601002896010038960100CB
:108DD00048960100589601006896010078960100B7
:108DE000889601009896010004960100A89601005B
:108DF000CC960100F096010014970100389701000D
:108E00005C97010078970100A0970100BC970100D2
:108E1000E097010008980100549801002098010093
:108E20002C9801004C980100609801007498010092
:108E3000889801007C98010098980100A89801008A
:108E4000B8980100D0980100E8980100FC98010052
:108E5000149901002C9901004899010064990100BE
:108E6000E097010008980100549801002098010043
:108E70002C9801004C98010060980100889801002E
:108E80007C98010098980100A8980100B89801000A
:108E9000D098010064990100709901008499010043
:108EA0009C990100AC990100C0990100D099010082
:108EB000C0990100DC990100E8990100F4990100D2
:108EC000C0990100049A0100189A0100149A010047
:108ED000289A0100349A0100409A0100509A01003A
:108EE000649A0100749A0100C0990100889A0100F7
:108EF0009C9A0100989A0100AC9A0100289A0100FE
:108F0000349A0100C09A0100D49A0100C09901006E
:108F1000EC9A0100009B0100FC9A0100289A0100D4
:108F2000109B0100249B01003C9B0100549B01000D
:108F3000689B0100C09901007C9B0100889B010097
:108F4000C09901007C9B0100989B0100A49B01003B
:108F5000C09901007C9B0100B49B0100C89B0100EB
:108F6000D09B0100DC9B0100E89B0100F49B010009
:108F7000C0990100049C0100189C0100289C01007C
:108F8000C0990100349C0100509C01005C9C0100D0
:108F9000649C0100789C0100909C0100A49C01004D
:108FA000B49C0100CC9C010004960100D89C0100F7
:108FB000E09C0100E89C0100F09C0100F89C01008D
:108FC000009D010004960100089D0100149D010010
:108FD000289D0100349D0100409D01004C9D010031
:108FE000589D0100649D0100709D0100889D010055
:108FF000A09D0100C09D0100D49D0100F09D0100D5
:10900000049E0100209E0100389E0100589E010030
:10901000689E0100809E0100909E0100A89E0100B4
:10902000C09E0100D89E0100E89E0100F89E01004C
:10903000049F0100189F0100289F0100389F010034
:10904000449F0100609F01007C9F0100989F0100E8
:10905000B09F0100CC9F0100DC9F0100F49F010044
:109060000CA0010024A00100449F010034A00100D5
:1090700048A001005CA0010070A0010080A00100D8
:1090800090A00100A49C0100A8A00100B8A00100CC
:10909000D0A00100109D01003C9501004895010001
:1090A000589501007495010094950100E4A0010019
:1090B000F4A0010014A1010038A1010058A1010091
:1090C00078A1010098A10100B8A10100D8A1010078
:1090D000F0A1010010A2010028A2010044A2010099
:1090E0005CA201006CA2010088A20100A8A20100FC
:1090F000C8A20100E0A20100FCA2010018A3010027
:1091000034A3010050A3010070A3010084A3010057
:10911000A49C0100B49C0100CC9C0100A0A3010010
:10912000B0A30100C0A30100D4A30100E8A3010083
:1091300008A4010024A4010048A4010060A40100C7
:1091400084A40100A0A40100C4A40100E0A40100C3
:1091500008A5010020A5010040A5010058A50100B7
:1091600074A5010090A50100ACA50100C4A50100F3
:10917000D8A50100ECA5010008A601001CA601006D
:1091800034A6010048A6010068A6010084A60100DB
:10919000A8A60100BCA60100D8A60100F4A6010003
:1091A00014A7010028A701003CA7010058A701004F
:1091B00070A7010084A70100A4A70100BCA70100BB
:1091C000D4A70100F0A7010000000000B801FF1FB4
:1091D000AC01FF1FA001FF1F000000000000000005
:1091E00000000000D400FF1FD800FF1FE400FF1F95
:1091F000E800FF1FEC00FF1F1C01FF1F4001FF1FC5
:109200004401FF1F5001FF1F7001FF1F7401FF1F6A
:109210007801FF1F7C01FF1F2823FF1F2423FF1F4E
:109220002023FF1F8801FF1F0823FF1F5C00FF1F73
:109230006000FF1F7400FF1F9000FF1F9400FF1FBE
:109240009800FF1F9C00FF1FA000FF1FA400FF1F2E
:10925000AC00FF1FB400FF1FC400FF1FCC00FF1FA6
:10926000D000FF1FDC00FF1FFC00FF1FFE00FF1FE0
:109270002001FF1F2201FF1F3801FF1F5A01FF1F9E
:109280005C01FF1F6001FF1F6A01FF1F6C01FF1FD0
:109290004000FF1F4200FF1F6400FF1FC000FF1FB0
:1092A000E000FF1F4801FF1F4901FF1F5601FF1F7C
:1092B0005701FF1F5E01FF1F5F01FF1F6801FF1FB6
:1092C0008001FF1FF000FF1FF400FF1FF800FF1FC9
:1092D0000001FF1F0401FF1F0801FF1F0C01FF1FFA
:1092E0001001FF1F1401FF1F1801FF1F2401FF1FA2
:1092F0002801FF1F2C01FF1F3001FF1F3401FF1F3A
:109300003C01FF1F6401FF1F8401FF1F5000FF1F6E
:109310005400FF1F5800FF1F6800FF1F6C00FF1F55
:109320007000FF1F7800FF1F7C00FF1F8000FF1FE1
:109330008400FF1F8800FF1FB800FF1FBC00FF1F35
:10934000C800FF1FDE00FF1F4C01FF1F5401FF1F5D
:109350005801FF1F4400FF1F4600FF1F4800FF1F6A
:109360004A00FF1F4C00FF1F6600FF1F4E00FF1F3B
:109370004F00FF1FA800FF1F109D0100109D01005E
:109380000CA8010018A80100000000000001000066
:109390000000704192017AFFFFFFFFFF0000000014
:1093A00000000000A000000086020000A5030000ED
:1093B0008C0C000000000100905F0100A0860100FD
:1093C00092010200400D0300FFFFFF01FFFFFF0FAE
:1093D00020000D2010004060100041600800606017
:1093E00008006160200062602000646020006B6003
:1093F00020006C60200071602000746020007760A5
:1094000020007A602000FF600000000002000300DE
:10941000070022003200F4010016FF17001AFF1B9C
:10942000FF7FFFFFFF000001020304050607080994
:109430002040FEFF00000080C0F2FCFF70A0FEFF95
:109440000000000000000000905F0100400D0300DC
:10945000FFFFFF7F0080FFFF00000000010002000F
:1094600004000800FF7F00008000000A24000000C4
:1094700003010000100007060C01000000000305B6
:1094800016010000000004050001000001000405B1
:1094900008010000000001060401000001000106AF
:1094A00005010000020001060101000000000206A3
:1094B00009010000410004060A0100000300010642
:1094C0000F010000420004060601000043000406EC
:1094D0001001000000000606110100001000070640
:1094E0000201000011000906120100003000090607
:1094F0000E010000310009060D01000032000906CE
:109500000B0100000000000813010000200000080B
:1095100014010000210000081501000022000008CD
:10952000070100004700040656312E3100000000FC
:1095300043313630563430310000000044657669DE
:1095400063652054797065004572726F72205265B0
:1095500067697374657200004D616E75666163744E
:109560007572657220446576696365204E616D652C
:10957000000000004D616E756661637475726572FE
:109580002048617264776172652056657273696FF5
:109590006E0000004D616E75666163747572657270
:1095A00020536F6674776172652056657273696FB8
:1095B0006E0000006E756D626572206F6620656ECC
:1095C000747269657300000056656E646F7220499D
:1095D0006400000050726F6475637420436F6465AB
:1095E000000000005265766973696F6E206E756DBC
:1095F0006265720053657269616C206E756D62659B
:10960000720000004E756D626572206F6620456EB7
:1096100074726965730000004D617070696E672037
:10962000456E7472792031004D617070696E6720EB
:10963000456E7472792032004D617070696E6720DA
:10964000456E7472792033004D617070696E6720C9
:10965000456E7472792034004D617070696E6720B8
:10966000456E7472792035004D617070696E6720A7
:10967000456E7472792036004D617070696E672096
:10968000456E7472792037004D617070696E672085
:10969000456E7472792038004D617070696E672074
:1096A000456E747279203900436F6D6D756E696314
:1096B0006174696F6E20547970652053796E6320F0
:1096C0004D616E616765722031000000436F6D6D02
:1096D000756E69636174696F6E205479706520538B
:1096E000796E63204D616E61676572203200000003
:1096F000436F6D6D756E69636174696F6E20547927
:1097000070652053796E63204D616E6167657220CC
:1097100033000000436F6D6D756E69636174696F2E
:109720006E20547970652053796E63204D616E61AF
:109730006765722034000000436F6D6D756E69635C
:109740006174696F6E20547970652053796E63205F
:109750004D616E6167657220350000004E756D6267
:109760006572206F662061737369676E656420524D
:109770007850444F0000000050444F204D617070FD
:10978000696E6720696E646578206F662061737307
:1097900069676E656420527850444F730000000082
:1097A0004E756D626572206F662061737369676EB6
:1097B000656420547850444F7300000050444F209B
:1097C0004D617070696E6720696E646578206F66A0
:1097D0002061737369676E656420547850444F004C
:1097E0004E756D626572206F662053796E63687284
:1097F0006F6E697A6174696F6E20506172616D6518
:10980000746572730000000053796E6368726F6E46
:1098100069736174696F6E2054797065000000008F
:1098200053686966742054696D65000053796E63EE
:1098300068726F6E697A6174696F6E2054797065B1
:109840007320537570706F72746564004D696E6932
:109850006D756D204379636C652054696D650000FA
:1098600043616C6320616E6420436F70792054699A
:109870006D6500004D696E696D756D2044656C61A4
:10988000792054696D650000476574204379636CE5
:10989000652054696D65000053796E63302043790B
:1098A0006C652054696D6500534D2D4576656E7469
:1098B000204D6973736564004379636C6520546956
:1098C0006D6520546F6F20536D616C6C000000005B
:1098D00053686966742054696D6520546F6F205316
:1098E000686F727400000000527850444F20546F2B
:1098F00067676C65204661696C6564004D696E69D7
:109900006D756D204379636C652044697374616E75
:10991000636500004D6178696D756D204379636CF6
:10992000652044697374616E636500004D696E69FA
:109930006D756D20534D2053796E632044697374A7
:10994000616E6365000000004D6178696D756D2082
:10995000534D2053796E632044697374616E63655F
:109960000000000053796E63204572726F72000030
:1099700053776974636820506172616D65746572B4
:109980007300000053746174757320616E64204528
:1099900072726F7220466C6167730000537570704D
:1099A0006C7920566F6C746167650000447269764B
:1099B00065722054656D7065726174757265000022
:1099C0004E756D4F66456E747269657300000000D8
:1099D0004D6F746F72506F6C657300004D617854F9
:1099E0006F727175650000004D617856656C6F632C
:1099F000697479004D6178416363656C6572617467
:109A0000696F6E0041637475616C43757272656E47
:109A10007400000052616D70546172676574437523
:109A20007272656E74000000505F506172616D6506
:109A300074657200495F506172616D657465720092
:109A400050495F546F727175655F4572726F720035
:109A500050495F546F727175655F4572726F725FC6
:109A600053756D0050495F466C75785F4572726F33
:109A70007200000050495F466C75785F4572726FE6
:109A8000725F53756D00000041637475616C5665BB
:109A90006C6F63697479000052616D705461726714
:109AA000657456656C6F6369747900004D6F746FEF
:109AB0007248616C74656456656C6F636974790093
:109AC00050495F56656C6F636974795F4572726F58
:109AD0007200000050495F56656C6F636974795F6E
:109AE0004572726F725F53756D000000416374754B
:109AF000616C506F736974696F6E000052616D70B4
:109B0000546172676574506F736974696F6E000099
:109B100050495F506F736974696F6E5F4572726F01
:109B20007200000054617267657452656163686514
:109B30006456656C6F6369747900000054617267E4
:109B400065745265616368656444697374616E63CA
:109B500065000000436F6D6D75746174696F6E20F0
:109B60004D6F64650000000056656C6F6369747921
:109B70002052616D70204D6F646500004163747503
:109B8000616C416E676C65004F70656E4C6F6F70F5
:109B900043757272656E7400496E76657273696F93
:109BA0006E000000496E746572706F6C6174696F4D
:109BB0006E0000005374657073506572526F74616B
:109BC00074696F6E000000004F6666736574000074
:109BD000446972656374696F6E000000496E697450
:109BE0004D6F646500000000496E697444656C61E6
:109BF00079000000496E697456656C6F6369747909
:109C000000000000456E61626C654272616B6543E5
:109C1000686F707065720000566F6C746167654C98
:109C2000696D69740000000048797374657265732A
:109C300069730000546865726D616C57696E646980
:109C40006E6754696D65436F6E7374616E74000066
:109C50004949744C696D69740000000049497453A6
:109C6000756D0000494974457863656564436F7597
:109C70006E74657200000000436C6561724949743E
:109C80004578636565646564466C61670000000043
:109C9000486F6D65204F6666736574204469737004
:109CA0006C6179004469676974616C20496E7075F4
:109CB0007473000053746F7265204178697320508B
:109CC0006172616D657465720000000048414C204E
:109CD00056657273696F6E00696E666F20310000A1
:109CE000696E666F20320000696E666F2033000077
:109CF000696E666F20340000696E666F2035000063
:109D0000696E666F203600004144435F494E5F3004
:109D1000000000004144435F53494E474C455F53A8
:109D200048554E54000000004144435F7068617321
:109D3000655F41004144435F70686173655F420045
:109D40004144435F56537570706C79004144435FE2
:109D500054656D7000000000436F6E74726F6C7715
:109D60006F726400537461747573776F726400006E
:109D7000517569636B2053746F70204F7074696FF5
:109D80006E20436F6465000053687574646F776E6E
:109D9000204F7074696F6E20436F6465000000008F
:109DA00044697361626C65204F7065726174696F9C
:109DB0006E204F7074696F6E20436F646500000001
:109DC00048616C74204F7074696F6E20436F6465D6
:109DD000000000004661756C74205265616374690F
:109DE0006F6E204F7074696F6E20436F6465000062
:109DF0004D6F646573206F66204F70657261746982
:109E00006F6E00004D6F646573206F66204F706544
:109E1000726174696F6E20446973706C61790000BF
:109E2000506F736974696F6E2044656D616E642054
